:020000040800F2
:1000000000000220F5F60008999A00089B9A000863
:100010009D9A00089F9A0008A19A0008000000001D
:10002000000000000000000000000000A39A00088B
:10003000A59A000800000000A79A0008A99A0008E5
:1000400039F7000839F7000839F7000839F70008D0
:1000500039F7000839F7000839F7000839F70008C0
:1000600039F7000839F7000839F700084D6600082D
:1000700039F7000839F7000839F7000839F70008A0
:1000800039F7000839F7000839F7000839F7000890
:1000900039F7000839F7000839F70008F59C00081F
:1000A00039F7000839F7000839F7000839F7000870
:1000B000A19C000839F7000839F7000839F7000853
:1000C00039F7000839F7000839F7000839F7000850
:1000D00039F7000839F70008099E000839F70008C9
:1000E00039F7000839F70008AD9A000839F7000819
:1000F00039F7000839F7000839F7000839F7000820
:1001000039F7000839F7000839F7000839F700080F
:1001100039F7000839F7000839F7000839F70008FF
:1001200039F7000839F7000839F7000839F70008EF
:1001300039F7000839F7000839F7000839F70008DF
:1001400039F7000839F7000839F70008DD9A000888
:1001500039F7000839F7000839F7000839F70008BF
:1001600039F7000839F7000839F7000839F70008AF
:1001700039F7000839F7000839F7000839F700089F
:0801800039F7000839F7000807
:1001880044A2050800000020A40B0020A80B0020B2
:10019800784F0020064B07481A68074B1A60074B30
:1001A80000221A70064B01221A7001F036BD00BFFA
:1001B800543C0020700E0020604200203C3C00208F
:1001C800F43B002008B5034801F027FD024B00224C
:1001D8001A7008BD00110020F43B002008B5054B3B
:1001E800012200201A7004F063FD0348BDE80840AE
:1001F80001F013BD78420020A41100202DE9F04140
:10020800144C204603F099F800201349134A02F0D1
:100218004BFE1349134A0746002002F045FE1249D7
:10022800124A0646002002F03FFED22105463A4611
:1002380023460A2002F050FFD22132462346FA20F4
:1002480002F04AFF5A20D2212A462346BDE8F0414F
:1002580002F042BFB80F0020E2910508CD01000866
:10026800EB910508E5010008F39105089D010008D8
:1002780008B5054B012200201A7004F019FD034847
:10028800BDE8084001F0C9BC78420020A411002054
:10029800044B054800221A70044B02221A7001F020
:1002A800BCBC00BF3C3C0020B80F0020F43B002041
:1002B80008B5034801F0B1FC024B00221A7008BDD2
:1002C80000110020F43B00202DE9F041144C204699
:1002D80003F033F800201349134A02F0E5FD1349EF
:1002E800134A0746002002F0DFFD1249124A06466B
:1002F800002002F0D9FDD22105463A4623460A20BD
:1003080002F0EAFED221324623465A2002F0E4FEE9
:10031800AA20D2212A462346BDE8F04102F0DCBEDD
:10032800700E0020E2910508B9020008FC9105084A
:10033800990200080592050879020008002008B50E
:1003480004F0B6FC064B00221A70064B1B78022BF1
:100358000CBF05480548BDE8084001F05EBC00BF79
:1003680078420020F43B0020B80F0020700E0020D7
:1003780010B5084C204602F0E0FF00200649074A65
:1003880002F092FDD22102462346E620BDE8104045
:1003980002F0A2BEEC1200200E92050845030008E8
:1003A80010B5074C4FF6E071206802F0D1F82068CC
:1003B800044902F07BF8BDE8104003F0F7B900BF2C
:1003C800A80B00201792050810B5074C4FF6E071EE
:1003D800206802F0BDF82068044902F067F8BDE81B
:1003E800104003F0E3B900BFA80B00202C920508C9
:1003F80010B5074C4FF6E071206802F0A9F82068A4
:10040800044902F053F8BDE8104003F0CFB900BF2B
:10041800A80B0020419205082DE9F04F774C85B0D4
:10042800FFF7BEFF002004F043FC23790BB9FFF768
:10043800DFFF6379714D53B928684FF6E07102F018
:1004480087F828686E4902F031F803F0AFF9A3790C
:100458000BB9FFF7B9FF694B5A79002A00F0C2803F
:100468001A79002A00F0BE80997900221A715A710F
:1004780001B19A71634BDFF8BCA1DFF8BC811A7037
:10048800614EDAF80010614CDFF8B0B1DFF8B091D6
:100498005F4F604D4FF4967006F049F9D8F8001098
:1004A8004FF4987006F043F931684FF49A7006F0EB
:1004B8003EF921684FF49C7006F039F9564A4FF41A
:1004C8009E701168019206F032F9DBF800104FF4C3
:1004D800A07006F02CF9D9F800104FF4A27006F0BD
:1004E80026F939684FF4A47006F021F929684FF409
:1004F800A67006F01CF9494B4FF4A87019680293CE
:1005080006F015F9DFF83CC14FF4AA70DCF80010CA
:10051800CDF80CC006F00BF9DFF808E14FF4AC7029
:10052800DEF8001006F003F9019AD4ED001A92EDF6
:10053800002A9AED000AD8ED000A96ED001A07F095
:100548001DFE029B9BED000A93ED002AD9ED000ADF
:1005580097ED001AD5ED001A07F01EFE9BED007A04
:10056800DAED007A2E49DDF80CC0029B019A77EE8D
:10057800677A99ED007AC1ED0A7AD8ED007A77EEBC
:10058800677A97ED007AC1ED0B7AD6ED007A77EEAF
:10059800677A95ED007AC1ED0C7AD4ED007A77EEA2
:1005A800677A93ED007AC1ED0D7ADCF80030134CD0
:1005B800CB63D2ED007A1B4A2068136877EE677A1E
:1005C8000B64C1ED0E7A4FF6E07101F0C1FF2068AF
:1005D800154901F06BFF07F02CFE03F0E7F813480C
:1005E80003F028F9FFF7DCFE002007F0E3FD1048D0
:1005F80005B0BDE8F04F01F010BB00BFA80B00200C
:1006080056920508F43B0020640E00204C0E002092
:10061800600E0020300E00205C0E0020340E0020FA
:10062800BC4500203C0E00206B920508809698007F
:1006380000110020480E0020500E0020580E002007
:10064800680E00206C0E002008B5002007F0B2FDEF
:100658000248BDE8084001F0E0BA00BF00110020E0
:100668002DE9F04F494D4A4E85B000244FF6FF78EA
:10067800284602F062FE4146224623464548009439
:10068800019401F029FF0427B060224623464FF663
:10069800E07141480097019401F01EFF2346306045
:1006A800414622463D480097019401F015FF3C4918
:1006B800F0603C4A204602F0F7FB3B493B4A0746BC
:1006C800204602F0F1FB3A493A4A8046204602F0B9
:1006D800EBFB3949394A8146204602F0E5FB3849A7
:1006E800384A8246204602F0DFFB3749374A8346BC
:1006F800204602F0D9FB36490390364A204602F0DC
:10070800D3FB21468446B268CDF808C02B46204664
:1007180002F0E2FC214632682B467D2002F0DCFC28
:100728002321F2682B46B42002F0D6FC37213A4642
:100738002B46FA2002F0D0FC692142462B46FA20CB
:1007480002F0CAFC9B214A462B46FA2002F0C4FC60
:10075800C82152462B46322002F0BEFC5A462B4690
:10076800C8216E2002F0B8FCDDF808C0C821624636
:100778002B46AA2002F0B0FC039AF020C8212B4691
:1007880005B0BDE8F04F02F0A7BC00BF5C10002028
:10079800A80B00207F920508569205088792050845
:1007A8008F920508B909000897920508650900089D
:1007B8009F92050829120008A7920508350F00081E
:1007C800AE920508F90E0008B59205085106000812
:1007D800BC9205082104000818B9044B93ED000ADF
:1007E8007047034B93ED000A704700BF480E002086
:1007F800580E002018B9044B93ED000A7047034BBC
:1008080093ED000A704700BF500E0020680E0020CC
:1008180018B9044B93ED000A7047034B93ED000A97
:10082800704700BF640E0020600E002018B9044B0A
:1008380093ED000A7047034B93ED000A704700BF21
:100848004C0E0020300E002018B9044B93ED000A1E
:100858007047034B93ED000A704700BF5C0E002001
:10086800340E002070B52DED028B9FED108A0446E2
:100878000E460A25F0EE488A07F042F978EE808A9B
:1008880007F044F90A4838EE008A02F0D3FF013D28
:10089800F2D1F2EE047AC8EEA78A88EE278AC4ED70
:1008A800008A86ED008ABDEC028B70BD0000000056
:1008B800A086010010B50E4C0E4802F0BBFF04F1F3
:1008C800140104F11000FFF7CDFF4FF6E07004F0BB
:1008D800C3F9FFF779FD5E220023DF206E2104F0C3
:1008E800CBFA01232371044B1A68044B1A6010BD1C
:1008F800A80B0020A0860100543C00206042002084
:1009080010B5002007F072FC0F4B104C186010480F
:1009180002F090FF04F11C0104F11800FFF7A2FF98
:100928004FF6E07004F098F9FFF762FD5E220023AD
:10093800DF203C2104F0A0FA01236371054B1A68FB
:10094800054B1A6010BD00BF3C0E0020A80B00200C
:10095800A0860100543C002060420020104908B5E0
:1009680001F120002431FFF77DFF4FF6E07004F01D
:1009780073F9FFF729FDB7206E215E22002304F0EA
:100988007BFA084B1A68084B1A60084B02224FF092
:10099800804001211A70BDE808400DF0DEB800BFA4
:1009A800A80B0020443C002060420020E00C0020FE
:1009B80008B5002007F00EFC114B1860114802F032
:1009C80039FF114901F128002C31FFF74BFF4FF691
:1009D800E07004F041F9FFF70BFDB7203C215E22DF
:1009E800002304F049FA094B1A68094B1A60094BAD
:1009F80001214FF080401970BDE808400DF0ADB8F6
:100A08006C0E0020A0860100A80B0020443C0020AA
:100A180060420020E00C00202DE9F84380462DEDCF
:100A2800068B10EE100A11EE905A11EE109A10EE85
:100A3800904A0DF0E3FF064648460F460DF0DEFFEC
:100A480041EC100B41EC180B0FF09AFF304653ECB9
:100A5800102B39460EF026F80EF006FBB0EE480AC9
:100A6800F0EE680A454B186009EE900A10F088F815
:100A7800304653EC102B39460EF014F80EF0F4FA09
:100A88003F4B09EE100A186020460DF0B7FF0646E6
:100A980028460F460DF0B2FF41EC100B41EC1A0B43
:100AA8000FF06EFF304653EC102B39460DF0FAFF6D
:100AB8000EF0DAFAB0EE4A0AF0EE6A0A314B186024
:100AC80008EE100A10F05CF8304653EC102B39464B
:100AD8000DF0E8FF0EF0C8FA08EE900A79EE688A81
:100AE80039EEC88A9FED287A68EEA87A48EE087A27
:100AF80028EE078A9FED257A68EE878A88EE278A8E
:100B0800234B1860C8EEA78A68EE897A17EE900A18
:100B18000DF074FF00221F4B0DF012FE68EE297ACB
:100B2800044617EE900A0D460DF068FF02460B4684
:100B3800204629460DF002FE68EEA99A0EF094FAB6
:100B480058EE499AB8F1000F09D1134B83ED008A8A
:100B5800124BC3ED008A124B1860124B08E0124B7F
:100B680083ED008A114BC3ED008A114B1860114BBD
:100B7800C3ED009ABDEC068BBDE8F883540E002047
:100B8800400E0020380E002000004842000048C2F5
:100B9800440E002000004940480E0020500E00205E
:100BA800640E00204C0E0020580E0020680E002015
:100BB800600E0020300E00202DE9F84380462DED10
:100BC800068B10EE100A11EE109A11EE905A10EEE4
:100BD800904A0DF013FF064648460F460DF00EFFEB
:100BE80041EC100B41EC190B0FF0CAFE304653ECE8
:100BF800102B39460DF056FF0EF036FAB0EE490AC2
:100C0800F0EE690A544B186008EE100A0FF0B8FFAE
:100C1800304653EC102B39460DF044FF0EF024FA01
:100C28004E4B08EE900A186020460DF0E7FE064687
:100C380028460F460DF0E2FE41EC100B41EC1A0B72
:100C48000FF09EFE304653EC102B39460DF02AFF6C
:100C58000EF00AFAB0EE4A0AF0EE6A0A404B186043
:100C680009EE900A0FF08CFF304653EC102B3946F2
:100C78000DF018FF0EF0F8F909EE100A78EEC98A9F
:100C8800384B38EE698A28EEA8AA186008EE08AA38
:100C9800B8F1000F0CD1344B18680DF0AFFE2CA33F
:100CA800D3E900230DF0FEFE304B04460D460BE061
:100CB8002F4B18680DF0A2FE25A3D3E900230DF0F1
:100CC800F1FE2C4B04460D4618680DF097FE0246BF
:100CD8000B46204629460DF0E5FE0EF0C5F9DFED7E
:100CE800267A06EE900A68EEA77A9FED247A67EED8
:100CF800A67A58EE077A87EE8AAA1AEE087A6AEE7A
:100D0800297AC7EE288A68EEA99A58EE897A5AEEA7
:100D1800499AB8F1000F0AD1194B83ED00AA194B73
:100D2800C3ED008A184BC3ED007A184B09E0184B45
:100D380083ED00AA174BC3ED008A174BC3ED007A69
:100D4800164BC3ED009ABDEC068BBDE8F88300BFD7
:100D58001F85EB51B81E1940540E0020400E00208C
:100D6800380E0020440E00206C0E00205C0E00207F
:100D78003C0E0020340E002000401C450000484274
:100D8800480E0020500E0020640E00204C0E00205B
:100D9800580E0020680E0020600E0020300E002043
:100DA8002DE9F74F044610EE109A10EE907A11EEE6
:100DB800105A11EE906A12EE108A002842D14FF6AE
:100DC800E07003F049FF48460DF018FE82463846A9
:100DD8008B460DF013FE5246CDE900015B464049B3
:100DE800404812F003FB3F4A23460520372104F010
:100DF80061F828460DF002FE824630468B460DF01B
:100E0800FDFD5246CDE900015B463749354812F0F1
:100E1800EDFA344A23460520692104F04BF8404690
:100E28000DF0ECFD2CA3D3E900230DF03BFE0246A8
:100E38000B462C482D4912F0D9FA05209B21294A46
:100E4800234641E04FF4FC6003F006FF48460DF0EE
:100E5800D5FD824638468B460DF0D0FD5246CDE989
:100E680000015B461E491F4812F0C0FA1D4A0023C4
:100E78000520502104F01EF828460DF0BFFD044659
:100E880030460D460DF0BAFD2246CDE900012B464D
:100E98001549144812F0AAFA124A002305208221A3
:100EA80004F008F840460DF0A9FD0BA3D3E9002390
:100EB8000DF0F8FD02460B460A480C4912F096FA66
:100EC800084A0520B421002303B0BDE8F04F03F021
:100ED800F1BF00BFAFF30080000000A2941A6D427A
:100EE800C3920508D80B0020D4920508E59205089E
:100EF8000C4A0D4B92ED092A92ED050AD2ED060A2D
:100F080092ED071AD2ED081A126C012083ED132A0C
:100F180083ED140AC3ED150A83ED161AC3ED171AEB
:100F28001A663DE7BC450020A80B00200C4A0D4B73
:100F380092ED042A92ED000AD2ED010A92ED021A0E
:100F4800D2ED031AD26B002083ED132A83ED140A25
:100F5800C3ED150A83ED161AC3ED171A1A661FE7B3
:100F6800BC450020A80B0020F0B52DED088B0446E9
:100F780083B06B4B002851D193ED0B1AD3ED091AAE
:100F880093ED0A0AD3ED080AFFF746FD654BD3ED4A
:100F9800009A654B93ED008A644BD3ED008A644B4D
:100FA800684601A993ED00AAFFF75CFC00980DF0D4
:100FB80025FD064601980F460DF020FD41EC100B6B
:100FC80041EC1B0B0FF0DCFC304653EC102B394680
:100FD8000DF068FD0EF048F8B0EE4B0AF0EE6B0A23
:100FE80009EE100A0FF0CCFD304653EC102B3946B1
:100FF8000DF058FD0EF038F807EE100A68EE077A83
:1010080028EE098A59EE897A09EE878A204677EE12
:10101800A88A38EE0A8A07F0DDF851E093ED071A3E
:10102800D3ED051A93ED060AD3ED040A0120FFF764
:10103800F3FC404BD3ED009A3F4B93ED008A3F4BB6
:10104800D3ED008A3E4B684601A993ED00AAFFF74D
:1010580009FC00980DF0D2FC044601980D460DF0ED
:10106800CDFC41EC100B41EC1B0B0FF089FC20462A
:1010780053EC102B29460DF015FD0DF0F5FFB0EEE1
:101088004B0AF0EE6B0A09EE100A0FF079FD2046C4
:1010980053EC102B29460DF005FD0DF0E5FF07EE8A
:1010A800100A68EE077A28EE098A59EE897A09EE5D
:1010B800878A002077EEA88A38EE0A8A07F096F821
:1010C800F1EE487A28EE088A08EEA88A064687EEE6
:1010D800888A18EE100A0DF091FC07EE106AF8EEF7
:1010E800C77A044617EE900A0D460DF087FC0AA34E
:1010F800D3E900230DF0D6FC02460B4620462946CC
:101108000DF0FAFD0DF0B0FF00EE100A03B0BDECD3
:10111800088BF0BDAFF300801F85EB51B81E194056
:10112800A80B0020480E0020500E0020640E00205E
:101138004C0E0020580E0020680E0020600E002083
:10114800300E002070B50120FFF70EFF274C284D08
:101158004FF6E07084ED000A03F07EFD5E22A021C8
:101168000023DF2003F088FE0126002095ED0A0AFF
:10117800D5ED080A95ED0B1AD5ED091AAE71FFF7F2
:101188001BFD304695ED060AD5ED040A95ED071AC4
:10119800D5ED051AFFF710FD164B93ED000A164B17
:1011A800D3ED000A154B93ED001A154BD3ED001A39
:1011B800144B002093ED002AFFF7F2FD124B93ED3C
:1011C800000A124BD3ED000A114B93ED001A114B94
:1011D8003046D3ED001A94ED002AFFF7E1FDFFF742
:1011E800DFF80D4B1A680D4B1A6070BD340E0020E5
:1011F800A80B0020480E0020500E0020640E00208E
:101208004C0E00205C0E0020580E0020680E0020B6
:10121800600E0020300E0020543C00206042002068
:1012280008B50020FFF7A0FE0D4B4FF6E07083EDE8
:10123800000A03F011FDB720A0215E22002303F06D
:101248001BFE084B1A68084B1A60084B03224FF024
:10125800804001211A70BDE808400CF07EBC00BF38
:101268005C0E0020443C002060420020E00C00207E
:101278002B4B2C48062210B51A704FF6E07400F07C
:10128800CCFC0020214607F0ADFA3120214607F0BA
:10129800A9FA6320214607F0A5FA9520214607F010
:1012A800A1FAC7204FF4FC6107F09CFA4EF29C703B
:1012B80003F0D2FC0520012100231B4A03F0FAFDAC
:1012C800052020210023194A03F0F4FD05205221AE
:1012D8000023174A03F0EEFD842100230520154A58
:1012E80003F0E8FD4FF4F06003F0B6FCB621124AB3
:1012F8000023052003F0DEFD4FF6FF7003F0ACFC81
:101308008720DC210D4A002303F0D4FD0C4B00227A
:101318001A6008F0B4FB0B4B01221A7010BD00BF15
:101328007842002034140020F39205082A93050817
:1013380022930508F792050844980508F9920508CC
:101348005C3C00203C3C002038B53C4B3C483D4DC3
:1013580007221A704FF6E07400F05FFC0020214667
:1013680007F040FA3120214607F03CFA6320214675
:1013780007F038FA9520214607F034FA2146C720AD
:1013880007F030FA4EF29C7003F066FC052001214C
:1013980000232D4A03F08EFD0520202100232B4A2F
:1013A80003F088FD052052210023294A03F082FD1D
:1013B800052084210023274A03F07CFD0520B6215F
:1013C8002A46002303F076FD40F213144FF4F06030
:1013D80003F042FC204601211F4A002303F06AFD66
:1013E800204620211D4A002303F064FD2046522197
:1013F8002A46002303F05EFD20468421184A002374
:1014080003F058FDB621174A0023204603F052FD89
:101418004FF6FF7003F020FC7D20DC21124A0023E8
:1014280003F048FD114B00221A6008F028FB104A0F
:10143800012313700F4A137038BD00BF7842002093
:10144800341400202D970508FE920508029305081C
:101458000693050809930508129305080E930508D5
:101468000D93050811930508169305085C3C0020A8
:101478003C3C0020E443002038B52E4B2E48052480
:101488001C704FF6E07500F0C8FB0020294607F0F5
:10149800A9F92720294607F0A5F94F20294607F082
:1014A800A1F97720294607F09DF99F20294607F0E2
:1014B80099F9C720294607F095F94EF29C7003F078
:1014C800CBFB0121002320461C4A03F0F3FC162124
:1014D800002320461A4A03F0EDFC3E210023204653
:1014E800184A03F0E7FC662100232046164A03F059
:1014F800E1FC8E2100232046144A03F0DBFCB621D0
:10150800134A0023204603F0D5FC4FF6FF7003F082
:10151800A3FB7D20DC210F4A002303F0CBFC0E4BFC
:1015280000221A6008F0ABFA0C4A012313700C4A27
:10153800137038BD78420020341400202D97050818
:101548002193050825930508299305082D93050877
:1015580031930508359305085C3C00203C3C00208D
:10156800E44300203C4B3D48042270B51A704FF606
:10157800E07400F052FB0020214607F033F93120D7
:10158800214607F02FF96320214607F02BF9952013
:10159800214607F027F9324E324D2146C72007F081
:1015A80021F94EF29C7003F057FB0520012100231E
:1015B800324603F07FFC0520202100232A4A03F04D
:1015C80079FC052052210023284A03F073FC0520EA
:1015D80084210023264A03F06DFC0520B6212A4603
:1015E800002303F067FC40F213144FF4F06003F09B
:1015F80033FB204601213246002303F05BFC2046E2
:1016080020211C4A002303F055FC204652212A467B
:10161800002303F04FFC20468421174A002303F0DF
:1016280049FCB621154A0023204603F043FC4FF637
:10163800FF7003F011FB7D20DC21114A002303F029
:1016480039FC104B00221A6008F019FA0E4A0123DF
:1016580013700E4A137070BD7842002034140020B5
:10166800569305082D9705084193050851930508D9
:10167800469305084B9305085093050855930508AC
:10168800599305085C3C00203C3C0020E4430020C2
:10169800F8B5344B3448354F354E03221A704FF69F
:1016A800E07400F0BAFA0020214607F09BF86320A6
:1016B800214607F097F8B3204FF4F06107F092F84D
:1016C8002146C72007F08EF84FF6FF7003F0C4FAE2
:1016D8004EF29C75DC2100237D20264A03F0EAFBAC
:1016E800284603F0B9FA0520012100233A4603F001
:1016F800E1FB0520522100231F4A03F0DBFBB62142
:1017080000230520324603F0D5FB40F213144FF4B2
:10171800F06003F0A1FA012120463A46002303F0C5
:10172800C9FB522120460023324603F0C3FBB621F1
:10173800124A0023204603F0BDFB284603F08CFA2A
:101748000520A2210E4A002303F0B4FB0D4B002212
:101758001A6008F094F90C4A012313700B4A1370AD
:10176800F8BD00BF784200203414002073930508A8
:101778002D970508649305086E930508729305086C
:10178800329305085C3C00203C3C0020E4430020E8
:1017980008B5084B084802221A7000F03EFA06F015
:1017A80019FF064B00221A6008F069F9044B012260
:1017B8001A7008BD78420020341400205C3C0020D8
:1017C8003C3C0020002008B503F072FA064B0022CA
:1017D8001A70064B1B78022B0CBF05480548BDE85C
:1017E800084000F01ABA00BF78420020F43B0020FD
:1017F800B80F0020700E00202DE9F14F2D4C204627
:1018080001F09BFD00202C492C4A01F04DFB2C498E
:101818002C4A8146002001F047FB2B492B4A0746FA
:10182800002001F041FB2A492A4A0646002001F01F
:101838003BFB2949294A0546002001F035FB284988
:10184800284A8046002001F02FFB2749274A824674
:10185800002001F029FBD22183464A462346E62090
:1018680001F03AFC28203A462346014601F034FCB0
:10187800462132462346282001F02EFC64212A46C0
:101888002346282001F028FC8221424623462820AE
:1018980001F022FC524623462820A02101F01CFC1E
:1018A80028205A46BE21234601B0BDE8F04F01F07A
:1018B80013BC00BFA41100200E920508CD17000824
:1018C8007793050899170008649305089916000886
:1018D800599305086D1500088293050881140008BE
:1018E8008D93050851130008F9920508791200082C
:1018F800034B01224FF4FC601A7003F0ADB900BF2E
:10190800D80C00200B4B10B5002420461C7003F0A7
:10191800CFF906F0CBFF06F089F9074B1C70074B8F
:1019280001221A7006F0BCFF0548BDE8104000F01F
:1019380074B900BFD80C002078420020F43B002086
:10194800700E00200A4B10B5002420461C7003F0CE
:10195800AFF906F0ABFF074B1C70074B02221A7059
:1019680006F09EFF0548BDE8104000F056B900BFDC
:10197800D80C002078420020F43B0020B80F00204B
:1019880008B5064B0020187003F092F9044B05487F
:1019980003221A70BDE8084000F03FB9D80C0020B7
:1019A800F43B00205C1000200C4B10B500220C4CBE
:1019B8001A7006F07BFF04F007F906F040FC06F009
:1019C8006FFF20684FF6E07100F0C2FD20680549FE
:1019D80000F06CFDBDE8104001F0E8BED80C002016
:1019E8000C0C0020979305080E4B002210B51A70B6
:1019F8000088C83880B2042805D90B480B4A0C4B1C
:101A0800872102F0FBF80B4CC0B204F067F920689C
:101A18004FF6E07100F09CFD20680749BDE81040D2
:101A280000F044BDD80C0020AB930508BCD20308D5
:101A3800CB9305080C0C0020FC9305082DE9F04F0A
:101A48005848594D87B0002401F077FC4FF6FF71D4
:101A58002246234655480094019400F03DFD042693
:101A680007464FF6E07122462346514800960194F6
:101A780000F032FD4FF6E0718046224623464D487D
:101A88000096019400F028FD4FF6FF71814622462A
:101A9800234649480096019400F01EFD234628601D
:101AA8004FF6FF71224645480096019400F014FD58
:101AB80043496860434A204601F0F6F94249434ADF
:101AC8008246204601F0F0F94149424A83462046C1
:101AD80001F0EAF940490390404A204601F0E4F950
:101AE8003F4904903F4A204601F0DEF93A46059006
:101AF80021462C4B204601F0EFFA21464246294B5D
:101B0800C82001F0E9FA0A214A46264BC82001F00C
:101B1800E3FA2A68234B6421782001F0DDFA782063
:101B28006A68204B014601F0D7FAC8250526282700
:101B3800E0B204F003F82C4A0146284601F0B4F953
:101B480094FBF6F106FB114179431E31024689B236
:101B58000020144B0134013501F0BEFA042CADB25B
:101B6800E6D1D221524605200E4B01F0B5FAD2211A
:101B78005A464C200B4B01F0AFFAD221039A094B7D
:101B88009C2001F0A9FAD221049A064BEC2001F01E
:101B9800A3FA059A034BEC20B42107B0BDE8F04F37
:101BA80001F09ABA001100200C0C00200C940508D2
:101BB80016940508239405082E940508189205081C
:101BC80042940508B11900084A94050889190008C3
:101BD800539405084D1900085C9405080D19000870
:101BE80065940508F9180008F119000808B500F00F
:101BF80043FAFEF703FBFEF733FDFEF765FBFFF73D
:101C0800FBFDFFF71BFFFEF7B3FB00F0DBFA00F06C
:101C1800D9F8BDE8084000F0A1B910B5044628B9C4
:101C28000F48104A104B452101F0E8FF0F4B186888
:101C3800844213D010B1C36900219847002003F0F3
:101C480037F8002003F01EF84FF6FF7003F004F891
:101C5800E369204601219847044B1C6010BD00BF72
:101C68006E940508CBD203088A940508140C00204A
:101C78000048D2E7001100204FF6FF7070474FF67A
:101C8800FF70704713B5002944D04FF2DE7003F09F
:101C98000FF8002003F0D6F80F2002F0DDFF1E4CED
:101CA8001E4A412101230A2003F004F9042003F00D
:101CB800C9F8236828209621042B21DC0123184A1F
:101CC80003F0F8F801A90DF10602206803F078FB8B
:101CD8000F2002F0C1FFBDF80400BDF8061014384B
:101CE8002822002380B202F0E7FFBDF80610BDF8F5
:101CF8000400143989B22822012302F0DDFF09E02B
:101D0800084A012303F0D6F81E20A521064A01231C
:101D180003F0D0F81CBD00BF180C00209A940508E9
:101D2800AD940508C9940508DF94050837B51E4C1D
:101D38002368042B05462BDC01A80DF1060103F0EE
:101D48003DFBBDF80630BDF804201849042009F011
:101D580009FF2368002B04DA1548164A164B592147
:101D680005E0042B05DD1248124A144B5A2101F0F4
:101D780045FF04EB8302BDF8041001339180BDF8E0
:101D880006102360052BD18008D1201D03F098FB95
:101D980000230B482360FFF740FF03E0284601219A
:101DA800FFF770FF3EBD00BF180C0020F694050831
:101DB8003B950508DDD203085D950508749505086F
:101DC8004812002037B50B4C204601F0B6FA0A4BF2
:101DD8000A49009300250120094A0A4B019501F0A0
:101DE80054F9294602462346284603B0BDE8304048
:101DF80001F072B9140F00208D1C0008811C000826
:101E0800871C0008351D00084FF6FF7070474FF615
:101E1800FF7070471FB54FF6E07002F049FF0020D1
:101E280003F010F80F2002F017FF0021294A2A4C6E
:101E380001230A2003F03EF8002002F00DFF0420E1
:101E480003F000F80A201921244A012303F032F88C
:101E58002521234A01230A2003F02CF81F2002F031
:101E6800FBFE01230A2037211E4A03F023F82378BA
:101E780073B301231E2096211B4A03F01BF86288C6
:101E88001A49684611F0B2FA01231E20A2216A46B7
:101E980003F010F8A2881649684611F0A7FAAE2197
:101EA8006A4601231E2003F005F80F2002F0D4FE35
:101EB8006088A188143880B22822002302F0FCFE32
:101EC800A1886088143989B22822012302F0F4FE1F
:101ED8001FBD00BFA2950508300C0020B495050869
:101EE800D4950508F4950508179605082996050858
:101EF8003696050801B18DE7704713B50DF1060157
:101F080001A803F00FFA144B01221A705988BDF882
:101F18000420891A0E311C2919460AD89C88BDF854
:101F28000600201A0E301C2803D8996801319960E0
:101F380001E000238B60084B9968012905DD002228
:101F48009A601A70FFF794FE05E05A80BDF80620E3
:101F58009A80FFF75FFF1CBD300C002037B50B4C93
:101F6800204601F0EAF90A4B0A49009300250120AE
:101F7800094A0A4B019501F088F82946024623468A
:101F8800284603B0BDE8304001F0A6B8481200204A
:101F9800FD1E0008111E0008171E0008031F000878
:101FA80008B5164B00221A6007F069FD144B1A6831
:101FB800144B1A6007F0D8FC134B1B78023B052B17
:101FC80015D8DFE803F00306090F120CFFF7E0FB52
:101FD8000DE0FFF75DFB0AE0FFF7C4FA07E0FFF743
:101FE800B3F904E0FFF748FA01E0FFF741F907F019
:101FF800B3FC064B01221A7008BD00BF5C3C0020F0
:10200800543C00206042002078420020E443002035
:1020180038B5104B104D00241C70104B1C7007F085
:102028002EFD0F4B4FF0FF321A600E4B1A680E4B05
:1020380020461A6002F03CFE0C4B1B78022B0CBFAA
:102048000B480C48FFF7E9FD2C70BDE8384007F055
:1020580083BC00BF78420020E44300203C3C0020C1
:102068005C3C0020543C002060420020F43B0020EF
:10207800B80F0020700E002070B5124C204601F0F9
:102088005CF900200146224600F086FA00200E493D
:102098000E4A00F009FF0E490E4A0646002000F0DD
:1020A80003FFD2210546324623464FF4827001F0E1
:1020B80013F8DC20D2212A462346BDE8704001F0FF
:1020C8000BB800BF34140020B59205081920000889
:1020D80043960508A91F000810B5064C4FF6FF7176
:1020E800206800F035FA044B20681968BDE81040F4
:1020F80000F0DCB93C0C00209801002008B5002055
:1021080002F0D6FD054B1868054B196800F0CEF9AA
:102118000448BDE80840FFF780BD00BF3C0C002024
:10212800940100200011002008B5FFF7D5FF00201A
:10213800014605F005FFBDE8084001F037BB0088FF
:10214800A0F5C87080B2092808B505D90748084A1B
:10215800084B8F2101F052FD074B1880074BFF21D8
:10216800197005F0EDFEBDE80840B5E7479605088B
:10217800EFD203086A960508D8140020DA14002064
:102188000088A0F5967080B2092808B505D90848D6
:10219800084A094B832101F031FD084B1880084B90
:1021A8000121197005F0CCFEBDE8084094E700BF96
:1021B8004796050804D303086A960508D814002032
:1021C800DA1400202DE9F34100243A483A4D01F091
:1021D800B4F8224623464FF6FF713848009401941C
:1021E80000F07AF904262246234607464FF6FF7187
:1021F80033480096019400F06FF923462860224680
:102208004FF6FF712E480096019400F065F92D49AC
:1022180068602D4A204600F047FE2C492C4A0646A5
:10222800204600F041FE214680463A462046214B92
:1022380000F052FF2A681F4B2046282100F04CFF6F
:102248003246D2211B4B5A2000F046FFAA20D22149
:102258004246184B00F040FF0F254FF4967440F2A9
:10226800351620461B491C4A00F01EFE0134024662
:10227800782128460F4BA4B2233500F02DFFB44235
:10228800ADB2EED10F254FF4C87440F2991620462E
:102298001249134A00F008FE013402469B212846E1
:1022A800044BA4B2233500F017FFB442ADB2EED10F
:1022B800BDE8FC81901300203C0C00209B9605088B
:1022C80029920508A796050831210008B096050847
:1022D80005210008B996050889210008BB9605085C
:1022E8004721000808B508B143682BB90348044AD8
:1022F800044B9B2101F082FC586908BDBD96050876
:1023080018D30308DF96050808B5FFF7EBFF8068C8
:10231800123080B208BD08B5FFF7E4FF4068063008
:1023280080B208BD2DE9F84F04468846FFF7DAFF6A
:102338006689E589074606F1030905F10F0AB8F130
:10234800000F1FD01F2002F087FC2046FFF7DCFF9C
:1023580083462046FFF7DFFF294603465FFA8BF2E4
:10236800F0B202F0ADFC042002F06CFD0B364FF623
:10237800FF70033502F070FCB0B2A9B23A680123CD
:1023880002F098FD3D69204641464A465346A84713
:10239800BDE8F88F13B504460DF1060101A802F057
:1023A800C1FF2046FFF79EFF6389BDF80410BDF802
:1023B8000620C91AE389D21A0339C3680F3A20469E
:1023C80098471CBDF7B5044614200D4616461F460F
:1023D80010F09AFC089BC7600361064B0649074A40
:1023E80080E8700000930190054B002000F04DFE3E
:1023F800FEBD00BF2D2300081F230008112300087D
:102408009D230008704708B508B143682BB90448F4
:10241800044A054BAD2101F0F1FB586908BD00BF26
:10242800FE96050830D30308DF960508F8B505467B
:102438000E46FFF7E8FF836B04461BB1284631467A
:10244800984700E018466F8994F83C30ED890EB93A
:10245800034310D0208E02F0FFFB608E02F012FCC6
:1024680094F8350002F0EEFC94F8343038462946EA
:10247800224602F01FFD002384F83C30F8BD08B561
:10248800FFF7C1FF90F83500BDE8084002F0EFBC47
:1024980038B5FFF7B8FF044611F02EF8054694F852
:1024A800350002F0DFFC684380B238BD38B50D4610
:1024B800FFF7A9FF29462E22044611F04DF850B126
:1024C800204629462E2211F099F8002384F82E3050
:1024D800012384F83C3038BD2DE9F74307464020F6
:1024E8000E461546984610F00FFC044628B91148C8
:1024F800114A124B4E2101F081FB114B114A12492E
:102508008DE818000020114B00F0BFFD39468146C8
:10251800FFF7CCFF9DF82830268684F835300B9BD2
:102528006586A363002384F8348084F83C304846E9
:10253800BDE8FE83FE96050848D303081C970508E6
:102548003524000887240008992400080D24000871
:1025580010B50C46FFF757FF0123048680F83C307E
:1025680010BD00BF4FF4A0707047C8207047704777
:10257800074B1B78022B07B508D1064B1B78022B9B
:1025880004D001A80DF1060102F0CCFE0EBD00BF7B
:10259800E44300207842002073B50A4B06460D46F6
:1025A8001446009300200849084A094B019000F09E
:1025B8006CFD294602462346304602B0BDE870400D
:1025C80000F08ABD772500086D25000873250008EE
:1025D8007925000813B502AB03E90600436843B147
:1025E800027C0124082A9C7004D11B692146984763
:1025F80000E01C4620461CBD30B500282BD0058BBA
:10260800002425E0036A1A7C012A05D15B681A8830
:102618008A421BD1187F30BD052A06D15B681A880B
:102628008A4213D193F82C0030BD032A06D15B6887
:102638001A888A420AD193F8250030BD062A05D1A6
:102648005B681A888A4201D1D87A30BD01340430D7
:10265800AC42D7D3002030BD08B181750120704746
:10266800F8B504460D46D0B1E175D0F898309847D2
:10267800012D0DD12746002606E0F86900F1080271
:10268800436906CA98470136238B04379E42F4D320
:10269800D4F898302046294698470120F8BDF8BD5F
:1026A800F8B50546084617460E4610F025FF013FC7
:1026B800B84234BF04463C463CB12846314622461F
:1026C80010F09CFF00232B55F8BD2C70F8BDF7B512
:1026D800044600200090019000296CD00E8B68E021
:1026E80000F1080351F823301D7C042D04D15D68E6
:1026F8002D88954247D0013000F1080351F8233066
:102708001D7C012D04D15D682D8895423BD0013098
:1027180000F1080351F823301D7C052D04D15D68B4
:102728002D8895422FD0013000F1080351F823304D
:102738001D7C032D04D15D682D88954223D001307E
:1027480000F1080351F823301D7C022D04D15D6887
:102758002D88954217D0013000F1080351F8233035
:102768001D7C072D04D15D682D8A95420BD0013060
:1027780000F1080351F823301D7C062D08D15D684F
:102788002D88954203D103F10801204615E0013058
:1027980000F1080351F823502B7C082B09D16F68EE
:1027A8003F88974204D105F1080120461A4605E002
:1027B8000130B04294D320466946082210F054FDF7
:1027C8002046FEBDF8B505460F461646002830D00F
:1027D8004388032B2FD0202010F096FA04460028B7
:1027E8002BD040F80C5B39460C22FFF759FF182014
:1027F800E66110F089FA0646B8B102230374012392
:1028080063760F4B446063600E4BA360002323760E
:102818006B8805EB830201339BB2012B50606B8000
:102828000CD16A685268137608E0204610F074FAF2
:1028380004E0064602E0002600E006463046F8BD01
:1028480094520408324F040837B5456802AB03E9CF
:1028580006003DB3037C0124042B85F8314022D1C6
:10286800688E02F0F9F995F8300002F0EBFA95F865
:10287800343043B9BDF80200BDF80610AA1C23463F
:1028880002F018FB0FE0012B03D1084840F2395140
:1028980004E0022B07D1054840F24151044A054B98
:1028A80001F0ACF92C4620463EBD00BF2F97050825
:1028B800081E04082D970508F8B504460F46164665
:1028C80010B3838A0A2B20D0202010F01DFA054669
:1028D800E8B14460102200F108003946FFF7E0FE35
:1028E8004FF6FF73A08A2B801F236B8000232B7663
:1028F800831D013080B20128EE6144F82350A08284
:1029080007D1A3691876F8BDF8BD0020F8BD0120ED
:10291800F8BD0120F8BD2DE9F0411D464B1C984239
:1029280080460C4617460CDD95420ADC013208F158
:1029380001035B1A521BC8B2D2B29BB2294602F0FD
:10294800BDF9A8F10208BDF81800C4EB080802F0A8
:1029580083F901261FFA88F808E0A919601C80B2DB
:1029680089B24246002302F0A7F901367B1B9E423A
:10297800F3D3BDE8F081F8B5C7B2144638461E4611
:102988000D4602F09FF9621E92B23846294602F0BF
:1029980099F9304602F060F9022606E0A21B92B2CD
:1029A8003846294602F08EF90136A642F6D3F8BD1C
:1029B80070B5044600F11E003C22002380B20D468B
:1029C80002F07AF91E3DA9B220463C220123BDE857
:1029D800704002F071B970B5044601380322002333
:1029E80080B20D4602F068F9013DA9B220460322E3
:1029F8000123BDE8704002F05FB9F7B5089D2E7B52
:102A0800EF7A1C463604AB7A06EB0726F618431A0B
:102A1800687B06EB00602D1800200190121B084609
:102A28002146009501F098FEFEBD30B5456885B099
:102A380004AB03E906007DB101242C736D68BDF871
:102A48000800BDF80A109DF80C209DF80E3000957E
:102A5800FFF7D3FF204600E0284605B030BD2DE93A
:102A6800F04385B004AB03E906004468BDF808608C
:102A7800BDF80C70002C41D0012384F8263094F85E
:102A880025300BB9A26800E06268FFB2BDF80A10F1
:102A98009DF80E30009230463A46FFF7AEFF04F13B
:102AA8000C08022002F0CEF9404610F025FD05463C
:102AB80000B1451E0F3F0024153E1FFA87F90DE0AF
:102AC80002F0CAF902F0CEF904FB106189B2484657
:102AD8002022002302F008FA0134E4B2AC42EFD31A
:102AE800002002F0B9F8B8B2B1B24246012302F0B0
:102AF800FBF9002002F0A6F9012000E0204605B00D
:102B0800BDE8F0832DE9F04385B004AB03E9060086
:102B18004568BDF80860BDF80C70002D3CD0012355
:102B28006B762B7EBDF80A10012B0CBF6A68AA6869
:102B38009DF80E300092FFB23A463046FFF75DFF2F
:102B48000C35022002F07EF9284610F0D5FC0E3F25
:102B580081460024163E1FFA87F80DE002F07CF942
:102B680002F080F904FB106189B24046202200235C
:102B780002F0BAF90134E4B24C45EFD9002002F072
:102B88006BF8B8B2B1B22A46012302F0ADF90020C1
:102B980002F058F9012000E0284605B0BDE8F083AE
:102BA8002DE9F04F85B00546DDF840900291484682
:102BB8009046039310F0A0FCDDF838A0DDF83CB097
:102BC8000646294600242F4611E024B1B4420CBF22
:102BD8005B46534600E0039B01F10805ADB2009344
:102BE8002846029A4346FFF708FF01342946B442B3
:102BF800EBDD002002F030F8022002F023F97D1D01
:102C080008F10508A8B21FFA88F14A46012305B061
:102C1800BDE8F04F02F04EB970B5406886B006AB1B
:102C280003E9060000282ED0012380F82D3086689D
:102C3800164BF21A534243EB020390F82C205AB178
:102C4800002B134D134B144A08BF1D46134B00F1BC
:102C58001C0418BF13460AE0002B0D4D0D4B0E4AFD
:102C680018BF1D460D4B00F10C0408BF1346BDF8F4
:102C78001200BDF81410BDF81620009601950294B4
:102C8800FFF78EFF012006B070BD00BF782704084B
:102C9800B42304085A290408962504083C2B040880
:102CA80070B5446886B006AB03E9060004B3012397
:102CB8006377A668104B227FF11A4B4243EB01035E
:102CC8000AB10BB904E01BB966680C4D0C4B01E066
:102CD8000C4D0D4BBDF81200BDF81410BDF81620B0
:102CE80000960C3401950294FFF75AFF012000E08A
:102CF800204606B070BD00BFC4320408002F040887
:102D0800E23004089A340408703604082DE9F043C8
:102D180085B004AB03E906004468BDF80860BDF857
:102D28000A90BDF80C50BDF80E80002C00F08C8085
:102D38000123A3740220676802F084F84FF6FF703D
:102D480001F0A0FF002001F087FFEDB25FFA88F8DC
:102D5800A6F1160189B230462A4643460097FFF786
:102D68004CFE277A002F2ED1A28A234600E0013795
:102D7800974204D29969097E04330029F7D002F0FA
:102D88006BF802F06FF8A9F116091FFA89F90E21FC
:102D980001FB10914FF6FF7208F101085FFA88F302
:102DA80089B2009248462A46FFF7B5FD022002F094
:102DB80049F81F2001F050FFA38A002B38D0103D9E
:102DC800E8B2303E2CE0E3685C68A28A2346013A08
:102DD800002700E00137974204D29969097E04333D
:102DE8000029F7D002F038F802F03CF80E2101FB78
:102DF80010914FF6FF7208F101085FFA88F389B263
:102E0800009248462A46FFF786FD022002F01AF88B
:102E18001F2001F021FFA38A53B1103DE8B21A3EEA
:102E28000637B1B254F827200123083202F05CF8C3
:102E3800002002F007F84FF6FF7001F023FF1F2073
:102E480001F00AFF012000E0204605B0BDE8F0834C
:102E58002DE9F04105463620884614461F460FF0F6
:102E680053FF0646E0B120F8025B41462E22FFF7E9
:102E780017FCBDF8183086F83440738618200123F3
:102E880086F8307086F831300FF03EFF044618B1EE
:102E980004234660037404E030460FF03DFF00E071
:102EA80004462046BDE8F081F8B5064624200F46C2
:102EB80015460FF029FF0446D8B10F4B06808360F2
:102EC8000E4B39464360102200F10C00FFF7E8FB77
:102ED8000126002318202562237766770FF014FF58
:102EE800054610B14460067404E020460FF014FF54
:102EF80000E005462846F8BDC43204081E2D040823
:102F0800F8B506462C200F4615460FF0FDFE044680
:102F1800E8B120F80C6B39461922FFF7C1FB0D4BBD
:102F2800A562A3600C4B6360002384F82530182049
:102F3800012384F826300FF0E7FE054618B1032375
:102F48004460037404E020460FF0E6FE00E0054606
:102F58002846F8BDD04B04086E48040810B504464E
:102F680014200FF0D1FE20B100234380014B0480D0
:102F7800036110BDCD27000838B5054644200FF081
:102F8800C3FE0446C0B10E4B058243600D4B03607F
:102F9800012383740023037283820B4B036418207C
:102FA8000FF0B2FE054618B107234460037404E02D
:102FB80020460FF0B1FE00E00546284638BD00BFA8
:102FC800644404085A400408C12800082DE9F04167
:102FD80005463420884614461F460FF095FE0646DF
:102FE80020B3144B05808360134B41464360102285
:102FF80000F10C00FFF754FB214606F11C001022DB
:10300800FFF74EFB002386F82C3018200123376386
:1030180086F82D300FF078FE044618B10523466077
:10302800037404E030460FF077FE00E004462046C3
:10303800BDE8F08178270408D22104082DE9F04181
:10304800044614200D46164698460FF05DFE0746C6
:10305800B8B1069B048003610023C3720123456055
:10306800068180F80A80037318200FF04DFE04468D
:1030780018B106234760037404E038460FF04CFE8D
:1030880000E004462046BDE8F0812DE9F041044601
:1030980018200D46164698460FF036FE0746B8B17A
:1030A80001238370069B04800361079B456086604B
:1030B800C0F80C80436118200FF026FE044618B1B2
:1030C80008234760037404E038460FF025FE00E04B
:1030D80004462046BDE8F0812DE9F34198461B8B54
:1030E8001D2B05460C4617464FF0000000F2B48031
:1030F800B5F5A07F0090019000F2AE80F02900F2B3
:10310800AB80127CADF80610511EADF802500729AD
:1031180000F28A80DFE801F045595E04456A1476BA
:103128007B684E4A7A611A8893F834303A80013BBA
:10313800DBB2012B7FD8ADF80240ADF806507AE03B
:1031480005F11602ADF8002004F11602ADF80420CE
:1031580002AE434A16E903007A6107F1080282E8E1
:10316800030003F10802013348F82270A8F8183068
:103178007B681A8A187A3A8000286CD1FFF7FCFE1F
:103188003849436859603849DF600126163D19609F
:1031980002461E72A8B2E1B24346FFF79DFF3046D1
:1031A8005AE0012A0CBF314B314B78687B6130F80B
:1031B8000C3B3B8010F0A0F9431CDB001A34ED18DF
:1031C800ADF80440ADF8005035E07B68294A1B682B
:1031D8007A6102E0284A7B687A611B8814353B8053
:1031E800ADF800501434ADF8044024E07B68234A5D
:1031F8007A611A883A801A899B7AAD18ADF800501E
:10320800E418F0E77E681E4B7B61338838463B80C4
:1032180073689847013D4519ADF80050B3683846C2
:103228009847013C0419DEE71648174A174B40F245
:103238001A3100F0E3FC02AA12E9030007F10803BF
:1032480083E80300B8F8183003F10802013348F89E
:103258002270A8F818300120BDE8FC815128000828
:10326800152D0008503C040846380408A92C00080D
:10327800212C00080D2B0008672A0008332A0008B3
:10328800DD2500082F970508181E04082D97050846
:10329800F8B51646002834D01378002B2ED0028BB0
:1032A800002327E0046A257C042D21D165682F8836
:1032B8008F421DD195F8313053B16F8E01F0F2FC79
:1032C80004F1080268866369204606CA98476F8633
:1032D800A81C31462E22FFF7E3F995F831307BB16F
:1032E80004F108026369204606CA98470120F8BD20
:1032F800013304309342D5D30020F8BD1846F8BDF9
:103308000120F8BD70B5B8B1068B0446002310E063
:10331800256A287C04280AD16D682888884206D145
:103328001046A91C2E22FFF7BBF9012070BD0133FE
:103338000434B342ECD3002070BD38B5044620B342
:10334800134BC361134BC0F89830134BC0F89C3033
:10335800124B00257822C0F8A0308575C575058305
:10336800294600F120000FF0C1FFD4F8983020461C
:10337800294698470A4A1388312B07D8094941F842
:10338800234001331380012038BD38BD284638BD9D
:10339800692600086126000801260008D7260008CB
:1033A800440C0020DC1400202DE9F04104460028DC
:1033B80000F0B380078B02460025A8E0136A1E7C44
:1033C800042E00F08780012E23D1586803888B4291
:1033D80040F09B8005F108070FF09EFC54F8270089
:1033E8004FF00008C0F804800FF096FC228B531EA3
:1033F8009D4208D00732238354F8221044F827103E
:1034080044F8228002E044F8278025833046BDE84E
:10341800F081052E5ED0032E5CD0022E13D15B689E
:10342800186803888B4270D14388013B9BB2438064
:103438000BB90FF071FC05F1080654F826305868EE
:103448000FF06AFC4EE0072E21D15E68338A8B426A
:103458005BD1002706E0BB1D013756F823000FF0AB
:103468005BFCFFB2B38ABB42F5D80027B78205F1EF
:10347800080654F8263058680FF04EFC54F8260019
:1034880033E044F8267025830120BDE8F081062E3C
:103498001ED1586803888B4237D105F108060FF012
:1034A8003BFC54F82600002747600FF035FC228BC0
:1034B800531E9D4209D00833013A54F82310228341
:1034C80044F8261044F82370DEE744F826701AE022
:1034D800082E1AD1586803888B4216D10FF01CFCAD
:1034E80005F1080654F82600002747600FF014FC81
:1034F800228B531E9D42C4D0073254F8221044F840
:10350800261044F822702383BEE701350432BD42F9
:10351800FFF454AF0020BDE8F081BDE8F08170B53C
:10352800044600282AD0068B751E083600EB86064E
:103538001EE056F8043D1A7C042A13D0012A11D043
:10354800052A0FD0032A0DD0022A02D15B681B6816
:1035580009E0072A02D15B68198A05E0062A01D02A
:10356800082A04D15B6819882046FFF71DFF013D32
:10357800681CDED100232383012070BD70BDF0B527
:1035880028B30023068B1A461EE0046A257C072D03
:1035980018D16468258A8D4214D1A78A002504EBC6
:1035A80083040DE004EB050C0435DCF818C09CF826
:1035B80018C0BCF1010F03F1010301D1D8B2F0BD6D
:1035C800BB42EFD301320430B242DED30020F0BD5B
:1035D80070B508B3048B00231BE0026A157C072D25
:1035E80015D15268158A8D4211D10023958A11464A
:1035F8001C46012007E013B99669307601E08E6910
:10360800347601330431AB42F5D3012070BD013368
:103618000430A342E1D3002070BD2DE9F04128B366
:103628000023078B1A461EE0046A257C072D18D153
:103638006468258A8D4214D1B4F814C0002504EBBF
:1036480083040CE066190435B66996F81880B8F159
:10365800010F03D106F10800BDE8F081013363458D
:10366800F0D301320430BA42DED30020BDE8F08145
:103678002DE9F04700282FD00023B0F818C01D46C8
:1036880027E0046A267C072E21D16468268A8E42A8
:103698001DD1B4F81480002604EB830915E009EB6A
:1036A8000604A7693C7E012C0DD192F800A0BAF15E
:1036B800000F08D007F1080011461022FEF7F0FFAE
:1036C8002046BDE8F087013304364345E7D301358A
:1036D80004306545D5D30020BDE8F087F0B5B0B11A
:1036E800068B002510E0046A277C062F0AD164683F
:1036F80027888F4206D123819DF814306260A37217
:103708000120F0BD01350430B542ECD30020F0BDF6
:1037180010B500210446FEF7A3FF20460121BDE8AD
:103728001040FEF79DBF38B598B1048B02460023C0
:103738000CE0106A058804328D4206D100F10802B7
:10374800436906CA9847012038BD0133A342F0D324
:10375800002038BD10B50C460021FEF781FF204639
:103768000121BDE81040FEF77BBF13B502AC04E9A8
:103778000C00BDF80230834206D8BDF80030834201
:1037880034BF0020012000E00020BDF806308B4245
:1037980006D8BDF804308B4234BF0021012100E077
:1037A8000021002818BF0846C0B21CBD38B5114B0F
:1037B800114A1988002319E052F8045FA87D0128EE
:1037C80012D100240CE004F1080355F82300037C0F
:1037D800082B03D1436800211B6998470134A4B220
:1037E8002B8BA342EFD838BD01339BB28B42E3D178
:1037F80038BD00BF440C0020D8140020704770B5B5
:10380800094CA5787DB9094B1E78012E0BD1636848
:10381800013363606268064B9A4204D9284601F076
:10382800D3FAA670656070BD440C002030000020FB
:1038380040420F00054A9060134602E0996801393A
:10384800996091680029F9D1704700BF440C0020A5
:10385800F0B585B001F064FD002800F0498100252D
:1038680002A80DF10A01ADF80850ADF80A5001F0B0
:1038780059FD03A80DF10E01ADF80C50ADF80E502E
:1038880001F09CFDBDF80C10BDF808200091BDF8B2
:103898000E10BDF80A3001912C46964D9649082025
:1038A80008F060F9A878012803D101F08DFAAC700E
:1038B80019E1924B5B78012B40F01581AB78002B16
:1038C80040F011816B6029888D4A09E152F8046F34
:1038D800B07D012840F002810025FAE005F10803D7
:1038E800BDF8080056F82340BDF80A1004F1080393
:1038F8000CCBFFF73AFF002800F0E980237C013B5E
:10390800062B00F29F80DFE803F00429159D1F9D18
:103918004C006668012304F10805337795E8060032
:10392800636920469847002333772046636995E802
:10393800060086E0636893F8252012F1FF3218BF6D
:10394800012283F8252077E0636893F82C2012F190
:10395800FF3218BF012283F82C206DE06268137EC5
:103968001568002B6ED16E882F462946184606E04A
:1039780051F804EFDEF804E001338EF81800B34282
:10398800F6D301231376002607E057F8040F00F159
:103998000802436906CA984701366B889E42F4D3E9
:1039A80050E0656820892E68A37B227B0096A0F1F1
:1039B800160189B2FFF721F81420FFF73BFF2B7A95
:1039C800C3B9AF8A29461A461E4609E0886990F8A5
:1039D80018E00676BEF1010F08BF13460431013224
:1039E800BA42F3D301220BB9AB6924E0053355F889
:1039F800233020E06368DB685A680023908A154604
:103A080019461F4609E0AE6996F818E03776BEF108
:103A1800010F08BF0B46043501318142F3D3411E23
:103A28008B4203D1053052F8203003E004D207332B
:103A380052F8233001221A7604F1080206CA636993
:103A480020469847237C013B072B4CD8DFE803F03E
:103A58000410074B0A0D123A63681B6A34E0636866
:103A68009B6A2DE063681B6B2AE063681B6927E08B
:103A7800636824E063681A7A7AB9988A1946013823
:103A880000E00132824204D28C69247E0431002C89
:103A9800F7D0063253F8223011E0DB685A68908A72
:103AA80011460138002300E00133834204D28C69B7
:103AB800247E0431002CF7D0063352F82330DB691A
:103AC800984710E06368DB68204698470BE00135AB
:103AD800ADB2338BAB423FF601AF04E001339BB28A
:103AE8008B427FF4F3AE01F061FC0F20FFF7A2FEDA
:103AF80005B0F0BD440C00205597050830000020A3
:103B0800D8140020034B9A6812B19A68013A9A6057
:103B1800704700BF440C00202DE9F3470120DFF86F
:103B2800D080DFF8D090014609F0B6FB00250124CB
:103B380003234FF480760227404669468DF8053006
:103B480000968DF804708DF806508DF8074008F03F
:103B5800FBFF40460821224609F076F8234BDFF8A0
:103B680098801A6844F2A243B2FBF3FA0AF1FF3ACA
:103B7800204621461FFA8AFA09F0BEFBC8F804A0BD
:103B880048464146A8F80050A8F80250A8F808503E
:103B980088F80A5009F04CFF7023A8F80C30042369
:103BA800A8F810300AF1FF3A6323642203FB0AF3F2
:103BB800B3FBF2F39BB2C8F8143008F10C01484685
:103BC800A8F80E40A8F81870A8F81A50A8F81C60B1
:103BD800A8F81E500AF04AF84846214609F0BDFFE9
:103BE800484621460AF0C3FABDE8FC879C0100203C
:103BF8000000024000000140540C002083B50E462E
:103C08000746154910201C46154607F0ABFF102043
:103C1800124907F0A7FF1020114907F0A3FF102051
:103C28000E4907F09FFF002310200E49019307F06B
:103C380099FF334610200C493A4607F093FF1020AD
:103C48000A492A4607F08EFF10200949224607F044
:103C580089FF019B0133E7E78F97050894970508CB
:103C6800B4970508C4970508D4970508E997050887
:103C7800FA97050808B5164B1A6A01321A621A6AC9
:103C8800012A1A4603D013484FF4A0710FE0586276
:103C9800194602E04B6A013B4B62506A0C4B002804
:103CA800F8D11A6A012A06D00A4840F24B110A4A8A
:103CB8000A4BFFF7A3FF1A6A013A1A621B6A2BB173
:103CC8000448054A064B40F24D11F2E708BD00BF13
:103CD800540C00200B980508F6550408359805087B
:103CE800469805080C4B0D491A6844F2A24364280B
:103CF800B2FBF3F3D4BF20EAE0706420013B9BB22F
:103D08004B60013B58436422B0FBF2F080B248613B
:103D180003480C3109F02DBF9C010020540C0020F1
:103D28000000014010B5134B93F828202AB112481F
:103D3800124A134B4FF40A710EE0012283F828202F
:103D480066234FF0C042013BDBB2108033B90A480A
:103D58000A4A0C4B40F23221FFF750FF1488A4B2F4
:103D68008442F0D1084B1980024B002283F82820A6
:103D780010BD00BF540C00200B980508005604081D
:103D8800579805082D9705080000026010B5FFF741
:103D9800C3FE6420FFF7A6FFE5204FF40041FFF7BC
:103DA800C1FF00200121FFF7BDFF01204FF4807102
:103DB800FFF7B8FF02204FF4E061FFF7B3FF0320DD
:103DC80041F23001FFF7AEFF04200021FFF7AAFF00
:103DD800082040F20221FFF7A5FF09200021FFF784
:103DE800A1FF0A200021FFF79DFF0C200021FFF70B
:103DF80099FF0D200021FFF795FF0F200021FFF705
:103E080091FF10200021FFF78DFF11200021FFF7FF
:103E180089FF12200021FFF785FF13200021FFF7FB
:103E280081FF102041F2B071FFF77CFF372111208C
:103E3800FFF778FF3220FFF71DFF122040F23B11F9
:103E4800FFF770FF3220FFF715FF13204FF4C05122
:103E5800FFF768FF0F212920FFF764FF3220FFF7E3
:103E680009FF20200021FFF75DFF21200021FFF737
:103E780059FF30200021FFF755FF31200721FFF7B8
:103E880051FF322040F20311FFF74CFF352040F27A
:103E98000741FFF747FF40F20444362040F60F1170
:103EA800FFF740FF37202146FFF73CFF38204FF44B
:103EB8008061FFF737FF39202146FFF733FF3C20A9
:103EC8000021FFF72FFF3D204FF48061FFF72AFF05
:103ED80050200021FFF726FFEF215120FFF722FF96
:103EE80052200021FFF71EFF532040F23F11FFF739
:103EF80019FF60204FF41C51FFF714FF61200121C6
:103F0800FFF710FF6A200021FFF70CFF8020002137
:103F1800FFF708FF81200021FFF704FF822000211E
:103F2800FFF700FF83200021FFF7FCFE842000211B
:103F3800FFF7F8FE85200021FFF7F4FE90201021FE
:103F4800FFF7F0FE92200021FFF7ECFE93200321FB
:103F5800FFF7E8FE95204FF48871FFF7E3FE9720FE
:103F68000021FFF7DFFE98200021FFF7DBFE072086
:103F780040F27311BDE81040D4E610B5FFF7CCFD50
:103F88006420FFF7AFFE21210720FFF7CBFE322088
:103F9800FFF770FE01210020FFF7C4FE3220FFF773
:103FA80069FE23210720FFF7BDFE3220FFF762FEDE
:103FB80000211020FFF7B6FE41F28830FFF75AFEC5
:103FC80033210720FFF7AEFE3220FFF753FE112002
:103FD80046F63001FFF7A6FE3220FFF74BFE4FF4FE
:103FE800C0610220FFF79EFE3220FFF743FE122039
:103FF80046F6EB41FFF796FE3220FFF73BFE032023
:104008004AF6A401FFF78EFE3220FFF733FE0021A7
:104018000C20FFF787FE3220FFF72CFE0D2040F61C
:104028000C01FFF77FFE3220FFF724FE0E204FF42D
:104038002C51FFF777FE3220FFF71CFEB0211E201F
:10404800FFF770FE3220FFF715FE012042F63F31E0
:10405800FFF768FE3220FFF70DFE05200021FFF76D
:1040680061FE3220FFF706FE00210620FFF75AFE08
:104078003220FFF7FFFD16204EF61C71FFF752FEA7
:104088003220FFF7F7FD172040F20311FFF74AFE31
:104098003220FFF7EFFD00210B20FFF743FE32200F
:1040A800FFF7E8FD00210F20FFF73CFE3220FFF765
:1040B800E1FD41200021FFF735FE3220FFF7DAFD50
:1040C80042200021FFF72EFE3220FFF7D3FD00210A
:1040D8004820FFF727FE40F23F143220FFF7CAFDC1
:1040E80021464920FFF71EFE3220FFF7C3FD0021BD
:1040F8004A20FFF717FE3220FFF7BCFD00214B20B6
:10410800FFF710FE3220FFF7B5FD44204FF46F4152
:10411800FFF708FE3220FFF7ADFD00214520FFF72D
:1041280001FE3220FFF7A6FD21464620FFF7FAFDE3
:104138003220FFF79FFD302040F20771FFF7F2FDB4
:104148003220FFF797FD31204FF40171FFF7EAFDA8
:104158003220FFF78FFD32204FF40171FFF7E2FDA7
:1041680040F202543220FFF785FD21463320FFF745
:10417800D9FD3220FFF77EFD342040F20751FFF7CA
:10418800D1FD3220FFF776FD35204FF40171FFF79E
:10419800C9FD3220FFF76EFD36204FF40171FFF79D
:1041A800C1FD3220FFF766FD21463720FFF7BAFD33
:1041B800A4F500743220FFF75DFD21463A20FFF791
:1041C800B1FD3220FFF756FD2F2041F2BE21FFF747
:1041D800A9FD3220FFF74EFD21463B20FFF7A2FD47
:1041E8003220FFF747FD00212320FFF79BFD3220F7
:1041F800FFF740FD00212420FFF794FD3220FFF750
:1042080039FD25204FF40041FFF78CFD3220FFF7E0
:1042180031FD00214F20FFF785FD3220FFF72AFDF1
:104228004E200021FFF77EFD3220BDE8104021E539
:1042380008B5124B93F829202AB11148114A124B9C
:1042480040F242210FE0012283F82920222166232F
:104258004FF0C042013BDBB2118033B90848094A2C
:104268000A4B40F25B21FFF7C9FC108880B2222874
:10427800F0D1024B002283F8292008BD540C0020FD
:104288000B9805080D560408579805082D9705083A
:1042980010B5224B49F22032032823D8DFE800F07A
:1042A800021A0B111C8846F6280041F22801944294
:1042B80018BF01461AE01C8841F2080046F60801BA
:1042C80004E01C8841F2300046F63001944208BFF1
:1042D80001460BE0188846F62001904208BF4FF4CB
:1042E800815103E00E4840F2792113E01B8848F61B
:1042F8008912934205D049F22032934207D1032014
:1043080000E01120FFF70EFDBDE8104090E70448DB
:1043180040F28521034A044BFFF770FC320000206D
:104328000B980508225604082D970508014B18809C
:104338000A209FE4000002604FF0C043188003F594
:1043480000331A881A88188880B270472DE9F0411E
:10435800022098B00121002408F09EFF01250226C2
:104368008C488DF85C5016A98DF85E408DF85F403A
:1043780016968DF85D6008F0E7FB1820294608F0CE
:104388008BFF2846294608F09FFF21460C228248C9
:1043980008F05AFC29460C227F4808F055FC0421F5
:1043A8000C227D4808F050FC05210C227A4808F0C0
:1043B8004BFC07210C22784808F046FC08210C2207
:1043C800754808F041FC09210C22734808F03CFCB0
:1043D8000A2171480C2208F037FC0B216E480C2288
:1043E80008F032FC0E210C226B4808F02DFC0F213E
:1043F8000C22694808F028FC07210C22674808F0BD
:1044080023FC08210C22654808F01EFC09210C2217
:10441800624808F019FC0A210C22604808F014FCD4
:104428000B210C225D4808F00FFC0C210A465B4862
:1044380008F00AFC0D210C22584808F005FC0E2152
:104448000C22564808F000FC0C2254480F2108F0B2
:10445800FBFB03274CF6B3734F48169316A98DF848
:104468005D708DF85E408DF85F408DF85C6008F0F7
:104478006BFB4FF6807316A9484816938DF85D704C
:104488008DF85E408DF85F408DF85C6008F05CFB4D
:1044980040F6B830FFF7EEFB224631463D4808F0BB
:1044A800C8FB44F6FF70FFF7E5FB2A46314639485A
:1044B80008F0BFFB40F6B830FFF7DCFB4FF4805341
:1044C800102709930DF13C084FF4002368460F9418
:1044D80010941294139514941594009401940294D2
:1044E80004940694079408940A9405940B940C93E6
:1044F80011960397CDF8348008F09FF80423684696
:104508001193109412941395149415940F96CDF852
:10451800388008F092F82946204608F00EF940F64F
:10452800B830FFF7A7FB2046FFF706FF04461C49F3
:104538001C4D3846224607F015FB48F689139C4265
:104548001AD049F220339C420DD041F289239C4273
:1045580012D03846144907F005FB1448144A154B85
:10456800A621FFF74BFB38461349224607F0FAFA13
:104578002C80FFF70BFC0AE0FFF7FFFC48F68912D6
:104588002A8010200D4941F2892307F0EBFA18B070
:10459800BDE8F08100040240000C02400010024017
:1045A8006C98050832000020839805080B980508C8
:1045B8003A5604082D970508BA980508EF98050893
:1045C8004FF0C04322221A8003F5003382B01A88C4
:1045D80092B2ADF806201B889BB2ADF80630BDF844
:1045E800060080B202B07047134B1B8848F6891248
:1045F800934210B504460BD049F22032934213D1AE
:10460800C1F1EF01202089B2FFF78CFB212006E0E1
:10461800C1F1EF014E2089B2FFF784FB4F202146FC
:10462800BDE81040FFF77EBB0448054A054B40F241
:10463800F321FFF7E3FA00BF320000200B980508CA
:10464800435604082D9705082DE9F0410D46C5F19C
:10465800F008411E5E18C2EB0802C5F1EF039BB2D9
:1046680092B2B6B29A422CBF904698469A4234BF4C
:1046780011461946864234BF3746074640F23F1373
:10468800864238BF06469E4228BF1E461B4B1B88E3
:1046980048F68912B8F1EF0F28BF4FF0EF089342A0
:1046A800044610D049F2203293421FD15020FFF720
:1046B80039FB51204146FFF735FB52203946FFF7B9
:1046C80031FB53200AE041EA082189B24420FFF770
:1046D80029FB45203946FFF725FB46203146FFF7E1
:1046E80021FB20462946BDE8F0417DE70448054AFC
:1046F800054B40F2DD21FFF781FA00BF32000020B0
:104708000B980508515604082D9705080020014606
:10471800F0224FF4A07397E7072040F27311FFF7D8
:1047280001BB07200021FFF7FDBA10B51446FFF7BB
:104738005BFFFFF77DFD2046BDE81040F6E508B5B4
:10474800FFF752FF4FF0C04322221A8003F50033CF
:104758001A88188880B208BDF8B580B202FB03F544
:1047680089B292B29BB2069C9DF81C60FFF76CFF61
:104778000020FFF78DFD002709E034F8020B1EB179
:10478800030A43EA002080B2FFF7D0FD0137AF42A9
:10479800F3DBBDE8F840B9E72DE9F74F16469DF879
:1047A80034200C9F01920546B2B280B20C4698465E
:1047B80089B29BB2FFF748FF4FF0000B0020FFF7CC
:1047C80067FDDA463DE0002D30DB09EB050340F2DA
:1047D8003F1293422ADC002C28DB0BEB0403EF2B5F
:1047E80024DC19F00F0F04D1B9F1000FC8BF0AF18A
:1047F800010A174B09EA0303002B03DA013B63F0B4
:104808000F030133019A0AB1C3F10F03012202FA1F
:1048180003F337F81A2013401BB213B10D4B588D10
:1048280001E00D4A508880B2FFF780FD09F10109C7
:1048380001E04FF00009C145C5DB0AF1010A0BF19F
:10484800010BB345F5DB03B0BDE8F04F5EE700BFF1
:104858000F000080540C0020320000202DE9F04F9A
:1048680085B004469DF83C00029200278A460390D2
:1048780088463E4640F23F1C9B463AE0002C2FDB20
:10488800E1452DDCBAF1000F2ADBB8F1EF0F27DC88
:104898002A0702D1002DC8BF01361B49294000292B
:1048A80003DA013961F00F010131039A0AB1C1F14C
:1048B8000F010E9830F8162003FA01F10A4012B2DF
:1048C80072B112494A8D019392B21FFA89F01FFA08
:1048D80088F1CDF800C0FFF728FFDDF800C0019B84
:1048E800013509F101095D45C8DB0136013708F1D9
:1048F8000108029A974203DAA14600250123F2E74C
:1049080005B0BDE8F08F00BF0F000080540C0020F8
:1049180082B0044BADF80600BDF8062092B25A8565
:1049280002B07047540C002082B0044BADF806006A
:10493800BDF8062092B25A8002B0704732000020BB
:1049480070B50646FFF7E2FE0020FFF7A1FCF02451
:1049580009E0013D3046ADB2FFF7E8FC002DF8D183
:10496800013CA4B214B14FF4A075F2E770BD70B564
:104978001D461446FFF738FE2846FFF789FC002538
:10498800054E05E0708D80B2FFF7D0FC0135ADB261
:10499800A542F7D170BD00BF540C00202DE9F041AD
:1049A8000C4616461F461A4600230546FFF7DFFF4A
:1049B800611E711828463A46002389B2FFF7D7FFCF
:1049C8002846214632460123FFF7D1FF013D7F19D2
:1049D800B8B2214632460123BDE8F041C7E770B5B9
:1049E80080B202FB03F489B292B29BB2FFF72CFEAD
:1049F8000020FFF74DFC0025054E04E0708D80B2C5
:104A0800FFF794FC0135A542F8DBBDE870407DE670
:104A1800540C0020F8B5561A0C46013189B21F46CD
:104A28000546FFF7E1FD0120FFF732FC4FF0C043D8
:104A380022221A800E4A0F491388B6B2002304E0D6
:104A48001088013321F8020B9BB2B342F8D12146FA
:104A58002846FFF7C9FD0120FFF71AFC002404E0EF
:104A68003846FFF763FC0134A4B2B442F8D1F8BD6C
:104A780000000260E643002070B5194B194AD98D31
:104A880092F9004064180025A4B2AC4208BF012482
:104A9800C62C28BFC6240F2615704FF6FF7288B0A3
:104AA8009E85DC855A8519200A222B462146FFF768
:104AB8005EFF21463046FFF742FE224603460A497A
:104AC80068460EF093FC6A4604A808490EF08EFC6E
:104AD8003220D22104AA2B4600F0ECF908B070BDB0
:104AE800540C0020902B00202E99050836990508B3
:104AF8002DE9F0431F2093B0FFF722FF4FF47840D1
:104B0800FFF71EFF4FF6E0754FF4FC60FFF718FF44
:104B18002846FFF715FF0020494CFFF711FF00203A
:104B28000146642203464FF6FF79A4F82A90FFF75E
:104B38001EFF00200A2164220346FFF718FF002009
:104B48000146642201234FF478476585FFF70FFF7C
:104B58007720EF21C82200234FF4FC666785FFF712
:104B680006FFBD213222012340F23F106685FFF780
:104B7800FEFEA0203222002378216785FFF7F7FE8A
:104B8800A0207821322201234FF01F086685FFF705
:104B9800EEFEA020782132220223A4F82A80FFF713
:104BA800E6FEA0207821322203236585FFF7DFFE89
:104BB800244B2549A3F8028002AD3C2228460EF07A
:104BC80053FBEB20C3210522302300950025A4F8D0
:104BD8002A900195FFF7E0FD32210A2096220B4624
:104BE8006785FFF7DBFE32213C2096220B4666855F
:104BF800FFF7D4FE32210B4696226E20A4F82A80B5
:104C0800FFF7CCFEFFF78DFDFFF786FD3220FFF79B
:104C180069F82846FFF766F86420FFF763F80B4B3E
:104C280003F110028DE8240028465A681B682946BB
:104C3800FFF792FD1195119B01331193FBE700BF1C
:104C4800540C00203200002066560408A87A010897
:104C580000487047A815002082B0064BADF8060042
:104C6800BDF8062092B21A80188880B202B0FFF709
:104C78004FBE00BFA4150020014B188880B27047B2
:104C8800A415002082B0064BADF80600BDF806203A
:104C980092B21A80188880B202B0FFF745BE00BFF2
:104CA800A6150020014B188880B27047A615002071
:104CB800FFF746BEFFF7C8BCFFF759BEFFF76EBE49
:104CC800FFF78DBE2DE9F04F4FEA420800253D4C15
:104CD80085B082468B46C8F1030817462E461FFA50
:104CE80087F909EB0B0C228805EB0A031FFA8CFCE9
:104CF8009BB26146184692B2CDF804C00293FFF702
:104D080014FDC9EB0B0292B20392029B228803990D
:104D1800184692B2FFF709FDDDF804C02288C5EBFA
:104D28000A039BB26146184692B20293FFF7FDFC54
:104D3800029B22880399184692B2FFF7F6FC05EB0E
:104D48000B0292B2039209EB0A03228803999BB2E1
:104D5800184692B20293FFF7E8FC029B2288C5EB43
:104D68000B0C1FFA8CFC1846614692B2CDF804C0B1
:104D7800C9EB0A09FFF7D9FC228803991FFA89F9B8
:104D880092B24846FFF7D1FC2288DDF804C092B2FF
:104D980048466146FFF7C9FCB8F1000F04DA08EB92
:104DA800860808F1060805E0F31B08F10A0808EB75
:104DB8008308013F01360135BE42ADB28FD905B037
:104DC800BDE8F08FA415002008B9FFF7AABC012898
:104DD80001D1FFF7A1BC7047704700200146F022BF
:104DE8004FF4A073FFF730BC704708B505280CD8FE
:104DF800DFE800F0121403050709094808BD09484F
:104E080008BD094808BD094808BD0948094A0A4BB0
:104E180040F24111FEF7F2FE084808BD084808BDF7
:104E280020000020100000200800002000000020C2
:104E38003B990508A25604082D970508280000206C
:104E48001800002010B50446FFF7CFFF014B18608B
:104E58001C7110BD38000020014B1879704700BF45
:104E68003800002008B5FFF7C0FF808808BD08B5E6
:104E7800FFF7BBFFC08808BDF7B51F460B4B0C4EAC
:104E88001D681446EA882B68203C5443A4B2AE1B24
:104E980003EB440418BF0126AB888DE8500017B116
:104EA800FFF7DCFC01E0FFF777FCFEBD38000020CF
:104EB800280000202DE9F0410F4698461546044683
:104EC800084E08E0204643463946FFF7D5FF3368C9
:104ED8009B88E418A4B215F8012B002AF2D1BDE88A
:104EE800F08100BF3800002010B50446084621466E
:104EF800BDE81040DEE7094B70B5044618790E4648
:104F08001546FFF7B4FFC6F1F001091A89B2204629
:104F18002A460023BDE87040CCE700BF38000020D7
:104F2800704700BF044B1A680AB9044A1A601A6825
:104F38001018186010467047840C0020784F002025
:104F48004FF0FF30704708B50248034A034B37213A
:104F5800FEF754FE5A990508B85604082D97050817
:104F68000120704710B504460A48022108F01AFCCF
:104F78000028F9D00748214608F0DDFB0548012143
:104F880008F010FC0028F9D00248BDE8104008F0ED
:104F9800CFBB00BF0038004010B51948022108F007
:104FA80001FC0028F9D01648002108F0C4FB144879
:104FB800012108F0F7FB0028F9D0114808F0B8FBE8
:104FC8000402A4B2002301E001339BB2002BFBD002
:104FD8000B48022108F0E6FB0028F9D00848002118
:104FE80008F0A9FB0648012108F0DCFB0028F9D0ED
:104FF800034808F09DFB2043C0F3CB0010BD00BF61
:10500800003800402DE9F0478AB00AAF0A20012194
:1050180008F042F94FF4604347F8143D474EDFF873
:1050280024A1012400254FF00208304639468DF8A6
:105038001A508DF818808DF819808DF81B4007F0EC
:1050480083FD30460D21052207F0FEFD30460E2176
:10505800052207F0F9FD052230460F2107F0F4FD7F
:1050680021464FF4804008F03BF9504608F016FA04
:105078004FF48273ADF802304FF40073ADF80A3084
:105088003823ADF80C30504607236946ADF8103088
:10509800ADF80050ADF80450ADF80650ADF8085022
:1050A800ADF80E5008F02CFA5046214608F0C3FA25
:1050B800A9468DF81A5030464FF480553946059563
:1050C8008DF818408DF819808DF81B4007F03CFDCD
:1050D8003046294607F0A9FD4025394618488DF87D
:1050E80018908DF819808DF81A908DF81B40059549
:1050F80007F02AFD21464FF4804008F0FDF806210C
:10510800032008F087FB0C2307A88DF821300795AA
:105118008DF820908DF8224007F00AFA17238DF8B1
:10512800243009A80F238DF825308DF826308DF806
:10513800274002F041FB0AB0BDE8F08700040240B6
:10514800000C024000380040014B1878704700BF3F
:10515800880C0020024B5A889B8802800B8070477D
:10516800880C0020014B00221A707047880C002020
:10517800F0B593B06846002148220EF0B7F86D46A6
:10518800002464484FF4805107F051FD002301E0EA
:1051980001339BB2002BFBD09020FFF7E3FE0023E6
:1051A80001E001339BB2002BFBD0FFF7F5FE4FF473
:1051B80080510746574807F038FD002301E00133C6
:1051C8009BB2002BFBD053484FF4805107F02FFDC2
:1051D800002301E001339BB2002BFBD0D020FFF766
:1051E800C1FE002301E001339BB2002BFBD0FFF787
:1051F800D3FE4FF480510646464807F016FD45F8A1
:10520800047B01342E6244484021E4B207F0FBFCE1
:1052180010B9092CB5D101E0092C78D19DE80C0012
:10522800D218029B03980699D218049BC018059BB4
:10523800C018079BCB180899032490FBF4F092FB45
:10524800F4F25B1893FBF4F3151AC11A9C1A002D9B
:10525800B8BF6D420029B8BF4942002CB8BF6442AC
:10526800502D03DD502909DD502C50DC8D4205DA24
:10527800AC424FF0020405DB111806E08C424FF0F7
:10528800020401DAD11800E0C1180A9B099A0C98A7
:105298000F9DD2180B9BD2180D9BC0180E9BC018DF
:1052A800109BEB18119D91FBF4F1032492FBF4F28F
:1052B80090FBF4F05B1993FBF4F3161AC41A9D1AC9
:1052C800002EB8BF7642002CB8BF6442002DB8BF8C
:1052D8006D42502E89B203DD502C09DD502D16DCAD
:1052E800A64205DAB5424FF0020405DB131806E0C2
:1052F800A5424FF0020401DAD31800E0C318074AA8
:1053080093FBF4F39BB2938001235180137013B085
:10531800F0BD00BF00040240000C0240880C0020D1
:10532800FFF712BFF7B505460C4601A80DF10601B7
:10533800FFF710FF1B4BBDF80660BDF8040093E8AB
:105348000600724301FB002299685218164992FB25
:10535800F1F207EE102AF8EEC77A40F23F17FCEE9A
:10536800E77A17EE902A92B2B2F5207F28BF3A4624
:105378002A801D69DA685B696E4302FB0060C01809
:1053880090FBF1F107EE101AF8EEC77AFCEEE77A17
:1053980017EE903A9BB2B3F5F07F28BFEF23238036
:1053A800FEBD00BF900C002040420F00FFF7DABEA0
:1053B800014B187E704700BF900C0020FFF7CABE53
:1053C800042808B505D90748074A084B7D21FEF788
:1053D80015FC054B03EB8000038B0B80438B13807C
:1053E80008BD00BF7B990508BE56040899990508B1
:1053F80008B5082001F08CF942F69643C31A5842C2
:1054080040EB030008BD10B50A2001F0A9F90C4CC7
:1054180020600E2001F0A4F96060122001F0A0F9CC
:10542800A060162001F09CF9E0601A2001F098F9BC
:1054380020611E2001F094F901236061237610BDDC
:10544800900C002010B5FFF7DDFD01F02BFA0446A3
:1054580001F034FA074903462246202006F082FB71
:10546800FFF7C6FF28B101F037FA10B9BDE81040C0
:10547800C9E710BDD599050810B5104C0A20216858
:1054880001F055F961680E2001F051F9A168122068
:1054980001F04DF9E168162001F049F921691A2057
:1054A80001F045F961691E2001F041F9082042F632
:1054B8009641BDE8104001F01DB900BF900C0020D6
:1054C8002DE9F04F0346A7B0B0F800C01C898688C4
:1054D800DF885D89CDF810C0B249B0F802C0B3F8D2
:1054E8000C90B3F80E80CDF824C00FFA84FB30B2CC
:1054F80001220FFA87FE0BEB000C0A7629B20FFA8D
:1055080089FACDF888C001EB0E0C0FFA88F2CDF8B5
:1055180090C00AEB0B0CCDF830C002EB010CCDF8B3
:1055280058C0B3F810C05B8ACDF800C00FFA8CFCE5
:1055380006910CEB00010A9102930CEB0A011BB2D5
:10554800239103EB0E010E9199182591049900FA05
:1055580081F0584450446044DDF824C006990EFA9E
:105568008CFEDDF810C01FFA80FB1CFB0CF08E448B
:1055780016FB0600964414FB0400009A19FB090068
:105588009E4412FB02001FFA8EFA09F015FADDF8A4
:1055980024C0029ACDE912011CFB0CF017FB07008E
:1055A80015FB050018FB080012FB020009F004FABD
:1055B800DDF824C0029ACDE9140104991CFB01F31B
:1055C80017FB063615FB0466009B18FB096612FBE1
:1055D800036009F0F1F9DDE91423CDE90001DDE903
:1055E800120109F05FFA04460D46DDE900010246A2
:1055F8000B4609F057FA02460B462046294609F0A1
:105608009DF8CDE91801584609F0E6F9CDE91001F1
:10561800DDE91023DDE9000109F044FACDE90601CE
:10562800504609F0D9F9804689464246DDE912011B
:105638004B4609F037FADDE91023CDE91C01DDE915
:10564800140109F02FFA002206460F46564BDDE9F1
:10565800180109F027FA424604460D464B46DDE993
:10566800060109F01FFA02460B4609F069F80246DE
:105678000B462046294609F063F8424604460D4683
:105688004B46DDE91C0109F00DFA02460B4620469F
:10569800294609F053F8DDE9102304460D46304643
:1056A800394609F0FFF902460B462046294609F01B
:1056B80045F8DDF828C0CDE902014FEA8C10DDF885
:1056C80030C000EB0C20DDF810C0A0241CFB040047
:1056D80009F072F9DDF838C0CDE90A014FEA8C10FB
:1056E800DDF858C000EB0C20DDF824C01CFB0400DA
:1056F80009F062F9CDE90C01504609F05DF9DDE9E0
:105708001023CDE91601DDE90C0109F0CBF9424679
:10571800CDE91E014B46DDE90A0109F0C3F942460D
:10572800CDE920014B46DDE9000109F0BBF932461D
:105738003B4609F003F8CDE90E01584609F03CF95B
:10574800DDE91C23CDE91A01DDE9060108F0F6FFC1
:10575800DDF88CC0C024CDE9060104FB0CF0DDF8AF
:1057680088C0302505FB0C00DDF810C078261CFB2E
:10577800060009F021F9DDF894C0824604FB0CF01C
:10578800DDF890C005FB0C00DDF824C01CFB06000A
:105798008B4609F011F9DDE9102306460F4609F09A
:1057A80081F903E0900C0020000014404246CDE946
:1057B80004014B465046594609F074F9DDE91423B3
:1057C80080468946DDE90A0109F06CF9DDE9002324
:1057D80004460D46DDE90C0109F064F902460B4662
:1057E8002046294608F0AAFF0022A14B09F05AF9E1
:1057F800DDE9202304460D46DDE91E0108F09EFF81
:1058080002460B46DDE9160109F04CF902460B4643
:105818002046294608F094FF002204460D46954B81
:10582800DDE90E0109F03EF902460B4620462946FD
:1058380008F086FFDDE9022309F05EFA88A3D3E9C0
:10584800002309F02FF909F0C7FB8B490860DDE94F
:105858001223DDE90C0109F025F9DDE900230446EE
:105868000D46DDE90A0109F01DF902460B462046FE
:10587800294608F063FF00227D4B09F013F9DDE9A2
:105888001E2304460D46DDE9200108F057FF0246B5
:105898000B46DDE91A0109F005F902460B462046D8
:1058A800294608F04DFF002204460D46714BDDE9FC
:1058B800060109F0F7F802460B462046294608F08B
:1058C8003FFFDDE9022309F017FA65A3D3E90023B6
:1058D80009F0E8F809F080FB674A5060DDE90E231B
:1058E800DDE90A0109F0DEF8DDE9062304460D4684
:1058F800DDE90C0109F0D6F802460B462046294698
:1059080008F01EFF002204460D465A4BDDE9180137
:1059180009F0C8F802460B462046294608F010FF51
:10592800DDE9022309F0E8F94DA3D3E9002309F0E2
:10593800B9F809F051FB504B59469860DDE914233A
:10594800504609F0AFF8DDE9002304460D4630461D
:10595800394609F0A7F802460B462046294608F0C2
:10596800EDFE0022424B09F09DF8424604460D46E2
:105978004B46DDE9040108F0E1FE02460B46DDE98D
:10598800160109F08FF802460B462046294608F012
:10599800D7FE35A3D3E9002304460D46DDE90E0101
:1059A80009F080F802460B462046294608F0C8FE52
:1059B800DDE9022309F0A0F929A3D3E9002309F0BE
:1059C80071F809F009FBDFF8B0C0DDE91223CCF863
:1059D8000C003946304609F065F8DDE90023044635
:1059E8000D465046594609F05DF802460B462046DA
:1059F800294608F0A3FE00221D4B09F053F8DDE903
:105A0800042304460D464046494608F097FE0246E0
:105A18000B46DDE91A0109F045F802460B46204617
:105A2800294608F08DFE10A3D3E9002304460D464D
:105A3800DDE9060109F036F802460B4620462946FC
:105A480008F07EFEDDE9022309F056F904A3D3E944
:105A5800002309F027F809F0BFFA074908610DE0AB
:105A68000000000080842E410000000000C0824039
:105A78000000144000008940900C0020DDE90E234E
:105A88005046594609F00EF8DDE9062304460D464E
:105A98003046394609F006F802460B4620462946A4
:105AA80008F04EFE11A3D3E9002304460D46DDE9B4
:105AB800180108F0F7FF02460B462046294608F071
:105AC8003FFEDDE9022309F017F90AA3D3E9002311
:105AD80008F0E8FF09F080FA034A506127B0BDE8F2
:105AE800F04FC9E4AFF30080900C002000000000E4
:105AF80000C082400000000080842E41AFF3008087
:105B0800064B074A596811601969064A1160D96934
:105B1800054A11609A6A054B1A60704740000020D8
:105B2800643C002084420020584200200C3C0020A5
:105B3800014B1878704700BFAC0C0020032808B54B
:105B480005D90548054A064B7121FEF757F80C237D
:105B58005843044B185808BD109A0508EA5604081B
:105B68002A9A050840000020032808B505D90648E8
:105B7800064A074B7621FEF741F8064B0C2202FB3A
:105B88000030406808BD00BF109A0508FA5604089E
:105B98002A9A050840000020034B044A1B780C2170
:105BA80001FB032398687047AC0C002040000020DC
:105BB800034B044A1B780C2000FB032399607047B1
:105BC800AC0C002040000020144B1B78012B10B5B2
:105BD800134B144C0ED11968C82000F0A8FD216899
:105BE800CC2000F0A4FD104BD020196800F09FFDD8
:105BF800D4200DE01968D82000F099FD2168DC2038
:105C080000F095FD084BE020196800F090FDE420B5
:105C1800064B1968BDE8104000F089BD2C0E002025
:105C2800643C002084420020584200200C3C0020A4
:105C3800144B1B78012B10B5134C0FD1C82000F062
:105C48008FFD2060CC2000F08BFD104B1860D02019
:105C580000F086FD0E4B1860D4200EE0D82000F02E
:105C68007FFD2060DC2000F07BFD084B1860E02001
:105C780000F076FD064B1860E42000F071FD054B3E
:105C8800186010BD2C0E0020643C002084420020C7
:105C9800584200200C3C002008B502F0BFFA10B1B1
:105CA800BDE80840C4E7BDE8084029E70148FBF71C
:105CB800B4BF00BF901300200148FBF7AEBF00BF80
:105CC800901300200148FBF7A8BF00BF90130020E5
:105CD8000148FBF7A2BF00BF90130020032808B5B6
:105CE80005D91448144A154B4E21FDF787FF144B6C
:105CF8001870144B02281870134B0FD0032813D0B8
:105D0800012805D0114A12681A60BDE80840CDE79D
:105D18000F4A12681A60BDE80840CDE70D4A1268BC
:105D28001A60BDE80840CDE70B4A12681A60BDE862
:105D38000840CDE7109A05080B570408549A05083F
:105D4800AC0C0020523C002098010020900100205B
:105D58008C0100208801002084010020064B07499F
:105D68005960C021002219721E211A70D9601A7454
:105D78005A611A76DA617047D415002040787D019F
:105D880010B50321FF22C02001F072F81F4C10212A
:105D980020608022C02001F06BF811212060802251
:105DA800C02001F065F8122120608022C02001F097
:105DB8005FF8132120608022C02001F059F81421D7
:105DC80020608022C02001F053F815212060802235
:105DD800C02001F04DF8802220601621C02001F07B
:105DE80047F82060C0201721802201F041F8206088
:105DF800074CC020227AB72101F03AF80023237417
:105E080063612376E3610123237010BD303C0020D9
:105E1800D415002038B5C0200321FF2201F028F84E
:105E28000B4D00242B19615D5A78C020023401F013
:105E38001FF8C82CF6D1B121AC22C02001F018F807
:105E4800C0200321002201F013F8002038BD00BF54
:105E58001F5704082DE9F34706460F4692461D468C
:105E68001AB90C1FE401914635E005EE902A06EEBA
:105E7800903AB8EE657AF8EE667AFC01C7EE277AB2
:105E8800A4F500749FED5C7A67EE877A17EE900AA6
:105E980008F0B4FD41EC100B0AF0CAFD59EC108B68
:105EA8004946404609F0C0F824184FEACA1008F0DD
:105EB80083FDCDE90001284608F07EFD4B464246A9
:105EC80008F0F0FD02460B46DDE9000108F036FC5B
:105ED80009F0AAF88146002E14BF4FF022084FF0AF
:105EE8001A08C5F307224146C02000F0C1FF08F197
:105EF8000101EAB2C02000F0BBFFC4F3014208F17F
:105F08000201C02000F0B4FFC4F3072208F1030126
:105F1800C02000F0ADFFE2B208F10401C02000F09B
:105F2800A7FFC9F3034305F4702243EA123208F1CC
:105F38000501C02000F09CFF08F10601C9F3072203
:105F4800C02000F095FF08F107015FFA89F2C02030
:105F580000F08EFFC020B121A02200F089FF07EEDB
:105F6800107A264CF8EEC77A0EBBD4ED015A06EE2D
:105F780090AAB8EE657A05EE905AB8EE666AF8EE21
:105F8800656A0123C6EE266A237477EEA67A67EE61
:105F9800277A17EE900A08F031FD41EC100B0AF051
:105FA80047FD51EC100B09F03FF8606120E005EE69
:105FB80090AAD4ED016AB8EE656A05EE905AB8EE7B
:105FC800667AF8EE656A0123C6EE266A237677EECE
:105FD800A67A67EE277A17EE900A08F00FFD41ECD3
:105FE800100B0AF025FD51EC100B09F01DF8E061CB
:105FF8000020BDE8FC8700BF00000043D415002046
:106008000022012326E7012838B50D4604D00228CE
:106018000CBF3C242C2400E034242146C02000F08E
:10602800A1FF05F0070200F00F0040EA0212214626
:10603800C020BDE8384000F01BBF2DE9F3470A9C9B
:106048001D4607468A461646524B01E06D0864080D
:106058009C42FBD82DB906F10076043EF601A9460C
:1060680034E006EE905AB8EE667A06EE904AF8EEFC
:10607800667AF601C7EE277AA6F500769FED467A8E
:1060880067EE877A17EE900A08F0B8FC41EC100B1F
:106098000AF0CEFC59EC108B4946404608F0C4FF84
:1060A8003618E80108F088FCCDE90001204608F020
:1060B80083FC4B46424608F0F5FC02460B46DDE9F8
:1060C800000108F03BFB08F0AFFF8146022F9BBFA1
:1060D800324BDB194FF0000893F8C880C4F307224D
:1060E8004146C02000F0C4FE08F10101E2B2C9B285
:1060F800C02000F0BDFE08F10201C9B2C6F301429A
:10610800C02000F0B5FE08F10301C9B2C6F30722AA
:10611800C02000F0ADFE08F10401C9B2F2B2C020FF
:1061280000F0A6FE04F47024C9F3034308F1050146
:1061380043EA1432C9B2C02000F09AFE08F1060101
:10614800C9B2C9F30722C02008F1070800F090FE81
:106158005FFA89F25FFA88F1C02000F089FEBAF18F
:10616800010F0CBF2F220F220DB942F04002012F60
:1061780006D002D3022F0AD105E0C020102104E086
:10618800C020112101E0C020122100F071FE002082
:10619800BDE8FC87FFFF0F00000000431F570408FD
:1061A80007B5012300930023FFF747FF0EBD002822
:1061B8000CBFFF22002208B5C020032100F058FEC2
:1061C800002008BD08B5C020B121AC2200F050FE67
:1061D800002008BD08B50420012107F05DF84FF440
:1061E80080700121BDE8084007F086B807B5022392
:1061F800009303238DF804300348002369468DF883
:10620800073006F0A1FC0EBD0008024030B5124D63
:106218008BB0002406A8069407940894099405F006
:1062280061FE00948DF804408DF8054002940394B3
:1062380004942846012469468DF8144005F023FE8D
:1062480028460B212246062305F098FE28462146BB
:1062580005F062FE0BB030BD0020014010B50021F2
:1062680004460122302000F003FEC0B9012001F0ED
:106278001FF8002CB8BF4034E4B210212246302069
:1062880000F0F6FD012001F013F83020112122461C
:1062980000F0EEFD0120BDE8104001F009B810BD86
:1062A80010B5002104460122302000F0E1FDC0B9FC
:1062B800012000F0FDFF002CB8BF4034E4B21221E9
:1062C8002246302000F0D4FD012000F0F1FF3020FC
:1062D8001321224600F0CCFD0120BDE8104000F05B
:1062E800E7BF10BD38B5012205460C463020002115
:1062F80000F0BEFDF0B9012000F0DAFF25EAE572F2
:106308005F2AA8BF5F223B21D2B2302000F0B0FD47
:10631800012000F0CDFF24EAE4725F2AA8BF5F22C3
:10632800D2B230203C2100F0A3FD0120BDE8384066
:1063380000F0BEBF38BD302810B504460ADC10F1A5
:106348007F0F02DB002802DB05E06FF07E0404F516
:10635800807400E03024002130200A4600F088FDD7
:10636800A8B90120E4B200F0A3FF41212246302061
:1063780000F07EFD012000F09BFF302042212246E4
:1063880000F076FD0120BDE8104000F091BF10BD7F
:10639800282810B5044609DC10F1180F02DB002884
:1063A80002DB04E06FF017047F3400E028240021AA
:1063B80030200A4600F05CFDA8B90120E4B200F0E4
:1063C80077FF53212246302000F052FD012000F0D3
:1063D8006FFF30205421224600F04AFD0120BDE81D
:1063E800104000F065BF10BD08B530200021012223
:1063F80000F03EFD60B9012000F05AFF3020332143
:10640800402200F035FD0120BDE8084000F050BFF3
:1064180008BD10B530200021012200F029FD0446F6
:1064280060B9012000F044FF30203321224600F0FB
:106438001FFD0120BDE8104000F03ABF10BD10B5A7
:1064480030200021012200F013FD0446A0B90120EC
:1064580000F02EFF34212246302000F009FD0120F3
:1064680000F026FF30203721224600F001FD0120F0
:10647800BDE8104000F01CBF10BD4020EEE64020F3
:106488000EE708B500210122302000F0F1FC0120C0
:1064980000F00EFF30203421024600F0E9FC012014
:1064A80000F006FF30203721024600F0E1FC012011
:1064B800BDE8084000F0FCBE08B5002101223020EC
:1064C80000F0D6FC012000F0F3FE302034210C222D
:1064D80000F0CEFC0120BDE8084000F0E9BE000055
:1064E800184B1949D3ED006A93ED017A00231A4637
:1064F8009FED166A03E0F0EE476AB0EE677A505EE9
:1065080005EE900AF8EEE57A0133C7EE867A9BB27B
:1065180018B204327F2877EEE67AECDD27EE077AA8
:1065280007EEA77A0A49074A0B80BDEEC77A00230F
:1065380013605360C2ED027A17EE102A054B9200E1
:106548001A607047B00C0020902700200000FA4520
:10655800C03B00205C1800202DE9F84F2E4B2F4A35
:1065680019682F4B19B92F4911602F4A02E02F499A
:1065780011602F4A1A602F4BDFF8BCA0DFF8BC90DF
:10658800DFF8BCB000221A80244A9846176830E029
:1065980007EB84036500B3F9023007EE103AF8EE12
:1065A800C77A013617EE900A08F028FA18A3D3E93B
:1065B800002308F077FA08F00FFD29F815002AF8EB
:1065C800140037F9243007EE103AF8EEC77A01358F
:1065D80017EE900A08F012FA0DA3D3E9002308F089
:1065E80061FA08F0F9FC2BF8140029F81500A8F84E
:1065F8000060B8F8006034B2FF2CC9DD00F05EF826
:1066080000F06AF801F07CF9BDE8F84F68E700BFD0
:106618009A9999999999E93F5018002044180020AF
:106628007C160020922F0020922B00209237002009
:1066380092330020C03B00209023002090270020A8
:106648009025002010B50B4C204605F0CAFE0A4BD9
:1066580018600A4805F0C5FE094B1860FFF77CFF73
:10666800084B0949012220469A81BDE8104005F0EF
:1066780039BF00BF106002405018002088600240F7
:106688006C180020B00C002020800010014B186806
:10669800704700BF5C18002008B5054B05481988ED
:1066A8000022012309F0B6F9034B187008BD00BF9A
:1066B8007000002078230020941E0020034804491D
:1066C800044A4FF4807309F01DBA00BF740000201B
:1066D800902300207621002003480449044A4FF4FF
:1066E800807309F00FBA00BF8000002090250020B9
:1066F800B019002038B505460C460135C1F307210D
:1067080000F0E4FDA8B2E1B200F0E0FD00B238BD4F
:1067180038B5044600F0EEFC01340546A0B200F09E
:10672800E9FCEDB2C0B240EA052000B238BD37B589
:106738000B0E8DF804300B0C8DF805300B0A8DF814
:1067480006308DF80710002400E0284601AB451CF0
:10675800E15C013400F0BAFD042CADB2F5D13EBDC8
:1067680037B5002400E02846451C00F0C3FC01AB07
:10677800ADB2E0540134042CF5D19DF805009DF824
:106788000430000440EA03609DF8073018439DF880
:10679800063040EA03203EBD38B50446642000F0C8
:1067A80087FD25786068AD00EDB2257006F031FAF6
:1067B800237A40FA03F000F003000543104B2570DC
:1067C80005F00F055A5D6378D218D2B2D3B2013200
:1067D800D2B2022A637001D80022A2705BB2012BE8
:1067E80003DD0123A3700023637094F901300133A2
:1067F80003DAFF23A3700023637094F9020038BD05
:10680800EA570408F7B504200121234F06F044FD98
:1068180002AD01214FF48040012406F06DFD0026F1
:106828004FF4B0733846694645F8083D8DF8046062
:106838008DF8074006F088F91020214606F02CFD57
:1068480078236946154800938DF804608DF8074051
:1068580006F07AF90420214606F01EFD21464FF481
:10686800804006F049FD1C233846694600938DF8A0
:1068780004608DF8074006F067F90220214606F00B
:106888000BFDB02306488DF8046069468DF8074073
:10689800009306F059F9FEBD0008024000100240BE
:1068A80000040240802108B5034806F0ACF9D0F195
:1068B800010038BF002008BD0004024008B54FF4AD
:1068C8008071044806F09FF9D0F1010038BF00201C
:1068D80008BD00BF0008024008B5FFF7E3FF08B194
:1068E800FFF7ECFFC0B208BD10B5642000F0E0FC73
:1068F8000F48FFF751FF044610B90E4B187009E016
:10690800FFF7DCFF30B9002C0A4B01DD012200E063
:10691800FF221A700848FFF73FFF0028074B01D1F4
:10692800187010BD01DD012200E0FF221A7010BDB1
:10693800C00000205C420020CC000020902B0020EA
:1069480007B50220012106F0A7FC012300938DF86A
:10695800043002238DF805300448002369468DF879
:1069680006308DF8073006F0EFF80EBD000402403F
:1069780010B5084C01210022204606F05AF940F2D1
:10698800FF4000F095FC012120460A46BDE8104072
:1069980006F04FB90004024008B5FFF7E9FF0021EF
:1069A8000A46302000F064FA012000F081FC012141
:1069B8000A46302000F05CFA012000F079FC002142
:1069C8000122302000F054FA012000F071FC01216E
:1069D8000822302000F04CFA012000F069FC022166
:1069E8000122302000F044FA012000F061FC00216F
:1069F8000A46302000F03CFA012000F059FC1B2127
:106A0800CD22302000F034FA012000F051FC04219E
:106A18000322302000F02CFA012000F049FC062166
:106A28000822302000F024FA012000F041FC072160
:106A38000A46302000F01CFA012000F039FC082139
:106A48008022302000F014FA012000F031FC1E21D1
:106A5800B022302000F00CFA012000F029FC0521BA
:106A68009122302000F004FA012000F021FC0D21D1
:106A78000322302000F0FCF9012000F019FC0E215F
:106A88000022302000F0F4F9012000F011FC14215C
:106A98008022302000F0ECF9012000F009FC0B21E5
:106AA8008822302000F0E4F9012000F001FC3020B9
:106AB8000C21822200F0DCF9012000F0F9FB122100
:106AC8008822302000F0D4F9012000F0F1FB1321D6
:106AD8008C22302000F0CCF9012000F0E9FB0021E5
:106AE8000122302000F0C4F9012000F0E1FB0C2164
:106AF8000822302000F0BCF9012000F0D9FB0D215C
:106B08000822302000F0B4F9012000F0D1FB0E215A
:106B18000822302000F0ACF9012000F0C9FB0F2159
:106B28000822302000F0A4F9012000F0C1FB002168
:106B38000A46302000F09CF9012000F0B9FB402102
:106B48000222302000F094F9012000F0B1FB00226D
:106B58004121302000F08CF9012000F0A9FB302001
:106B68003F21D42200F084F9012000F0A1FB00218C
:106B78000122302000F07CF9012000F099FB10215F
:106B88000F22302000F074F9012000F091FB112150
:106B98000F22302000F06CF9012000F089FB12214F
:106BA8000022302000F064F9012000F081FB13215D
:106BB8000022302000F05CF9012000F079FB092167
:106BC8003C22302000F054F9012000F071FB002134
:106BD8000122302000F04CF9012000F069FB302040
:106BE8003421024600F044F9012000F061FB302016
:106BF8003721024600F03CF9012000F059FB36210C
:106C08000322302000F034F9012000F051FB392133
:106C18000322302000F02CF9012000F049FB3B2131
:106C28003C22302000F024F9012000F041FB3C21F7
:106C38000A46302000F01CF9012000F039FB002141
:106C48000A46302000F014F9012000F031FB5121F0
:106C5800C022302000F00CF9012000F029FB302080
:106C68005221002200F004F90120BDE8084000F09C
:106C78001FBB00BF2DE9F04F454E464D93B0012193
:106C88004FF4001006F008FB304605F0ABFA4FF061
:106C9800C0630293404B0393404B002404934FF48A
:106CA80000794FF400334FF480684FF400674FF4D5
:106CB800005A4FF4807B304602A90C930193099740
:106CC800CDF8189005940794CDF82080CDF828A029
:106CD800CDF82CB00D9405F011FB22463046304912
:106CE80005F067FB3046012105F06DFB01210A46DE
:106CF8004FF0402006F03EFD284605F073FA294A79
:106D0800019B0392284A0C9304922846402202A928
:106D1800059209970294CDF818900794CDF8208031
:106D2800CDF828A0CDF82CB00D9405F0E7FA22464E
:106D380028461E4905F03DFB2846012105F043FB86
:106D480042F2107701220221194806F013FD384655
:106D580000F0AEFA3046012105F00BFB0121284670
:106D680005F007FB384600F0A3FA0B238DF84430F2
:106D780011A801238DF845408DF846408DF847301D
:106D880000F01AFD384600F093FA13B0BDE8F08F12
:106D980010600240886002400C400040923700209A
:106DA800922F00200C3C004092330020922B0020B0
:106DB800003C004002481021012205F051BB00BFF1
:106DC8001060024013B50220012106F065FA4FF465
:106DD80010730E4C009302238DF804308DF80530A3
:106DE80001238DF806302046002369468DF80730C8
:106DF80005F0AAFE20460621042205F025FF2046BC
:106E08000921042205F020FF1CBD00BF0004024038
:106E180030B5154D85B001214FF4001006F060FA29
:106E2800284605F027FF0023ADF804304BF6FF7322
:106E3800ADF806303323ADF808304FF48063ADF871
:106E48000A304FF48043ADF80C3004AC074B2846A9
:106E5800012144F8103D05F0AFFF2846694605F0CA
:106E680037FF05B030BD00BF00540040801A06004F
:106E780073B54FF4961306460D461446019304E085
:106E8800019B5A1E0192002B57D031484FF4003114
:106E980006F0AAF80028F3D12D48012105F098FF43
:106EA8004FF48053019304E0019B5A1E0192002B7A
:106EB80045D02748274906F082F80028F4D024480E
:106EC8003146002205F09CFF4FF48053019304E003
:106ED800019B5A1E0192002B33D01D481E4906F013
:106EE8006EF80028F4D01A48294606F00CF84FF43A
:106EF8008053019303E0019B5A1E01921BB314486F
:106F0800164906F05CF80028F5D01148214605F02E
:106F1800FAFF4FF49613019303E0019B5A1E019266
:106F28009BB10B480E4906F05FF80028F5D00848D9
:106F3800012105F059FF002008E0012006E00220A9
:106F480004E0032002E0042000E005207CBD00BF2F
:106F58000054004001000300820007008000070081
:106F68000400001037B54FF4961304460D460193FC
:106F780005E0019B5A1E0192002B00F09B805648A9
:106F88004FF4003106F030F80028F2D152480121C0
:106F980005F01EFF4FF48053019305E0019B5A1E34
:106FA8000192002B00F088804B484C4906F007F806
:106FB8000028F3D048482146002205F021FF4FF46D
:106FC8008053019304E0019B5A1E0192002B75D057
:106FD8004148434905F0F3FF0028F4D03E482946CC
:106FE80005F091FF4FF48053019304E0019B5A1E72
:106FF8000192002B64D038483A4905F0F5FF002883
:10700800F4D03548012105F0E3FE4FF48053019395
:1070180004E0019B5A1E0192002B53D02E482F49A1
:1070280005F0CDFF0028F4D02B482146012205F0B9
:10703800E7FE4FF48053019304E0019B5A1E01922E
:10704800002B41D0244C2849204605F0CDFF0028CC
:10705800F3D02046002105F0DBFE20460121238BDA
:1070680005F0C2FE4FF48053019304E0019B5A1EC1
:107078000192002B2AD018481C4905F0B5FF0028BA
:10708800F4D0154805F041FF4FF480530193124A9C
:1070980003E0019B591E0191D3B113889B05F8D4D5
:1070A800012104460C4805F0B3FE0B48104905F0D1
:1070B800B5FF0EE001240CE002240AE0032408E0F6
:1070C800042406E0052404E0062402E0072400E086
:1070D800082420463EBD00BF0054004001000300C4
:1070E8008200070004000010020000104000001099
:1070F8000004001013B54FF496130446019305E0FD
:10710800019B5A1E0192002B00F0B08061484FF499
:10711800003105F069FF0028F2D15E48012105F031
:1071280057FE4FF48053019305E0019B5A1E0192CC
:10713800002B00F09D805748574905F040FF002874
:10714800F3D05448A021002205F05AFE4FF4805392
:10715800019305E0019B5A1E0192002B00F08A80E2
:107168004C484E4905F02BFF0028F3D0C4F3052105
:10717800484805F0C8FE4FF48053019304E0019B92
:107188005A1E0192002B77D04248454905F02CFF42
:107198000028F4D0E1B23F4805F0B5FE4FF4805323
:1071A800019304E0019B5A1E0192002B66D03948D6
:1071B8003B4905F019FF0028F4D03648012105F0B5
:1071C80007FE4FF48053019304E0019B5A1E01927D
:1071D800002B55D02F48304905F0F1FE0028F4D097
:1071E8002C48A121012205F00BFE4FF48053019396
:1071F80004E0019B5A1E0192002B43D0254C2949DB
:10720800204605F0F1FE0028F3D02046002105F0C5
:10721800FFFD20460121238B05F0E6FD4FF4805346
:10722800019304E0019B5A1E0192002B2CD01948AF
:107238001D4905F0D9FE0028F4D0164805F065FE72
:107248004FF480530193134A03E0019B591E0191A7
:10725800E3B113889905F8D4012104460D4805F0D7
:10726800D7FD0C48114905F0D9FE10E001240EE0C5
:1072780002240CE003240AE0042408E0052406E0C4
:10728800062404E0072402E0082400E0092420463C
:107298001CBD00BF0054004001000300820007002D
:1072A800040000100200001040000010000400104C
:1072B80082B0002304E0019B01330193009B01335A
:1072C8000093009B8342F6D302B0704737B54FF462
:1072D800805304460D46019304E0019B5A1E019217
:1072E800002B6ED03D484FF4003105F07DFE00289C
:1072F800F3D13A48012105F06BFD4FF48053019317
:1073080004E0019B5A1E0192002B5CD0334834499B
:1073180005F055FE0028F4D03048A021002205F0E1
:107328006FFD4FF48053019304E0019B5A1E0192B4
:10733800002B4AD029482B4905F041FE0028F4D0FB
:10734800C4F30521254805F0DEFD4FF48053019371
:1073580004E0019B5A1E0192002B38D01F48224995
:1073680005F02DFE0028F4D0E1B21C4805F0CBFD55
:107378004FF48053019303E0019B5A1E019243B3DB
:107388001648194905F01BFE0028F5D01348294670
:1073980005F0B9FD4FF49613019303E0019B5A1EC3
:1073A8000192C3B10D48114905F01EFE0028F5D021
:1073B8000A48012105F018FD0D48FFF779FF002064
:1073C8000AE0012008E0022006E0032004E004208F
:1073D80002E0052000E006203EBD00BF005400404A
:1073E800010003008200070080000700040000106D
:1073F800A0860100F7B54FF4805304460D461646A3
:10740800019304E0019B5A1E0192002B75D041485C
:107418004FF4003105F0E8FD0028F3D13D48012183
:1074280005F0D6FC4FF48053019304E0019B5A1EEB
:107438000192002B63D03748374905F0C0FD00287A
:10744800F4D03448A021002205F0DAFC4FF4805330
:10745800019304E0019B5A1E0192002B51D02D4844
:107468002E4905F0ACFD0028F4D0C4F305212948C5
:1074780005F049FD4FF48053019304E0019B5A1E27
:107488000192002B3FD02348254905F098FD00289C
:10749800F4D0E1B21F4805F036FD4FF48053019354
:1074A80004E0019B5A1E0192002B2ED019481C495A
:1074B80005F085FD0028F4D000244FF4961710E05D
:1074C800295D144805F01FFD019703E0019B5A1E32
:1074D8000192E3B10F48134905F086FD0028F5D065
:1074E8000134E3B2B342EBD30A48012105F07CFC36
:1074F8000D48FFF7DDFE00200AE0012008E0022029
:1075080006E0032004E0042002E0052000E0062055
:10751800FEBD00BF005400400100030082000700C8
:107528008000070004000010A086010013B50520A4
:10753800012105F0B1FE184C4FF4E05300930223EB
:107548008DF804308DF805302046002369468DF803
:1075580006308DF8073005F0F7FA20460A21062292
:1075680005F072FB20460C21062205F06DFB062271
:1075780020460B21A4F5006405F066FB4FF4004398
:1075880020466946009305F0DFFA20460F210622BF
:1075980005F05AFB1CBD00BF000802401FB5044699
:1075A800FFF7CEF9FFF734FCFFF7F6F9FFF7BEFF58
:1075B80001214FF4004005F093FE02940F4C102374
:1075C800ADF80230204600236946ADF80430ADF826
:1075D8000C30ADF80030ADF8063005F0B0FF694664
:1075E8004FF0402006F07FF82046012106F02FF8E2
:1075F8004FF04020012106F02AF81FBD003C004052
:10760800014B1860704700BFCC0C0020704710B5C4
:107618000A4A1379262B04D80949C854013313712F
:1076280010BD074A0123591ED45C0133272B54543B
:10763800F9D1034B83F8260010BD00BFCC0C002005
:10764800943B0020704710B504462078FFF7DFFF11
:1076580014F8013F002BF8D110BD38B504460D468B
:10766800013D14F8010BEDB2FFF7D1FF002DF7D162
:1076780038BD00BF014B1878704700BFD40C0020FC
:10768800014B5878704700BFD40C0020024B187883
:1076980080F00100704700BFD40C0020024B00228C
:1076A8001A705A70704700BFD40C0020014B012299
:1076B8001A707047D40C0020014B01225A70704791
:1076C800D40C002082B0002304E0019B0133019315
:1076D800009B01330093009B8342F6D302B07047AE
:1076E80007B50420012105F0D7FD01214FF48040A2
:1076F80005F002FE4FF40073009300238DF8043068
:107708000348012369468DF8073005F01DFA0EBDC0
:10771800000802400D4B07B51A680D484FF47A73FC
:10772800B2FBF3F20B4B013A5A600B4AF02182F894
:10773800231000229A6007221A60084B084A009317
:107748000121084B03F02EFF0EBD00BF9C01002055
:10775800683C002010E000E000ED00E0B8020020E6
:107768009C02002004020020054B1A6812B11A6816
:10777800013A1A60034B1A6801321A60704700BF59
:107788001C3C0020343C002082B0044B0190019A3C
:107798001A601A68002AFCD102B070471C3C00200D
:1077A800704700BF40F0BE60024B40F42020D86014
:1077B800704700BF00ED00E0C37810B503B3164B67
:1077C8004278DB688478DB43C3F30223C3F1040106
:1077D800C9B202FA01F10F2242FA03F2C9B22240F9
:1077E8000A430E4B01781201CB18D2B283F800235A
:1077F80003780122590903F01F0302FA03F307E093
:1078080003780122590903F01F0302FA03F3203118
:10781800024A42F8213010BD00ED00E000E100E02E
:1078280021F0604121F07F01014B084398607047C7
:1078380000ED00E0044B1A6909B1104301E022EAA7
:1078480000001861704700BF00ED00E0044B1A68A3
:1078580004280CBF42F0040222F004021A607047A8
:1078680010E000E000000000034A044B1A60044ADC
:10787800044B1A60704700BF0000FA4564180020E6
:10788800DB0FC93F60180020034B00221A60034A2F
:10789800034B1A60E8E700BF904200200000FA4559
:1078A8005C17002007EE100A024BF8EEC77AC3ED0A
:1078B800007A70475C17002038B510EE100A07F000
:1078C8009DF80DA3D3E9002307F0ECF8084B044614
:1078D80018680D4607F092F80B46024629462046DE
:1078E80007F00AFA07F0C0FB024B186038BD00BF6A
:1078F8006418002060180020182D4454FB211940FA
:107908002DE9F04F2DED068B6F4CDFF8F0A189B013
:107918000027A34637F80A506C4B2580FE5A6C4B5B
:107928006680186807F06AF865A3D3E9002307F0B2
:10793800B9F807F051FB6368664AC018011101F5F0
:1079480080610905090D6060C0F30B100DF1200C72
:1079580032F8203032F82120616A238115FB02F0C9
:10796800628115FB03F516FB02F216FB03F60CEB1E
:107978004103E0602561C0F3CF30C5F3CF356261C4
:10798800A661C2F3CF32C6F3CF3623F8200C23F812
:10799800105C23F8182C23F8086C4F4BA083013196
:1079A8000B40002BE5832284668403DA013B63F0F5
:1079B80003030133CBF82430002B76D14748484ADB
:1079C8006946042308F05EFB4648474A04A9042395
:1079D80008F058FB4548464A02A9042308F052FB20
:1079E800444A454806A9042308F04CFBB4F928305A
:1079F80007EE903AB4F92A30B8EEE79A07EE903AD3
:107A0800B4F92C30B8EEE78A07EE903AB4F92E3084
:107A1800F8EEE79A07EE903AF8EEE78A68EE087A09
:107A280049EE097A17EE900A06F0E8FF41EC100BD0
:107A380009F08AF951EC100B07F016FB68EEA87AEA
:107A480049EEA97A0AEE100A206317EE900A06F0AA
:107A5800D5FF41EC100B09F077F951EC100B07F04A
:107A680003FB68EE897A58EE297A28EE288A0AEE0E
:107A7800900A606309EE298A17EE900A06F0BEFFA5
:107A8800804618EE100A894606F0B8FF49EC108BBC
:107A980041EC110B09F0D0F88AEE2AAA51EC100B30
:107AA80007F0E2FA84ED0FAAA0630237B7F5007F6A
:107AB8007FF430AF09B0BDEC068BBDE8F08F00BF96
:107AC80039D6C56D305FC440E40C0020B0190020E1
:107AD800601800200458040803000080B400002047
:107AE8000C0D0020A80000200E0D00209C00002096
:107AF800100D0020120D002090000020762100209B
:107B0800014B93ED0F0A7047E40C0020014B93EDF5
:107B18000E0A7047E40C0020014B93ED0C0A7047E5
:107B2800E40C0020014B93ED0D0A7047E40C002093
:107B380010B5FEF725F90020012324210246FEF79F
:107B480089F9114B1C780020012C05D10146FEF75C
:107B58005AFA2046002104E00721FEF754FA0120D2
:107B68000721FEF750FA63221221C020FFF780F99F
:107B780002200121FEF747FAFEF724FB0120BDE8A9
:107B88001040FEF714BB00BF2C0E00200D4B1B78D5
:107B9800012B05D10C4B0D4A196812688A181A6016
:107BA8000B4B1B78012B084B196805D1094A9142E8
:107BB80007DD01321A607047074A914201DD013240
:107BC8001A607047F43B002060420020F03B002020
:107BD8002C0E00207FD1F008FF1FA1070E4B1B7849
:107BE800012B05D10D4B0E4A196812688A1A1A60C2
:107BF8000C4B1B78012B094B05D10B4A1968914294
:107C080008DC1A6070471A68B2F57A2FDCBF4FF4A7
:107C18007A221A60704700BFF43B002060420020BF
:107C2800F03B00202C0E002040420F00024B1A6847
:107C3800024B1A60704700BF543C0020604200208D
:107C48002DE9F04F824658488BB0B0FBF1F00C4656
:107C580006F0B2FE41EC100B08F0EAFE51EC100BF6
:107C680007F0E2F9C307074648BF471E04FB07F0C1
:107C780006F0A2FE46A3D3E9002307F03DF8044628
:107C88000D4645EC104B08F0D3FE59EC108B2046FE
:107C980042464B46294606F051FDCDE904014946C6
:107CA800404607F0C1F93CA3D3E900230990DDE978
:107CB800040107F073F900283DD1002401234FF097
:107CC8001509224698462046DFF8E4B003E023462B
:107CD80042462C46B04600FB04355D452ED800FBD5
:107CE8000826DDE904012EA3D3E9002307F056F99D
:107CF80030BBDDE9042300202C4906F0FDFF41ECF0
:107D0800100B0390029108F093FE0398029953EC2C
:107D1800102B8DED060B06F011FD09F1FF39CDE9A9
:107D280004015FFA89F9DDE9060107F07DF9B9F187
:107D3800000FCCD104E00125002601E02546464687
:107D4800099BD9B2BAF1000F0BD132462B465046E7
:107D5800FEF780F801230093504651463A465346B1
:107D680009E032462B460120FEF774F80120009006
:107D780001463A460023FEF760F9FEF723FA012090
:107D88000BB0BDE8F04FFEF712BA00BFAFF30080AA
:107D98000000000084D77741956479E17FFDA53D17
:107DA800BBBDD7D9DF7CDB3D00E9A4350000F03F3F
:107DB800FFFF0F0038B5284B1B78022B4AD0274B02
:107DC800274A1968274B284C1B68CB189342236015
:107DD80018DC0020FFF734FF01202168FFF730FF8F
:107DE800224B1C780020012C05D10146FEF70BF927
:107DF8002046002104E00721FEF705F901200721AC
:107E0800FEF701F91A4B1B78022B14D1194B1A4DA6
:107E18001A68124C2B68D31822689A420BDA174B4F
:107E28001B78012B07D1164B186800F081F82268DF
:107E38002B68D3182360084B1A78012A0AD10D4AF7
:107E480011680D4A12688A1804490968914201DBD1
:107E580002221A7038BD00BFE443002060420020AF
:107E680080D1F0087C420020804200202C0E0020A7
:107E7800F43B0020443C0020F03B00203C3C002028
:107E88000C3C0020AFF3008008B5FEF70BFD094B52
:107E98005A78187002435A701AB19A7801329A7057
:107EA80030B99B78034A012B02D900235370937091
:107EB80008BD00BF240D002007B50420012105F0EE
:107EC800EBF94FF46043009301238DF8043002234B
:107ED8008DF805300448002369468DF806308DF882
:107EE800073004F031FE0EBD00080240084B1A6846
:107EF8004FF47A73B2FBF3F2064B013A5A60064A22
:107F0800F02182F8231000229A6007221A60704735
:107F18009C01002010E000E000ED00E0034B5A68EF
:107F280012B15A68013A5A60704700BF240D002008
:107F3800024B58605A68002AFCD17047240D002073
:107F480030B585B004460D4601A85C490A220BF0FD
:107F58008BF95B4B1B78032B10D8DFE803F0020585
:107F6800080B01A8574907E001A8574904E001A8F0
:107F7800564901E0564901A80BF060FA04AA131902
:107F880013F80C3C5D19EDB22F2D01D80A3502E02B
:107F9800392D01D90A3DEDB204AB1C194FF6FF701B
:107FA80004F80C5CFCF758FE0020FCF74BFF0DF1C1
:107FB80003050F24204623345A21002315F8012FE6
:107FC800A4B2FCF759FFB4F5A57FF3D164205A2178
:107FD8002C220023FCF750FF0023CD205A212C220D
:107FE800FCF74AFF0020FCF737FE354B1B78032BC4
:107FF80062D8DFE803F002284B5601A931480BF09C
:108008001DFA0A2200212F480BF0BCFB314A324BE3
:1080180012781860012A06D1304A904201DC0132F8
:108028001A602F4A06E0B0F5FA5FBCBF4FF4FA5267
:108038001A602C4A1B689342C4BF274B1A602A4B0C
:108048001A682A4B20E001A91F480BF0F7F90A2209
:1080580000211D480BF096FB1E4A254B127818602C
:10806800012A06D11D4A904201DC01321A601C4ADD
:1080780006E0B0F5FA5FBCBF4FF4FA521A60194A2D
:108088001B68934218DD1A4B1A6015E001A90F48C6
:108098000BF0D4F90D4800210A220BF073FB154BA5
:1080A80009E001A90A480BF0C9F9094800210A2288
:1080B8000BF068FB104B186005B030BD519B0508EC
:1080C800523C0020203C0020483C00206542002013
:1080D800103C00202C0E0020643C00203F420F0082
:1080E80080D1F00840420F00543C0020604200203C
:1080F80084420020584200200C3C002010B50D4B53
:108108000D4C1A680D4821460BF070F90C4B0D48C0
:108118001A6821460BF06AF90B4B0C481A6821467D
:108128000BF064F90A4B0B481A682146BDE8104069
:108138000BF05CB9643C00205B9B0508203C0020E8
:1081480084420020483C002058420020654200201C
:108158000C3C0020103C00209FED010A704700BF36
:10816800000000009FED010A704700BF00000000FA
:108178009FED010A704700BF00000000054B83ED2A
:10818800000AC3ED010A83ED021AC3ED031A83ED59
:10819800042A7047BC450020054B83ED050AC3ED52
:1081A800060A83ED071AC3ED081A83ED092A7047FA
:1081B800BC450020044B18B1012801D1034A00E056
:1081C800034A12681A60704760420020443C00204D
:1081D800543C002010B9034B18687047024B1868CC
:1081E800704700BF643C0020543C002010B9034B8A
:1081F80018687047024B1868704700BF8442002017
:10820800443C002008B54FF49570FEF781FA40F21F
:108218006523C31A584240EB030008BD08B5C620C1
:10822800FEF776FA40F28D13C21A504240EB020074
:1082380008BD4FF4957040F26521FEF75BBAC62081
:1082480040F28D11FEF756BA08B50020F8F7C4FAC7
:10825800BCEEC00A4FF4967010EE101AFEF767FADB
:108268000020F8F7C7FABCEEC00A4FF4987010EE79
:10827800101AFEF75CFA0020F8F7CAFABCEEC00A3A
:108288004FF49A7010EE101AFEF751FA0020F8F722
:10829800CDFABCEEC00A4FF49C7010EE101AFEF72F
:1082A80046FA0020F8F7D0FABCEEC00A4FF49E70E8
:1082B80010EE101AFEF73BFA0120F8F78DFABCEE23
:1082C800C00A4FF4A07010EE101AFEF730FA012021
:1082D800F8F790FABCEEC00A4FF4A27010EE101A2C
:1082E800FEF725FA0120F8F793FABCEEC00A4FF41E
:1082F800A47010EE101AFEF71AFA0120F8F796FA91
:10830800BCEEC00A4FF4A67010EE101AFEF70FFA72
:108318000120F8F799FABCEEC00A4FF4A87010EEE5
:10832800101ABDE80840FEF702BA2DE9F04F85B0F3
:10833800FFF768FF002875D04FF49670FEF710FA23
:10834800624ADFF8BCB110604FF498700192FEF7F2
:1083580007FA5F4BDFF8ACA118604FF49A700293EC
:10836800FEF7FEF9CBF800004FF49C70FEF7F8F921
:10837800CAF800004FF49E70FEF7F2F9DFF8889112
:10838800DFF88881C9F800004FF4A070FEF7E8F91B
:10839800C8F800004FF4A270FEF7E2F94D4F4E4EB8
:1083A80038604FF4A470FEF7DBF930604FF4A67024
:1083B800FEF7D6F9494D4A4C28604FF4A870FEF7ED
:1083C800CFF920604FF4AA70FEF7CAF94549086052
:1083D8004FF4AC700391FEF7C3F984464248C0F8E5
:1083E80000C0029B41481B68019AC360DBF800305B
:1083F80003990361DAF8003012684361D9F8003054
:1084080082608361D8F80030C0F834C0C3613B682B
:108418000362336843622B6883622368C3620B6814
:1084280003630EE0314B324C324833499C600022E2
:10843800DA6018615A619961DC611A6258629A625D
:10844800D9622A4A2D4B116BD2ED023AD2ED034A7A
:10845800D2ED045AD2ED056AD2ED067A92ED073ACA
:1084680092ED084A92ED095A92ED0A6A92ED0B7A5A
:10847800C3ED003AC3ED014AC3ED025AC3ED036AE6
:10848800C3ED047A73EE633A74EE644A75EE655A86
:1084980076EE666A77EE677A526BD96383ED053AB2
:1084A80083ED064A83ED075A83ED086A83ED097A5E
:1084B800C3ED0A3AC3ED0B4AC3ED0C5AC3ED0D6A7E
:1084C800C3ED0E7A1A6405B0BDE8F08F480E00209F
:1084D800500E0020680E0020600E0020300E002094
:1084E800340E00206C0E00203C0E0020240D0020CD
:1084F8000000F04200008CC2CCBC8C2CBC45002093
:10850800640E00204C0E00205C0E0020580E002047
:1085180060EEA00AB7EE007AF0EE606A70EE077AB5
:1085280040EE006A47EEA70A36EEC77A08B5C7EEEE
:10853800200A10EE900A06F061FA0022084B06F0B5
:10854800B1FA0022074B06F0FBF806F08DFD07EEA6
:10855800900AFDEEE77A17EE900A9F3008BD00BF3B
:10856800000059400000E03F38B52DED028BF7EED2
:10857800008AB0EE608A70EE288A10EE900A28EE23
:10858800088A06F03BFA08EEA88A00220F4B06F08C
:1085980089FA044618EE100A0D4606F02FFA02462C
:1085A8000B462046294606F0A7FB0022084B06F09A
:1085B800C7F806F059FD07EE900AFDEEE77A17EEC8
:1085C800900A7730BDEC028B38BD00BF00006940CF
:1085D8000000E03FF0B56A4D2DED068B95E80F00E1
:1085E8008DB008AE103586E80F000FCD01AC0FC472
:1085F80095E807004FF6FF7384E807009F2077216E
:108608006422FAF7B8F9A020772164224FF6FF73A5
:10861800FAF7B1F99E20772164224FF6FF73FAF733
:10862800AAF99F20762164224FF6FF73FAF7A3F97F
:108638004FF6FF73782164229F20FAF79CF90020F7
:10864800FCF766F99F2077216522FCF73BFB9F200A
:1086580077216422FCF736FB07AD0C36F7EE009A5B
:108668000435F7EE008A95ED009A4FF49674B0EE53
:1086780068AA18EE900A06F0C1F93FA3D3E90023CF
:1086880006F010FA06F0F0FC08EE900A38EEE98AD7
:10869800B0EE490AF0EE480AFFF73AFFB0EE490A91
:1086A800F0EE480A0746FFF75FFFBFB281B20F221C
:1086B8003846FCF73AF8013CDBD14FF49674F7EEF4
:1086C800008A18EE900A06F099F92BA3D3E9002343
:1086D80006F0E8F906F0C8FC08EE900A39EEE88AD8
:1086E800B0EE490AF0EE480AFFF712FFB0EE490A69
:1086F800F0EE480A0746FFF737FFBFB281B20F22F4
:108708003846FCF712F8013CDBD1B542A8D16C46DB
:1087180007AE043494ED009A4FF4C875F7EE008A5A
:1087280018EE900A06F06AF913A3D3E9002306F0BD
:10873800B9F906F099FC08EE900A38EECA8AF0EE0C
:10874800490AB0EE480AFFF7E3FEB0EE480AF0EE39
:10875800490A0746FFF708FFBFB281B20022384630
:10876800FBF7E3FF013DDBD1B442D2D10DB0BDEC44
:10877800068BF0BDAFF30080295C8FC2F528F03F6F
:1087880004980408121A06EE902A081AB8EEE67A37
:1087980006EE900AF8EEE67AC7EE277A9FED047A9D
:1087A80067EE877AFDEEE77A17EE900A704700BF0A
:1087B8000000A0438A1A06EE902A081AB8EEE67A54
:1087C80006EE900AF8EEE67AC7EE277A9FED047A6D
:1087D80067EE877AFDEEE77A17EE900A704700BFDA
:1087E8000000484370B506460D460024610704D5CD
:1087F800A0B231462A46FBF798FF0134B4F5A07FB2
:10880800F4D170BD70B506460D460024600704D546
:10881800A1B230462A46FBF788FF0134C82CF5D1AF
:1088280070BD114B11481B781149124A0068012B81
:10883800114B09D1126808601A60104B1A68104B66
:108848001A60104B1A680CE01268D2011A600B4BC0
:108858001A680B4BD2011A600A4B1A68C0010860EB
:10886800D201094B1A6070472C0E0020643C00208E
:10887800543C002084420020443C00205842002000
:10888800F03B00202C3C00207C420020024B1A6860
:10889800024B1A60704700BF543C00206042002021
:1088A80008B5FFF7BEFFBDE80840EFE770B5002147
:1088B8000A221948194D1A4E1A4C0AF063FF002172
:1088C80028600A2218480AF05DFF002130600A2259
:1088D80016480AF057FF0A222060002114480AF0BF
:1088E80051FF144B326818602B68D31A06EE903A81
:1088F8002368B8EEE67A06EE903AF8EEE67A0E4B82
:10890800C7EE277AFCEEE77A17EE902A01321A8032
:10891800BDE87040C4E700BF203C0020643C002054
:108928008442002058420020483C00206542002034
:10893800103C00200C3C0020904500200022F0B59F
:108948001346202603254FF02C0C00E02646303E27
:10895800F6B217460132092E10F8014B0AD897FBD8
:10896800F5F605FB16772FB9CE1801F803C0747019
:10897800023301E0CC540133092AE7D12022CA543A
:10898800CB1848225A707A229A700022DA70F0BD09
:1089980070B58CB005460C4608A80E491E460AF06C
:1089A80025FD08A86946FFF7C9FF6A460A4904A8D1
:1089B8000AF01CFDBDF84000FCF74EF93046FCF704
:1089C80061F92846214604AA0023FCF773FA0CB083
:1089D80070BD00BF619B0508369905082DE9F04F69
:1089E800CD4B2DED0A8B1B78022BC5B000F0E68429
:1089F800CA4B1A78CA4B22B91A68802392FBF3F93A
:108A080001E0D3F80090C74CC74EE36BC3EB0902F3
:108A180007EE102A226CD31AF8EEC78A07EE103A2E
:108A2800F8EEC77ADFEDC1AAC8EEA78AFFF768F8A3
:108A380086ED0E0AFFF76AF8D4ED0A7A94ED008AFB
:108A480094ED019A08EEA78AD4ED0B7A86ED0F0A09
:108A5800B06B08EEA79A10EE105A05F0CFFF8246C9
:108A680028468B4605F0CAFF41EC100B41EC1B0B66
:108A780007F086FF504653EC102B594606F012F8C3
:108A880006F0F2FAB0EE4B0AF0EE6B0A0AEE100AA4
:108A980008F076F8504653EC102B594606F002F8C9
:108AA80006F0E2FA07EE100AD4ED0C6AD4ED027A69
:108AB80069EE079A48EEA67A58EE0A9A29EE0A9ABB
:108AC80079EEA79A08EE079AD4ED037A94ED0D7A19
:108AD80048EE877A9FED96AA39EE279A954BB4EE21
:108AE800CA9AF1EE10FA69EE097AB1EE49BAC8BF2E
:108AF800B0EE4A9AB4EE6A9A49EEA97AF1EE10FA03
:108B080048BFB0EE6A9AC3ED009A83ED019A19EE58
:108B1800900A8BEE27BAC9EEA7BA05F06FFF0022BC
:108B2800854BCDE9040105F009FE044669EE097A92
:108B38000D4617EE900A05F061FF224682468B46E5
:108B48002B462046294605F0ADFF52465B4605F008
:108B5800F7FD41EC100B08F0F7F80022DDE90401FD
:108B6800754B8DED020B05F0EBFD02460B4605F04B
:108B780099FF52465B4605F0E3FD41EC100B08F007
:108B8800E3F8DDE9020155EC104B06F06DFA2946D1
:108B980008EE100A204606F067FA08EE900AC8EEBA
:108BA800288A664C664DB7EE00CA18EE900A05F0A2
:108BB80025FF53A3D3E9002306F0E6F9DFED617A38
:108BC800002818BFF0EE678AF4EE4C8ADFED5E7A73
:108BD800F1EE10FAC8BFF0EE678ADFED5C7A6BEE53
:108BE800277AC4ED008A17EE900A05F007FFDFED3B
:108BF800587A4BEEEB7A4BEE4B7A82468B4617EE61
:108C0800900AC5E902AB05F0F9FE4BEC10AB41EC5C
:108C1800110BC5E9000108F00FF838EE8C8A3CEE1C
:108C280068CA51EC100B88EE0C8A06F01DFA494B05
:108C38001B7880F0004AB4EE4A8AF1EE10FAC8BFF9
:108C4800B0EE4A8AB4EE6A8AF1EE10FA48BFB0EE86
:108C58006A8A022BC4F804A040F0A6803E4D2C6816
:108C6800002CC0F2A18018EE900A05F0C7FE002281
:108C78003A4B05F017FF06F0D7F9074680465046ED
:108C880005F0BCFE20A3D3E9002305F00BFF20A3C9
:108C9800D3E9002305F054FD06F0C6F9304BC3F8BC
:108CA800009006EBC403C9F30722013483F841207E
:108CB800C9F3074283F8422083F844704FEA1962E7
:108CC800C7F3072783F84600082CC0F3072083F86A
:108CD800409083F8432083F8457083F847002C6060
:108CE80045D1B6F88000002300F580602B6080B283
:108CF80006F140014022FEF77DFB98B3FEE700BF76
:108D08002D431CEBE2361A3FCDCCCCCC0C5FC440D3
:108D180000000000C0FFDF40E44300202C0E0020CC
:108D280060420020BC450020240D0020003C1CC6E9
:108D3800003C1C46DC43002000004940C44200209F
:108D48009845002017B7D13872F97F3F0AD7233DDD
:108D580017B7D139F43B00205C3C00200000F040FC
:108D6800D4430020B6F880304033A6F88030924BC8
:108D7800924C1A88238801339BB29A42238013DCD1
:108D88008F4DB5F8800000F5806080B205F1400194
:108D98004022FEF72FFB00B1FEE78A4BA5F88000C2
:108DA8004FF0FF3220801A60FEF7B6FE844C84ED47
:108DB800210AFEF7B7FE84ED220AFDF767FC4A4652
:108DC800C4F88C00804934A80AF010FBD4F8840059
:108DD80005F014FE02460B4624A87C490AF006FB5F
:108DE800D4F8880005F00AFE02460B4628A8784900
:108DF8000AF0FCFA1BEE900A05F000FE06460F4644
:108E080032463B4673492CA80AF0F0FA1BEE100ACA
:108E180005F0F4FDCDE90201DDE902236E4930A831
:108E28000AF0E4FADDE904236C4910A80AF0DEFA36
:108E380019EE100A05F0E2FDCDE90801DDE9082385
:108E4800674914A80AF0D2FA18EE900A05F0D6FD80
:108E5800CDE90601DDE90623624918A80AF0C6FA39
:108E6800504605F0CBFD82468B4652465B465E492E
:108E78001CA80AF0BBFA18EE100A05F0BFFDCDE9F0
:108E88000A01DDE90A23594920A80AF0AFFA0CA81B
:108E98005749D4F88C200AF0A9FA564B1B78013BA5
:108EA800DBB2012B00F27C82534B1B78072B00F2BC
:108EB8007782DFE813F008007502AB0032016F011A
:108EC800BF014B0217020220FBF7BCFF4FF6FF70F1
:108ED800FBF7D8FE1F20FBF7BFFE19210023474AE6
:108EE8002D20FBF7E7FF4FF6FF70FBF7CBFE0020C6
:108EF8000024FBF7B1FE0F20B4214A464FF6FF735A
:108F08000094FFF745FD0F20772124AA2346FBF79D
:108F1800D1FFA0200DEB000277212346FBF7CAFF03
:108F28000F20412118AA2346FBF7C4FFA0204121A6
:108F38001CAA2346FBF7BEFF0F2065212CAA234657
:108F4800FBF7B8FF30AA2346A0206521FBF7B2FF44
:108F58000F20532110AA2346FBF7ACFFA020532172
:108F680014AA2346FBF7A6FF0F209B2120AA23461D
:108F7800FBF7A0FF124BD3F88C30B3F57A7FCCBF48
:108F88004FF4FC604FF47840FBF77CFE0CAAA0205D
:108F98009B210023FBF78EFF194B1B780221012B25
:108FA8000CBF184A184A4FF48C700023FBF782FF55
:108FB8001F20FBF767FEF3E190450020C042002028
:108FC800240D00205C3C0020669B0508709B05086A
:108FD8007B9B0508869B0508909B05089A9B0508BE
:108FE800A59B0508B09B0508BB9B0508C69B050803
:108FF800D29B0508F43B002078420020DF9B05083F
:109008002C0E0020FE9B0508029C050832463B46B4
:109018003EA8A7490AF0EAF9DDE9022341A8A549D3
:109028000AF0E4F9DDE9042338A8A3490AF0DEF9D7
:10903800DDE908233BA8A1490AF0D8F9E620022176
:109048003EAA0023FBF736FFE620162141AA00239B
:10905800FBF730FF0220C82138AA0023FBF72AFFBC
:109068003BAA00230220DC21FBF724FFDFED947AE2
:1090780068EEA78A4FF6E07518EE900A05F0BEFC78
:109088004BEC10ABCDE9020107F07AFC57EC106B02
:109098004BEC10AB07F074FD00205BEC10ABFBF75A
:1090A800F1FD0A214A46002305200095FFF770FCD0
:1090B8004FF47840FBF7D0FDDDE9020132463B462C
:1090C80005F0F0FC6CA3D3E9002305F039FB05F0AB
:1090D80083FF524684B25B46DDE9020105F0E2FCFB
:1090E80002460B4666A1D1E9000105F027FB05F011
:1090F80073FF81B22046F9F76EFC9D207721052287
:109108000023FBF7D9FD9F20752105220123FBF7DA
:10911800D3FD2846FBF7A0FD42E16A4B18686A4B6D
:109128004A4619689FED698AFFF72CFBF4EEC89A46
:10913800F1EE10FA044614D5F5EEC09AF1EE10FAE5
:109148000FDDFDEEE99A4FF4FA7119EE902A00202E
:10915800FFF730FBA3B281B24FF6FF721846FBF758
:10916800E4FAB4EEC89AF1EE10FA40F11981DFED95
:10917800587AB4EEE79AF1EE10FA40F31181BDEE99
:10918800C99A544819EE102A4FF4FA71FFF712FBE6
:10919800A4B2D6E04B4B18684B4B4A461968FFF708
:1091A800F1FAF5EEC0BAF1EE10FA04461DDD3046CC
:1091B800394635A3D3E9002305F0E6FEA8B134A368
:1091C800D3E900233046394605F06CFC02460B46CD
:1091D8000020414905F0B2FA05F0FEFEA5B281B2C1
:1091E8004FF6FF722846FBF7A0FADDE902012AA331
:1091F800D3E9002305F0E6FE002800F0D180DDE980
:10920800020121A3D3E9002305F0BEFE002800F0E7
:10921800C78023A3D3E90023DDE9020105F042FC5E
:1092280002460B4600202D49A4B205F087FA05F046
:10923800D3FE86E0234B1868234B4A461968FFF78C
:10924800A1FA19A3D3E900230446DDE9060105F0D4
:10925800B9FE68B19DED060B07F0F0FC002251EC59
:10926800100B1F4B05F01EFC05F0B6FE014600E092
:10927800C821A0B289B28FE00000000000E063407E
:109288000000000000C05D409A9999999999B93FEA
:109298000000000000409F409A9999999999B9BF98
:1092A8000000000000408F4089B5F81400E3693FD2
:1092B800069C0508109C05081A9C0508249C0508AE
:1092C8000000C842643C0020844200200000FA43A9
:1092D8000000FAC30CFEFFFF00006940000059407F
:1092E800000054C03C4B18683C4B4A461968FFF7CD
:1092F80049FADFED3B7A48EEE77A84B2FDEEE77A89
:10930800204617EE901A4FF6FF7289B2FBF70DFA56
:109318002DA3D3E900235046594605F0C3FB2CA3DF
:10932800D3E9002305F0E8FC05F09EFE07EE900A5D
:10933800FDEEE77A6FF0B30017EE902AB421FFF73D
:1093480039FA81B24FF4FC62204627E0DFED257A36
:10935800B4EEE78AF1EE10FA22D51F4B18681F4BBE
:109368004A461968FFF70EFA9DED0A0B044607F006
:1093780065FC53EC102B1046194600221A4B05F0D9
:1093880091FB02460B460020184905F0D7F905F075
:1093980023FEA4B281B220464FF6FF72FBF7C5F94F
:1093A800134B1B78022B09D043B14FF6FF73009380
:1093B8000520DC214A460023FFF7EAFA45B0BDEC58
:1093C8000A8BBDE8F08F00BF0000000000807640E7
:1093D8001F85EB51B81E1940643C002084420020D0
:1093E800000048430000C84200005940000069409E
:1093F800784200202DE9F04F774B2DED048B93ED4B
:10940800008A78EE087A83B017EE900A05F0F6FA2B
:10941800724B064618680F4605F0F0FA68EE088A9F
:1094280082468B46F7EE009A4BEC10AB07F0A8FA91
:1094380078EEA97A55EC104B17EE900A05F0DEFA93
:1094480022462B46804689463046394605F02AFB97
:1094580002460B464046494605F070F905F004FE01
:1094680079EEE88A09EE100AC8EE898ADFED5C7A9F
:109478004BEC10AB68EEA78A07F082FB304653EC42
:10948800102B394605F00EFB044619EE100A0D465E
:1094980005F0B4FA02460B462046294605F02CFC96
:1094A800504B002205F0FEFA05F0DEFD4E4B1B780E
:1094B800033B09EE100A042B78D8DFE803F0031207
:1094C8002F58460018EE900A05F098FA044619EE4F
:1094D800100A0D4605F092FACDE9000143484449C7
:1094E80017E029EE098A08EEA88AB1EE499AC8EE73
:1094F800888A89EE088A18EE900A05F07FFA0446F1
:1095080018EE100A0D4605F079FACDE90001374842
:10951800384922462B4609F069FF47E018EE100A41
:1095280005F06CFA41EC100B07F088FB0022324B77
:1095380051EC100B05F0B6FA05F096FD05F05EFA51
:1095480002460B4629482D492EE018EE100A05F070
:1095580055FA1DA3D3E9002304460D465046594643
:1095680005F0A0FACDE9000120482549D1E718EE19
:10957800100A05F043FA16A3D3E9002305F022FDEB
:10958800DFED207A002818BFB0EE678A78EE297AD6
:1095980079EEC89AC7EEA99A19EE900A05F02EFA44
:1095A80002460B461148184909F020FF0F4A0220CD
:1095B800CA21002303B0BDEC048BBDE8F04FFBF7D4
:1095C80079BC00BFAFF30080F6285C8FC2A54C4081
:1095D800AE47E17A14AEEF3FCC420020D0420020E3
:1095E8000000484200004940784200209A4200208A
:1095F8002E9C05083E9C0508000034C04E9C0508BA
:10960800609C0508A4707D3F7C9C050873B50646E0
:10961800002800F0BA80624B18888619B6B232B2B8
:10962800002A05DB40F23F139A42C8BF1E4600E0FD
:1096380000260121FAF7D8FF0120FAF729FE594D33
:109648000024605B0234FAF771FEB4F5C67FF8D1E6
:10965800C722B0B201214EF29C73FBF7DBF9504BE5
:10966800514D1E80514B2C681B6836B206EE906A2D
:109678001B1BB8EEE67A06EE903AF8EEE67A00267C
:1096880067EE277A17EE900A05F0B8F940A3D3E9F8
:10969800002305F031FB05F09FFC4FF6FF732418FB
:1096A800224600930520DC210023FFF771F9404B87
:1096B80028681B68241A94FBF3F005F08DF9002242
:1096C8003C4B3D4C05F03CF805F0CEFC07EE900A0B
:1096D800FCEEE77A17EE905AED00ADB205F580651D
:1096E800A8B2FDF707FD2070681C80B2FDF702FDE7
:1096F8006070A81C80B2FDF7FDFCA070E81C80B269
:10970800FDF7F8FCE070281D80B2FDF7F3FC60F36C
:109718000706681D80B2FDF7EDFC60F30F26B6B2B0
:1097280007EE906AB8EE677ADFED247A244C67EE8C
:10973800277AA81DC4ED007A80B2FDF7DBFC073557
:10974800002660F30706A8B2FDF7D4FC60F30F26E5
:10975800B6B2A6F5FE46FF3E06EE906AF8EEE67A49
:10976800184D17EE900A05F049F90BA3D3E9002329
:1097780005F0C2FA05F078FC134B28601A782046E9
:10978800294602B0BDE8704034E602B070BD00BFA3
:109798000000000000F07340CDCCCCCC0C5FC4407E
:1097A80098420020E6430020643C002084420020C8
:1097B800584200200000E03FD443002000008037DA
:1097C800CC420020D04200207842002013B5104C33
:1097D800B4F89030ADF80630BDF806309BB25BB1F6
:1097E800BDF806004EF29C7380B20121C722FBF738
:1097F80011F90023A4F89030064B1B78022B06D1F0
:10980800054C94F90000FFF701FF002323701CBDED
:10981800240D0020E4430020902B0020444B2DE928
:10982800F0431A88434BDFF80C811988914288BFAE
:109838001A808DB000276BE04FEAC7091FFA89F933
:1098480009F580691FFA89F0FDF754FC60F30704F5
:1098580009F1010080B2FDF74DFC60F30F2409F116
:10986800020080B2FDF746FC60F3174409F10300DB
:1098780080B2FDF73FFC60F31F6409F1040080B279
:10988800FDF738FC60F3070609F1050080B2FDF723
:1098980031FC60F30F2609F1060080B2FDF72AFCBF
:1098A80009F1070960F307051FFA89F0FDF722FCA3
:1098B80060F30F25B0B205F08FF800221E4B05F0BB
:1098C800F1F805F0D1FB05F099F8CDE90001A8B24F
:1098D80005F082F812A3D3E9002304F02FFF12A3A6
:1098E800D3E9002305F008FA05F0BEFB05F086F879
:1098F8002246CDE90201114905A809F077FDC1B258
:1099080005A801F0F9FC0120FEF712FB0137BFB2F0
:10991800B8F80030BB428FD80DB0BDE8F08300BF67
:1099280000000000C0FFDF40E17A14AE47C1664086
:10993800583C0020904500200000F03E879C050818
:1099480008B50021C620FCF7D5FE4FF4957000211C
:10995800BDE80840FCF7CEBE024B4FF6FF721A80F6
:10996800704700BF9842002000200146C8224FF4EB
:10997800A073FBF734B807B50DF1070001F0BDFC83
:109988009DF807000EBD08B5FFF7F5FF0028FBD1CD
:1099980008BD30B5044687B010EE100A0D4605F034
:1099A8002DF802460B4601A8054909F01FFD20467F
:1099B800294601AA0023FBF77DFA07B030BD00BF96
:1099C8009A9C050808B5084802F020FB06480221C1
:1099D80002F0EDFB0028F9D0034802F043FB07EE44
:1099E800900AB8EE670A08BD0020014010B50C4C7B
:1099F80000232DED028B23809FED0A8A06E0FFF7F6
:109A0800E1FF238838EE008A013323802388182B4E
:109A1800F5D99FED050A28EE000ABDEC028B10BDB2
:109A2800C03B002000000000ACC8683910B54FF4F6
:109A3800C770FCF76DFEDB2805D14FF4C870FCF742
:109A480067FE84B219E041F2E104214644F20100C4
:109A5800FCF750FE44F20100FCF75AFEA04214BF86
:109A680080244FF4007421B24FF4C870FCF742FE12
:109A78004FF4C770DB21FCF73DFE204610BD024BBA
:109A880000221A80704700BFC0420020AFF3008058
:109A98007047FEE7FEE7FEE7FEE77047704770474E
:109AA800FEF73CBA10B5094CA37A4BB1084B1A68BB
:109AB80022F006021A6000F013F8204600F04FFE6C
:109AC8004FF48020BDE8104002F09ABD683C0020A9
:109AD80010ED00E0014801F011B800BF683C00201B
:109AE800364BD3F8882042F47002C3F88820344BF0
:109AF8001A6842F001021A6000229A60196821F07F
:109B0800847121F4803119602E495960196882B036
:109B180021F480211960DA60009201921A6842F4F7
:109B280080321A601A6802F400320192009A0132F7
:109B38000092019A1AB9009AB2F5A06FF2D1204B9F
:109B48001B6813F4003318BF01230193019B012BF9
:109B58002ED11B4B1A6C42F080521A641A4A1168B3
:109B680041F4804111609A689A609A6842F4004210
:109B78009A609A6842F4A0529A60144A5A601A6825
:109B880042F080721A6019680D4A8901FBD5104BA2
:109B980040F205611960936823F0030393609368AA
:109BA80043F002039360936803F00C03082BFAD187
:109BB800024B4FF000629A6002B0704700ED00E07F
:109BC800003802401030002400700040085440075C
:109BD800003C0240184B194A996801F00C0104290D
:109BE80003D0082903D0164B19E0164B17E0596823
:109BF8005A6811F4800F596814BF124B104B02F0C9
:109C08003F02B3FBF2F30C4A5268C2F30142C1F3BC
:109C18008811013252004B43B3FBF2F3074A136039
:109C2800054B9A68054BC2F303129A181968127902
:109C380021FA02F21A607047003802409C010020A5
:109C48000024F40000127A0037B51C2301240025F3
:109C580001A88DF804308DF805508DF806408DF870
:109C68000740FDF7A9FD2046214603F039FB0949C5
:109C78004CF24F334B6053230B800D814D804FF0D6
:109C8800804003F0D5FE4FF080402146224604F084
:109C980094FA3EBD0446002010B54FF080400121E3
:109CA80004F0A0FA00281DD001214FF080400E4C8E
:109CB80004F0A3FA00214FF0804003F04EFF237810
:109CC800022B07D0032B09D0012B0BD1BDE8104084
:109CD800F6F716BEBDE81040F6F7ECBDF7F732FA16
:109CE8000023237010BD00BFE00C002008B5402001
:109CF80002F078FC30B1FBF73BFA4020BDE80840A1
:109D080002F07EBC08BD0000014608B5044804F016
:109D180033FC0348402104F0DCFC0028F9D008BDDE
:109D280000440040F0B589B04FF4E13301200193BD
:109D380000232B4CADF808301E460146ADF80A301A
:109D4800ADF80C30ADF810300C23ADF80E3003F040
:109D5800A3FA4FF40030012103F0C2FA206802216F
:109D6800072202F071FF07226068032102F06CFFEE
:109D78000125022704232068059305A98DF81A6098
:109D88008DF81B508DF818708DF8197002F0DCFEF4
:109D980008236068059305A98DF8187002F0D4FEB1
:109DA800A06801A904F03EFB2A4640F225510D485F
:109DB80004F076FC262307A88DF81C308DF81D606A
:109DC8008DF81E608DF81F50FDF7F6FCA068294637
:109DD80004F0A5FB044A054B1A6009B0F0BD00BFAA
:109DE800B001002000440040119D0008704F002081
:109DF800024B9868002104F092BB00BFB00100201C
:109E080010B5094C40F22551204604F06CFC50B1C5
:109E1800A288D2B2112A02D1044B01211970044B35
:109E280019884A401A8010BD00440040D90C00200F
:109E3800B80D00207047704773B50120014603F044
:109E48002BFA264C4FF4D8530093022303268DF89F
:109E580004302046002369468DF806308DF8073017
:109E68008DF8056002F070FE204608210A2202F0F3
:109E7800EBFE204609210A2202F0E6FE20460B21CD
:109E88000A2202F0E1FE0A2220460C2102F0DCFE42
:109E980001254FF480632046694600938DF80650EB
:109EA8008DF807508DF8056002F04EFE0A210A462B
:109EB800204602F0C9FE29464FF4804003F01CFA00
:109EC8008020294603F0F4F94FF08050294603F02A
:109ED80043FA284602F094FB7CBD00BF0000024014
:109EE80007B54FF4C060FDF75DFC43238DF80430DF
:109EF8000322012301A88DF805308DF806208DF87E
:109F08000730FDF759FC0EBD782358430723B0FBF3
:109F1800F3F0002301338342FCD970474FF47A737E
:109F28005843F1E737B50023104C01930546032049
:109F3800FFF7EAFFEB681A69013C019213D0019A16
:109F4800002AF4DA019A42F001020192019A1A6198
:109F5800064A1969013A019102D00199C907F8D452
:109F68000320FFF7D1FF00203EBD00BF410D0300D5
:109F780010B5C47874B900EB820003339B10D0F895
:109F8800D000224603E051F8044C01320460043149
:109F98009A42F8D1002010BD033230B59210D0F8A3
:109FA800D0400B46002003E02568013043F8045CEC
:109FB80004339042F8D101EB800030BD0122F0B5A6
:109FC8000023827040220129C37082800CD10823AB
:109FD8000370042343704FF4A073C38002230372F9
:109FE800C1724FF0A04309E041B90C230370062366
:109FF80043704FF4A063C3801F4BC17203F5006226
:10A008000261C3604678044601461A46002508E006
:10A0180002F5106C02F530620A65C1F814C001350A
:10A028003A460431B54202F12007F1D303F58062C4
:10A03800426103F58862C0F8CC20067803F5A06574
:10A048000146002203E0C1F88C500132203504316A
:10A05800B242F8D31946002202E0C4F8CC1001320B
:10A068000434B24201F58051F7D303F56063C0F8B8
:10A078000C310020F0BD00BF0000044038B5037A61
:10A08800C2680025012B044625D1936B417A65F3FC
:10A09800104309B143F480139363D36823F4800316
:10A0A80023F0500343F010036FF3C3036FF3C71398
:10A0B8006FF351436FF3D343D3602046FFF732FF6A
:10A0C800E378012B3ED1052363F34405E36845F0AB
:10A0D80020059D6036E0D36843F04003D360FFF766
:10A0E80021FF237A627A032B14BF4FF434134FF401
:10A0F8003C130AB143F48013E26814209363FFF71A
:10A108000DFFE268217AD368032908BF43F480333E
:10A11800D360237A032B15D1156B012363F39B6559
:10A128006FF3D7552D2345F0805563F31645156316
:10A13800C820FFF7F3FEE36845F400051D63C82057
:10A14800FFF7ECFEE378012B07D1E3689D68052251
:10A1580062F3440545F020059D60002038BDC368C2
:10A168009A6842F001029A6000207047C3689A68B2
:10A1780022F001029A600020704707B5002301937E
:10A18800019B43F020030193019B61F38A13019320
:10A19800019BC2681361064B1169013B019102D012
:10A1A80001998806F8D40320FFF7AEFE00200EBD03
:10A1B800410D030007B500230193019B43F01003F1
:10A1C8000193019BC2681361064B1169013B019120
:10A1D80002D00199C906F8D40320FFF795FE0020A4
:10A1E8000EBD00BF410D030008B5C268D368012940
:10A1F8006FF35D736FF39E7302D143F0005302E077
:10A2080009B943F080433220D360FFF787FE00206E
:10A2180008BDC368586900F001007047C3685B69EE
:10A2280013F0010F14BF002001207047C36858695C
:10A2380000F001007047C3685A6998691040704778
:10A24800C3685868704703691A6861F301021A60A5
:10A258007047C268002393614FF0FF335361536026
:10A2680053610B4B9361C3789169002B14BF4FF472
:10A2780000634FF4016343F4701343F4405343F015
:10A28800080321EA03010B4393610020704700BFD4
:10A2980000080080F8B5D0F80C3100221A60036974
:10A2A80015461A6865F3CC221A60C37A012B044656
:10A2B8001BD10321FFF7C7FFE36880214FF4800219
:10A2C80061F30F0259629A62C02262F30F0561F3CB
:10A2D8001F454FF4A072C3F8045162F30F056FF3E2
:10A2E8001F45C3F80851C3F80C5110212046FFF749
:10A2F80044FF2046FFF75EFF226900234FF0FF313D
:10A308001361204653611E469161FF25D3612146A2
:10A3180010E082691768C7F3076707F08007FFB284
:10A32800002F14BF4FF090470027176001331661C4
:10A338000430956062789342EBD300231D46FF20DA
:10A3480010E04A6D1668C6F3076606F08006F6B296
:10A35800002E14BF4FF09046002616600133156199
:10A368000431906062789342EBD323691A6942F40E
:10A3780080721A61E278012A04D1054A402161F30A
:10A3880059421A632046FFF764FF0020F8BD00BF5A
:10A398000301010003699B68C3F34103013B022BDE
:10A3A8009ABF024AD05C0320704700BF4C9804084B
:10A3B80010B5036981699C680A68C4F341000228E2
:10A3C80002D06FF30A0202E0032060F30A020A6077
:10A3D8005A6842F480725A60002010BD30B54D783A
:10A3E8000B780022012D00EB830405D105FA03F355
:10A3F800A46963F30F0205E0012505FA03F3646D10
:10A4080063F31F422368C3F3072505F08005EDB207
:10A418006DB98D6865F30A03CD78C98865F39343F0
:10A4280061F3995343F0805343F400432360036975
:10A43800D9690A43DA61002030BD30B54D780B7810
:10A448000024012D224600EB830105D105FA03F310
:10A45800896963F30F0205E0012505FA03F3496DE5
:10A4680063F31F4203696FF3CF340C60D96921EAA3
:10A478000202DA61002030BDF8B54F780B78012F61
:10A4880000EB830349D19E694C69356833692A46D4
:10A4980064F3120314B967F3DC430BE08F68E41923
:10A4A800013CB4FBF7F7CC7867F3DC43012C08BF19
:10A4B80064F35E733361C378012B06D10B780C69A2
:10A4C80000EB83039B695C610CE0CB78012B09D01E
:10A4D8004B693BB103690C785E6B012707FA04F4FA
:10A4E80034435C63CB78012B07D103699B68DB0598
:10A4F80054BF45F0005245F080520B7800EB8303BF
:10A5080042F004429B691A60CB78012B38D10A7853
:10A518008B8AC968FFF72CFD32E05E6D4F6935689C
:10A528008C6833692A462FB964F31203012464F353
:10A53800DC430AE03F19013FB7FBF4F7BF05BF0D45
:10A5480067F3DC437C4364F312033361C378012B64
:10A5580005D10B780C6900EB83035B6D5C61CB78EC
:10A56800012B06D14B7913B145F0005201E045F0BB
:10A5780080520B7800EB830042F00442436D1A606E
:10A588000020F8BD73B54D78012D3DD183694A6926
:10A598001E681C690094E4B242B962F306048DF89F
:10A5A80000409DF8024065F3C4040EE08D68AA429D
:10A5B80086BF4D6165F3060462F306048DF800401A
:10A5C8009DF80240012262F3C4048DF80240009A0B
:10A5D8001A61C278012A05D10A780C6900EB820257
:10A5E8009269546146F004421A60C378002B34D152
:10A5F8004B69002B31D003690A78586B012101FAA5
:10A6080002F202435A6328E00B784E698C6800EB2B
:10A6180083035B6D1A681D690095EDB206B14C6144
:10A6280064F306059DF802408DF80050012565F396
:10A63800C4048DF80240009C1C61C378012B05D12D
:10A648000B780C6900EB83035B6D5C610B7800EBA6
:10A65800830042F00442436D1A6000207CBD4B78B1
:10A66800012B0B7800EB83000AD182691368C3F3CE
:10A67800076101F08001C9B221B143F0804301E0D4
:10A68800426D136843F400131360002070474B7841
:10A69800012B0B78C97800EB83000CBF8269426DEF
:10A6A80002391368C9B26FF35553012998BF43F0B3
:10A6B800805313600020704703699A69D869104075
:10A6C800000C704700EB810102694B6D9B68506973
:10A6D8001840704703699869DB69184080B2704771
:10A6E80082B000230093C0238DF803300122002399
:10A6F80062F3C4038DF8023018238DF80030009AF5
:10A70800436D1A61C278012A06D100F5B960586113
:10A718001A684FF080221A6002B07047D0F81431DE
:10A7280010B50446D3B103699A68D20716D5827A60
:10A7380042B1D0F80C21D0F80C116FF341026FF33D
:10A7480000020A605A6842F001025A600520FFF7C9
:10A75800E5FB23695A6822F001025A6010BD837A2A
:10A7680063B103699B68D90708D5D0F80C31D0F8D4
:10A778000C216FF341036FF300031360704701234B
:10A7880010B5002280F8123104460346FF2104E088
:10A7980058698160186D01328160607804338242A3
:10A7A800F6D3236900221A615A61DA614FF0FF3249
:10A7B8009A612046FFF7FEFC20461021BDE81040B4
:10A7C800DBE44B78012B0B7800EB83000FD1836916
:10A7D8001868C0F3074000F02003DBB2CBB900F0E3
:10A7E8000200C0B200280CBF302020207047436D03
:10A7F8001868C0F3074000F02003DBB25BB900F033
:10A808000200C0B200280CBF4FF440504FF4005073
:10A818007047102070474FF4805070474B78012BD9
:10A828000B7810B500EB83030AD19C69102A2368C2
:10A8380002D1BDE8104012E7202A0CD0302A0FE0E0
:10A848005C6DB2F5805F236802D143F400131BE00E
:10A85800B2F5005F02D143F0006315E0B2F5405F46
:10A868000FD1C3F3074202F02002D2B222B1002373
:10A878004B71BDE810400AE743F0806343F0802342
:10A8880002E00AB962F3CF33236010BDF8B504467D
:10A89800FFF794FB0122002384F8122184F8133176
:10A8A80028271646194640250CE007FB03F000F55B
:10A8B8008C7022182354D3805670D1709560D16063
:10A8C8005161013362789342EFD300232826194659
:10A8D80040250CE006FB03F000F55C7022182354B9
:10A8E800D3805170D1709560D16051610133627825
:10A8F8009342EFD32046FFF739FC2046FFF7BEFB13
:10A9080000212046FFF770FC2046FFF7C3FC2046D5
:10A91800BDE8F840FFF723BC70B5CDB20C464FF048
:10A92800280601F07F0106FB010115F0800F14BF16
:10A9380001F58C7101F55C7104F07F04ED090C7070
:10A948004D708A60CB7005B1CC80022B01D10023F9
:10A958000B71FFF743FD002070BD10B5CAB201F0BE
:10A968007F034FF0280404FB030312F0800F14BF89
:10A9780003F58C7303F55C7301F07F01D20919703C
:10A988005A701946FFF759FD002010BD38B501F07F
:10A998007F0528246C4304F55C7401194B6100237E
:10A9A8008B614B70EBB20355CA60C478012C08BFA9
:10A9B8000A6113B9FFF7E6FD01E0FFF75DFD00202E
:10A9C80038BD70B501F07F042825654305F58C7501
:10A9D80041190126E4B2CA600A6100224E7044554A
:10A9E8008A614B6114B9FFF7CDFD01E0FFF744FD23
:10A9F800002070BDCAB212F0800F10B54FF02803C6
:10AA080006D001F07F0403FB040303F58C7303E015
:10AA180003FB010303F55C73D209012401F07F01F4
:10AA280019709C705A701946FFF719FE002010BD66
:10AA3800CAB212F0800F10B54FF0280306D001F00B
:10AA48007F0403FB040303F58C7303E003FB01039A
:10AA580003F55C730024D20901F07F0119709C7022
:10AA68005A701946FFF713FE204610BD08B50B06AD
:10AA780004D501F07F01FFF780FB01E0FFF79AFBA7
:10AA8800002008BD0369002261F30A1219680A430D
:10AA98001A60704703695A6803206FF341025A60CD
:10AAA800FFF73CBA03695A68032042F002025A6071
:10AAB800FFF734BA11F0800F4FF0280306D001F0E9
:10AAC8007F0103FB010101F58C7103E003FB010128
:10AAD80001F55C71FFF775BE11F0800F4FF0280388
:10AAE80006D001F07F0103FB010101F58C7103E041
:10AAF80003FB010101F55C71FFF790BE2DE9F74FEB
:10AB08000446FFF78BFB002800F03F822046FFF742
:10AB180092FB0546002800F03882C0F3074000F099
:10AB28000800C0B2002861D02046FFF7C5FDA14645
:10AB3800824627464FF00008DFF86CB32E4650E0F7
:10AB48001AF0010F46D05FFA88F2114620460092AB
:10AB5800FFF7B8FD10F0010F0546009A20D07B6D75
:10AB680001259D60E178A94207D11B69D9F87813BE
:10AB7800C3F31203CB1AC9F88833DBF80030204638
:10AB88001B6811469847E378012B09D1B8F1000FEB
:10AB980006D194F81131052B02D12046FFF7A0FD0C
:10ABA80005F00203DBB213B17B6D02259D6005F051
:10ABB8000403DBB213B17B6D04259D6005F0080525
:10ABC800EDB23DB1DBF8003020469B6898477B6DBD
:10ABD8000820986008F101084FEA5A0A043709F179
:10ABE8002809BAF1000FABD135460120C5F3074358
:10ABF80003F00403DBB2002B00F0AF802046FFF720
:10AC080069FD264683464FF0000801959FE01BF03A
:10AC1800010F00F0978023695FFA88F919695D6B65
:10AC280004EB890225FA09F59269ED019268EDB203
:10AC38000D431540EA071CD55A6B012000FA08F1AC
:10AC480022EA01025A63B369974A98601368054675
:10AC58005B68204649469847E378AB4209D1B8F18A
:10AC6800000F06D194F81131042B02D12046FFF7CA
:10AC780037FD05F00403DBB213B1B36904259D6009
:10AC880005F00803DBB213B1B36908259D6005F030
:10AC98001003DBB213B1B36910259D6005F02003E2
:10ACA800DBB213B1B36920259D6005F04003DBB228
:10ACB80013B1B36940259D6005F00203DBB213B1FF
:10ACC800B36902259D6025F07F0515F0FF0F39D087
:10ACD800282505FB084505F58C75C246AB696A69E8
:10ACE800C3EB020CAB689C4528BF9C460CF1030CD7
:10ACF800B3694FEA9C0C9B696746A04614E0AA68B2
:10AD0800E9681C1B944228BF1446A3B240464A4631
:10AD1800FFF72EF9EB681B19EB60AB69E71C1C19F0
:10AD2800AC61B3699B69BF089BB2BB4205D9AC69EA
:10AD38006B699C4201D2002BE1D1B369802544465E
:10AD48009D60D04608F101084FEA5B0B0436BBF161
:10AD5800000F7FF45CAF019D012005F00203DBB218
:10AD680013B1E36802225A61C5F3076303F0800355
:10AD7800DBB2CBB1A37A43B1D4F80C31D4F80C21AF
:10AD88006FF341036FF30003136023695A6822F0DD
:10AD980001025A60444B1B6820469B699847E36848
:10ADA8004FF000425A610120C5F3072303F008035E
:10ADB800DBB2F3B13C4B1B6820465B6998472369BB
:10ADC800E2689B684FF400615161A27A82B1DB07A7
:10ADD8000ED5D4F80C311A6842F001021A601A68CC
:10ADE80042F003021A60314B1A6942F006021A61F6
:10ADF800012005F00803DBB243B12B4B1B6820464A
:10AE0800DB689847E36808225A61012005F01003BF
:10AE1800DBB2002B33D0E3689A6922F010029A6102
:10AE28001F6A282607F00F0306FB0346C7F34343B0
:10AE3800022B06F55C7602D0062B1AD10EE047F6F7
:10AE4800F0733B40ABB1C7F30A172046F1683A46A6
:10AE5800FFF7A2F8F368DB19F36007E004F5B961BE
:10AE680020460822FFF798F8C7F30A17B369DF19D5
:10AE7800B761E3689A6942F010029A610120C5F34C
:10AE8800072303F01003DBB2002B39D023695A687B
:10AE9800002622F001025A6031462046FFF76DF97C
:10AEA80023463246FF2108E04C02002000ED00E076
:10AEB80058698160186D013281606078043382427C
:10AEC800F6D3236901274FF0FF3267F30F069A6123
:10AED80067F31F460F22DE615A612F221A611A6832
:10AEE8006FF30A121A602046FFF7FAFBE3684FF483
:10AEF80080525A61264B1B6820461B699847384682
:10AF0800C5F3072303F02003DBB2EBB12046FFF7BC
:10AF18004FFAE3682046DE68FFF73CFA032806D1BB
:10AF28000023A3704FF40073A380092304E00123D6
:10AF3800A3704023A380052363F38D26E3684FF4B1
:10AF48000052DE6001205A61C5F3074303F0100385
:10AF5800DBB24BB10E4B1B682046DB699847E368B0
:10AF68004FF480125A610120C5F3074505F020050A
:10AF7800EDB255B1064B1B6820461B6A9847E3683B
:10AF88004FF400125A610120FFE7BDE8FE8F00BFB1
:10AF98004C02002043230B8000487047BC0100206E
:10AFA80038B51F4B1A68511C052A196035D1197913
:10AFB800002201291A6030D09968B1F5006F08BFE6
:10AFC8009A60174B9968DC68A1421A4602D10022A0
:10AFD8001A7122E086BFC1F500631361C1EB040456
:10AFE800D0F8EC3598BF14611569B3F839300C4CBA
:10AFF8009D428AB204D95918ED1AA160256104E06E
:10B008006918A1600021ABB22161054901240C71C6
:10B0180004498A188121FFF7D4FC002038BD00BFFD
:10B02800BC0D0020A346002038B528230A4D03FB99
:10B0380001010A4BB1F888131B6904462846984752
:10B04800D4F8EC352046B3F8403001212A46FFF702
:10B058009DFC002038BD00BF5B4600203802002060
:10B0680070B50B7813F0600506460C4625D0202DE8
:10B078001FD1CD88B5B113F0800F487808D0214B87
:10B0880021499B682A469847E2881F49304625E0AF
:10B098001E4B1D4958641E4B30465D612A4600F020
:10B0A80022FB1DE0174B48789B6829462A4698479B
:10B0B80025E000F077FB022521E04B780A2B11D020
:10B0C8000B2B14D0062B1AD14B881B0A212B03D12A
:10B0D800CA883A2A28BF3A220E49304600F0EAFACE
:10B0E80000250CE00C49012200F0E4FA07E08B7817
:10B0F8001BB9074A1D46936101E000F053FB28463F
:10B1080070BD00BF380200209B460020BC01002013
:10B11800BC0D0020CE010020D40D002010B58121E7
:10B128000446FFF71AFC01212046FFF716FC82218E
:10B138002046FFF712FC024B5B689847002010BDC1
:10B148003802002038B5D0F8EC350446B3F8392079
:10B1580081210223FFF7E0FBD4F8EC350121B3F895
:10B16800402020460223FFF7D7FB82210822032331
:10B178002046FFF7D1FB094B022200251A715D71A9
:10B18800074B1B689847D4F8EC35064AB3F84030AB
:10B1980020460121FFF7FAFB284638BD7C02002033
:10B1A800380200205B46002010B5074C606CFF2871
:10B1B80007D0064B064A9B68064952699847FF2301
:10B1C8006364002010BD00BFBC01002038020020CD
:10B1D800BC0D00209B46002038B510490B79012B87
:10B1E80019D10C690CB90C7115E0D0F8EC358D68E3
:10B1F800B3F839309C42AAB203D95D198D60E41ABC
:10B2080003E0A3B22C198C6000240C610449521885
:10B218008121FFF7D6FB002038BD00BFBC0D002000
:10B22800A346002000207047002070470023F0B597
:10B23800084A094E1D4609E01468C75C37550134B1
:10B248000133B4F5006F146008BF15608B42F3D169
:10B258000020F0BDC80D0020A3460020104B114A65
:10B26800D3F800C000232DE9F0410F4F16461D46C4
:10B278000DE0146810F8038007F804800134802C6E
:10B2880008BF2C4614603468644505D001338B42EE
:10B29800EFD10020BDE8F0810220BDE8F08100BFB9
:10B2A800244F0020384F0020A44E002021280FD121
:10B2B800084B1A680A701A68120A4A705A888A7003
:10B2C800DA78CA701A790A715A794A719B798B713E
:10B2D800002070473002002007B502AB012103F8B7
:10B2E800010D1846FFF7A2FF0EBD002100E0013155
:10B2F800435C002BFBD199E798E70B4B0B491A6885
:10B30800096891420BD00A498A5C02701A680132B6
:10B31800802A1A6005D100221A6001207047002097
:10B3280070470120704700BF244F0020384F00208D
:10B33800A44E0020204B1A68204B1B689A42F0B597
:10B3480009D135E00133802B08BF00239A4203D18D
:10B358001A4B1A602CE01A4CE15C0029F2D00A2939
:10B36800F0D00D29EED0154C1549134D23600E462B
:10B378000023CF182268BA5CC254226801339F1890
:10B38800802F08BF53422F689A18974210D0B25C9A
:10B398001AB10A2A01D00D2AEBD10022C254074A59
:10B3A800116859187F29116003D98039116000E0AC
:10B3B80000231846F0BD00BF384F0020244F00205E
:10B3C800A44E0020704700BFD0F8E43510B51B69C3
:10B3D80004469847032384F81231002010BD08B5AD
:10B3E800042380F81231D0F8E435DB689847002050
:10B3F80008BD08B5D0F8E035DB6903B198470020EF
:10B4080008BD08B5D0F8E0351B6A9847002008BD8C
:10B4180008B5D0F8E0355B6A9847002008BD0021E0
:10B4280010B5402204460B46FFF776FA80214022E9
:10B4380000232046FFF770FA012384F81231D4F86C
:10B44800E435A0785B689847002010BD13B56946BD
:10B45800044600F085F99DF8001001F01F03012B48
:10B4680007D0022B0AD073B92046694600F026FAA5
:10B478000FE02046694600F007FA0AE020466946D0
:10B4880000F0A2F905E021F07F01C9B22046FFF7DC
:10B49800B1FA00201CBD38B5044600293DD190F80A
:10B4A8001131022B42D1D0F83421D0F820319A4200
:10B4B80011D9C178D21A0129C0F8342104D1D0F8A1
:10B4C8002411CB18C0F8243192B22046D4F82411A4
:10B4D80000F000F92AE0D0F83821B2FBF3F503FBBD
:10B4E800152565B99A420AD3D0F83C319A4206D25A
:10B4F80029462A4600F0EEF8C4F83C5116E0D4F884
:10B50800E035DB682BB194F81221032A01D12046DB
:10B518009847204600F00FF908E0D0F8E0355B695D
:10B5280023B190F81221032A00D19847002038BD92
:10B5380010B5044659BB90F81131032B30D1D0F81F
:10B548008C23D0F878339A4214D9C178D21A0129B9
:10B55800C0F88C2304D1D0F87C13C918C0F87C1328
:10B568009A4228BF1A4692B22046D4F87C1300F0BB
:10B57800CAF815E0D0F8E0351B6923B190F812211C
:10B58800032A00D19847204600F0C6F808E0D0F812
:10B59800E0359B6923B190F81221032A00D198471E
:10B5A800002010BD2DE9F041069F04461646984636
:10B5B8000D46FEF741FC20462946C4F8E085C4F84C
:10B5C800E475C4F8E865FFF761F9D4F8E4351B6859
:10B5D80098472046BDE8F041FEF782BC002070473E
:10B5E800D0F8E03510B504461B689847D4F8E43520
:10B5F8009B689847002010BD08B5D0F8E0355B6817
:10B608009847002008BD000012230B8000487047AF
:10B618007C02002004230B80004870478E02002023
:10B6280010B5044C04480A46214600F075FA204635
:10B6380010BD00BF3C4F0020A29C05080A4608B573
:10B648000248034900F068FA014808BDB59C05089E
:10B658003C4F00200A4608B50248034900F05CFA4E
:10B66800014808BDC39C05083C4F002008B50A46A0
:10B6780008B9044800E00448044900F04DFA0348BA
:10B6880008BD00BFCE9C0508DB9C05083C4F002088
:10B6980008B50A4608B9044800E00448044900F01F
:10B6A8003BFA034808BD00BFE89C0508099D05084A
:10B6B8003C4F002010B513460C46C0F83821C0F89E
:10B6C8003421022280F8112100212246FFF779F95E
:10B6D800002010BD10B50C46134600212246FFF786
:10B6E80070F9002010BD10B513460C46C0F8902321
:10B6F800C0F88C23032280F8112100212246FFF78D
:10B7080045F9002010BD10B50C461346002122460D
:10B71800FFF73CF9002010BD0021042310B50A46AC
:10B72800044680F811310B46FFF74BF92046FEF727
:10B73800D7FF002010BD0021052310B50A46044696
:10B7480080F811310B46FFF721F92046FEF7C8FFB4
:10B75800002010BD282303FB0100B0F888037047C0
:10B7680090F8C8350B7090F8C9354B7090F8CB2518
:10B7780090F8CA3503EB02234B8090F8CD2590F85A
:10B78800CC3503EB02238B8090F8CF2590F8CE358B
:10B7980003EB02239BB2CB80C0F83C31012380F835
:10B7A8001131704710B591F90030002B044601DBC8
:10B7B800CB880BB9802100E00021FFF71BF9204658
:10B7C800BDE81040FEF78CBF38B50D4604466B78CF
:10B7D8000979012B10D027D3032B51D190F81231BE
:10B7E800022B28D0032B47D16B889BB991B18029B4
:10B7F80010D0FFF7FFF80DE090F81231022B1AD0A5
:10B80800032B39D16B88002B3AD149B1802907D055
:10B81800FFF70EF9D4F8E03520469B68294698478B
:10B828002046FFF779FF2BE090F81231022B02D067
:10B83800032B21D106E019B3802921D02046FFF738
:10B84800D9F81DE011F0800F4FF0280306D001F061
:10B858007F0103FB010393F81A2103E003FB0101B5
:10B8680091F87223074B02B101221A60204605495C
:10B878000222FFF71FFF03E020462946FFF792FF49
:10B88800002038BDD80D002038B590F81231032BB0
:10B8980004460D460CD10B79012B09D8D0F8E035B8
:10B8A8009B689847EB883BB92046FFF735FF03E0D4
:10B8B80020462946FFF776FF002038BD73B54B7840
:10B8C80004460D46092B00F21C81DFE813F0D10075
:10B8D80008011A01E4001A0172000A001A01C000E6
:10B8E80092004B881A0A013A062A00F20A81DFE818
:10B8F80012F007001A0027000801080108010801D2
:10B90800D4F8E835A0781B680DF106019847EB8854
:10B91800402B014603D094F81231012B3AD1082369
:10B92800ADF8063036E0D4F8E035A0789B6A0DF122
:10B9380006019847022343700146C4F8EC0529E044
:10B94800DBB2052B00F2DD80DFE803F003080D12FF
:10B95800171CD4F8E835A0785B6817E0D4F8E83508
:10B96800A0789B6812E0D4F8E835A078DB680DE091
:10B97800D4F8E835A0781B6908E0D4F8E835A07851
:10B988005B6903E0D4F8E835A0789B690DF10601FE
:10B9980098470146BDF80630002B00F0B680EA88CB
:10B9A800002A00F0B2809A4228BF1A46ADF8062055
:10B9B8005CE08B88002B40F0A480CB88002B40F003
:10B9C800A08094F812214B88032A00F09A8003F093
:10B9D8007F05204684F813512946FFF753F820467F
:10B9E800FFF79AFE0DB1022300E0012384F812311B
:10B9F8008BE08978464E0129317100F2828094F8F3
:10BA08001231022B02D0032B7BD108E0002962D02F
:10BA18000121032384F8101184F8123113E041B98D
:10BA2800022384F8123184F810112046FFF7E4FD50
:10BA380051E094F81011012920464DD0FFF7DCFDA4
:10BA4800317984F810112046FFF7CAFD43E0CA880F
:10BA5800012A56D194F81231022B02D0032B50D16F
:10BA680002E020462B4913E004F5887120460FE0D8
:10BA780094F81231023B012B43D8D4F814312449ED
:10BA8800002B0CBF0123032341F80C3F2046012261
:10BA9800FFF710FE39E04B88012B29D0022B34D157
:10BAA8008B8813F0FF0F30D121691B0A013B4A68CC
:10BAB800042B0FD8DFE803F0030507090B00012367
:10BAC80006E0022304E0032302E0042300E0052348
:10BAD80063F306124A602046FFF71EFE15E094F84D
:10BAE8001231023B012B0CD84B88012B0DD10023BE
:10BAF800C4F81431D4F8E03520469B6829469847A5
:10BB0800E9E720462946FFF74DFE00207CBD00BF2F
:10BB1800D80D0020E00D002030B5C8B10023DDB2FB
:10BB28000133C41814F8014C002CF8D16B1C5B00CD
:10BB380013800B7003234B70022305E0CA545A1C70
:10BB4800D2B202338C54DBB210F8012B002AF5D1A3
:10BB580030BD00BF704770477047704770477047E7
:10BB6800704700000EB403B070470A2810B50446A9
:10BB780002D10D20FFF7F9FF064A13681BB103F83D
:10BB8800014B136010BD044B1B680BB1204698474E
:10BB980010BD00BFE80D0020704F002010B504460E
:10BBA80001E0FFF7E2FF14F8010B0028F9D110BDFE
:10BBB8002DE9F04F044685B00D464FF00A0A00E023
:10BBC80035462078002800F0C480252801D00134AB
:10BBD80067E06078302803D1A0780123033407E0B8
:10BBE8002D2802D00234002302E0A0780223033477
:10BBF8004FF0000805E00AFB080814F8010BA8F14B
:10BC08003008A0F13002D2B2092AF4D96C2801D048
:10BC18004C2803D114F8010B43F00403002800F06A
:10BC28009880602886BFA0F12002D2B202464F2A2F
:10BC38003DD006D8432A2DD0442A09D0422A30D1F3
:10BC480033E0552A04D0582A29D0532A29D101E0B3
:10BC58000A272DE02E1D2F68002500E001357A5DAA
:10BC6800002AFBD104E02020FFF77FFF4D4601E0CA
:10BC7800980704D4454505F10109F4D34D463846E3
:10BC8800FFF78CFF03E02020FFF76FFF01354545E4
:10BC9800F9D395E728782E1DFFF767FF90E710275F
:10BCA80006E0FFF762FF2E468AE7022700E0082732
:10BCB8002E1D442A296804D1002902DA494243F09A
:10BCC8000803002200E02A46B1FBF7FE07FB1E111D
:10BCD800CDB2092D714607D9782814BF4FF0070C4B
:10BCE8004FF0270C6544EDB230350DF80250551C65
:10BCF800BEF1000F02D0102DE5D10F22190705D58E
:10BD080004A94D192D2105F8101C951C13F0010FDD
:10BD18000CBF4FF0200B4FF0300B9B072F4604D57C
:10BD280008E05846FFF721FF4F46474507F101094C
:10BD3800F7D34F46013D1DF80500FFF716FF002D0C
:10BD4800F8D103E02020FFF710FF01374745F9D36A
:10BD580036E705B0BDE8F08F70B5064D0C462E6885
:10BD6800286001E0FFF701FF14F8010B0028F9D162
:10BD78002E6070BD704F00200FB407B504A951F8AC
:10BD8800040B0191FFF714FFBDE80E4004B07047A3
:10BD98000EB417B505A9084C51F8043B20601846A5
:10BDA8000191FFF705FF2268002313702360BDE8A7
:10BDB8001E4003B0704700BFE80D00200EB433B535
:10BDC80005A9074C51F8043B2568206018460191E5
:10BDD800FFF7EEFE2560BDE83C4003B0704700BFAA
:10BDE800704F002070B51E4604461C481546FFF7E4
:10BDF800C3FF022E1FD0042E25D0012E2AD105E024
:10BE0800A15D1748FFF7B8FF013600E00026AE42F3
:10BE1800F6DB2020FFF7A9FE002609E0A05DA0F1CF
:10BE28002003DBB25E2B88BF2E20FFF79EFE013673
:10BE3800AE42F3DB0EE034F8021B0A48FFF79CFF22
:10BE4800013DF8D106E054F8041B0748FFF794FFBA
:10BE5800013DF8D10A20BDE8704086E62A9D050814
:10BE6800319D0508379D05083D9D050808B5012148
:10BE78004FF4807001F07CFA4FF480700021BDE827
:10BE8800084001F075BA43680A6823F0407323F448
:10BE9800807313430A7943EA02234360CA680B6933
:10BEA80030B51A4384688D68084B2A4323401343EE
:10BEB8004A7943EA420383600B7DC26A013B22F45C
:10BEC8007002DBB242EA0353C36230BDFDF7FFC024
:10BED80000230360037143718360C360036101231E
:10BEE80003757047074A084B516810B50B4090E836
:10BEF800120021438468C068214301430B43536007
:10BF080010BD00BF00230140E030FCFF00230360A8
:10BF180043608360C3607047836811B143F00103D5
:10BF280001E023F0010383607047436823F4400372
:10BF380023F400730B434360704741628262704789
:10BF4800436823F01F030B4343607047044B5A6850
:10BF580010B142F4000201E022F400025A60704776
:10BF680000230140044B5A6810B142F4800201E0FA
:10BF780022F480025A60704700230140092970B5F5
:10BF88000CB20CD904EB44041E3CC6680725A54036
:10BF980026EA0505A34045EA0304C4600AE00669E9
:10BFA80004EB44040725A54026EA050513FA04F422
:10BFB8002C430461062A0CD80523013A5A43446BE2
:10BFC8001F23934024EA0303914043EA010242639A
:10BFD80070BD0C2A12B20CD802EB8202233A046B11
:10BFE8001F23934024EA0303914043EA01020263BA
:10BFF80070BD02EB8202413AC46A1F23934024EACF
:10C008000303914043EA0102C26270BD836843F0B2
:10C018008043836070478068C0F3805070478368AE
:10C0280011B143F4806301E023F4806383607047B7
:10C03800836811B143F0020301E023F00203836037
:10C0480070474368013923F4604343EA413343604E
:10C058007047436811B143F4006301E023F40063BF
:10C0680043607047C06C80B27047014B18687047D6
:10C0780008230140836811B143F4807301E023F47D
:10C08800807383607047836811B143F4007301E0E3
:10C0980023F4007383607047044B5A6810B142F46C
:10C0A800005201E022F400525A6070470023014018
:10C0B800092970B50CB20CD904EB44041E3CC668BF
:10C0C8000725A54026EA0505A34045EA0304C46000
:10C0D8000AE0066904EB44040725A54026EA05059D
:10C0E80013FA04F42C430461836BC3F30154121B49
:10C0F8000232D2B202EB82021F24944023EA0403E4
:10C1080091400B43836370BD836B013923F4401363
:10C1180043EA01538363704782B00023019301907F
:10C12800019BCB180193019B1A6002B0704783688A
:10C1380023F470230B4383607047836823F4401310
:10C148000B4383607047836843F4800383607047C0
:10C158008068C0F380507047436811B143F480632E
:10C1680001E023F4806343607047436811B143F4EE
:10C17800805301E023F480534360704782B000236A
:10C1880001930190019B28335B180193019B186868
:10C1980080B202B070470123C9B213FA01F14368B3
:10C1A8000AB1194301E023EA0101416070470368BD
:10C1B80019420CBF002001207047C9430160704735
:10C1C8004368006810EA112007D00122C9B212FAA8
:10C1D80001F119420CBF0020012070476FEA1121BC
:10C1E80001607047036823F00103036000230360C4
:10C1F80043608360C3600361212343612C4B9842F1
:10C208001CD02C4B984220D02B4B984225D02B4B3E
:10C2180098422AD02A4B98422FD02A4B984233D0A2
:10C22800294B984237D0294B984204D14FF03D52C0
:10C2380043F8AC2C7047264B984203D13D2243F873
:10C24800082C7047234B984204D14FF4746243F88A
:10C25800202C7047204B984204D14FF4741243F8B5
:10C26800382C70471D4B984204D14FF0746243F844
:10C27800502C70471A4B984203D11A4A43F8642C41
:10C288007047194B984203D1184A43F87C2C7047E1
:10C29800174B984203D1174A43F8942C7047164B12
:10C2A800984204BF4FF03D5243F8AC2C704700BF92
:10C2B800106002402860024040600240586002401E
:10C2C8007060024088600240A0600240B86002408E
:10C2D80010640240286402404064024058640240EE
:10C2E800706402403D00002088640240400F002036
:10C2F800A064024000003D20B86402400268134B6D
:10C3080010B51340CC680A6822434C6922438C69F3
:10C318002243CC6922430C6A22434C6A22438C6A2A
:10C3280022434C6B22438C6B2243134303604269C4
:10C338000C6BCB6A22F007022343134343610B695A
:10C3480043604B6883608B68C36010BD3F801CF0FE
:10C358000023036043608360C360036143618361BA
:10C36800C361036243628362C3620363436383639B
:10C378007047036811B143F0010301E023F00103A2
:10C3880003607047036811B143F4004301E023F4EC
:10C39800004303607047036811B143F0200301E0D4
:10C3A80023F020030360704741607047406880B203
:10C3B8007047036812B143F4002301E023F400231B
:10C3C800036001617047036811B143F4802301E001
:10C3D80023F48023036070470AB101617047C1608C
:10C3E80070470068C0F3C0407047006800F0010063
:10C3F8007047406900F0380070470A4A0A4B10B588
:10C408000A4CA04288BF13468A004CBF5B681B6871
:10C4180021F0F02121F0821119420CBF00200120E7
:10C4280010BD00BF00640240006002400F6402407B
:10C4380010B5084B084A094CA04288BF134611F0B2
:10C44800005F21F0F02121F0821114BFD9609960BA
:10C4580010BD00BF00600240006402400F6402404B
:10C468000B0607D5436912B143F0800301E023F0BE
:10C4780080034361802909D001F01E01036812B1CD
:10C4880019430160704723EA010101607047124BAC
:10C49800124A10B5124CA0428CBF14461C4621F01B
:10C4A800F02323F0C3132BB1026802F01E0202EA44
:10C4B800D12202E0426902F0800288004CBF636822
:10C4C800236821F0F02121F08210184002D0101CBE
:10C4D80018BF012010BD00BF006002400064024088
:10C4E8000F64024010B5084B084A094CA04288BFA7
:10C4F800134611F0005F21F0F02121F0821114BFE2
:10C50800D960996010BD00BF00600240006402401D
:10C518000F640240044B00221A605A609A60DA6085
:10C52800024A5A61704700BF003C0140FFFF7F008C
:10C53800837910B5002B29D01A4B01681C68CA43AF
:10C5480014401C605C6822405A60027902F1804203
:10C5580002F59E3214682143116002689C68D14339
:10C568000C409C60DC682140D9604179102906D1D3
:10C57800996811439960D9680A43DA6010BD01F1DE
:10C58800804303F59E3319680A4308E0037901687C
:10C5980003F1804303F59E331A6822EA01021A6008
:10C5A80010BD00BF003C014000230C220360037152
:10C5B800427183717047024B1A6902431A617047CE
:10C5C800003C0140034B5B6918420CBF002001206E
:10C5D800704700BF003C0140014B5861704700BFE5
:10C5E800003C0140054B1A685B69034004D01042C7
:10C5F8000CBF00200120704718467047003C0140DE
:10C60800014B5861704700BF003C01404FF0204388
:10C6180018B943F2DB021A6003E043F2D20243F88E
:10C6280020204FF02042411C6FF0704342F8213027
:10C6380002F5827242F82030704770B58468456808
:10C64800C368C16A026825431D4303691D434369E2
:10C658001D4383691D43C3691D43036A1D43436A20
:10C668001D43836A1D43036B0D431D434FF0204355
:10C67800082C43F8225005D153F8224044F04004D6
:10C6880043F82240436B9E691D6835435E6845EA5E
:10C6980006159E6845EA0625DE6845EA06451E69D0
:10C6A8005B6945EA0655541C45EA03654FF020438B
:10C6B800B1F5804F43F8245010D1836B98691968FD
:10C6C8000143586841EA0011986841EA0021186955
:10C6D8005B6941EA005141EA036101E06FF0704192
:10C6E800014B43F8221070BD040100A002224260F1
:10C6F8004FF480524262416B4FF4005210B582628F
:10C7080000230F22FF2403608360C3600361436139
:10C718008361C3610362C36203630A604A608C6019
:10C72800CA600A614A618B61816B0A604A608C60E9
:10C73800CA600A614A618B6110BD4FF0204321B184
:10C7480053F8202042F0010203E053F82010024A77
:10C758000A4043F820207047FEFF0F0010280CBF46
:10C76800064B074B4FF040024FF0180119605A6012
:10C778004FF0FC329A60DA60704700BF600000A09A
:10C78800800000A030B5836844681C43C36844F047
:10C7980008041C4303691C43436944EA432483692E
:10C7A80044EA4334C36999685A68090441EA022192
:10C7B8001A68DB68114341EA0361036A9A685D6895
:10C7C800120442EA05221D68DB682A4342EA036232
:10C7D8000368102B0CBF034B034B1C609960DA6095
:10C7E80030BD00BF600000A0800000A010230360DF
:10C7F800C269002343608360C3600361436183614E
:10C80800FC23136053609360D360026A1360536023
:10C818009360D360704741B110280CBF074B084B99
:10C828001A6842F004021A60704710280CBF034AC5
:10C83800034A044B11680B4013607047600000A066
:10C84800800000A0FBFF0F0041B110280CBF084B6F
:10C85800084B1A6842F040021A60704710280CBF53
:10C86800034A044A044B11680B401360704700BF29
:10C87800600000A0800000A0BFFF0F00102802D1B8
:10C88800024B58697047024B58697047600000A016
:10C89800800000A0054B18221A6000225A604FF051
:10C8A800FC329A60DA601A61704700BFA00000A0ED
:10C8B8000268436842F0100242EA4322836842EA6F
:10C8C8004332144B10B51A60C26891685468090461
:10C8D80041EA04211468D268214341EA02629A605D
:10C8E800026991685468090441EA04211468D2680D
:10C8F800214341EA0262DA6042699168506809049A
:10C9080041EA00211068D268014341EA02621A61D3
:10C9180010BD00BFA00000A0C268002303604360F0
:10C928008360FC23136053609360D36002691360D3
:10C9380053609360D3604269136053609360D3601F
:10C948007047054B18B11A6842F0040202E01968F2
:10C95800024A0A401A607047A00000A0FBFF0F00BF
:10C9680062B1102801D10E4B03E0B0F5807F03D1EE
:10C978000C4B5A68114311E00B4BFAE7102804D10D
:10C98800074B5A6822EA010108E0B0F5807F0CBF26
:10C99800044B054B5A686FEA010111405960704712
:10C9A800600000A0800000A0A00000A0102801D115
:10C9B800064B04E0B0F5807F0CBF054B054B5B6868
:10C9C8000B420CBF00200120704700BF600000A090
:10C9D800800000A0A00000A0102804D1074B5A68CE
:10C9E80022EA010108E0B0F5807F0CBF044B054B3B
:10C9F8005A686FEA0101114059607047600000A051
:10CA0800800000A0A00000A0102801D1084B04E07D
:10CA1800B0F5807F0CBF074B074B5B6813EA01003A
:10CA280004D013EAD1010CBF00200120704700BFD9
:10CA3800600000A0800000A0A00000A0102804D181
:10CA4800084B5A6822EAD10109E0B0F5807F0CBF93
:10CA5800054B064B5A684FEAD10122EA0101596099
:10CA6800704700BF600000A0800000A0A00000A0E8
:10CA780008B52C4B984205D10120014600F048FC2E
:10CA8800012048E0284B984205D10220012100F0FE
:10CA98003FFC02203FE0254B984205D104200121AC
:10CAA80000F036FC042036E0214B984205D10820DE
:10CAB800012100F02DFC08202DE01E4B984205D1E5
:10CAC8001020012100F024FC102024E01A4B984289
:10CAD80005D12020012100F01BFC20201BE0174B72
:10CAE800984205D14020012100F012FC402012E0BC
:10CAF800134B984205D18020012100F009FC8020C9
:10CB080009E0104B98420BD14FF48070012100F0DE
:10CB1800FFFB4FF480700021BDE8084000F0F8BB2F
:10CB280008BD00BF000002400004024000080240A7
:10CB3800000C02400010024000140240001802409D
:10CB4800001C0240002002402DE9F0470023D1F8E4
:10CB580000801A464FF0010C03270CFA02F404EA8D
:10CB68000805A5422ED1066817FA03F4E4432640C7
:10CB780006600E79D0F8009006FA03FA013E4AEAF8
:10CB88000909012EC0F8009014D8866891F805901C
:10CB980026408660866809FA03F949EA060686602F
:10CBA800466826EA050545608D7946689540ADB228
:10CBB80035434560C5682C40C460CC79C5689C4045
:10CBC8002C43C46001320233102AC6D1BDE8F08775
:10CBD8004FF6FF7303600023037143718371C371C0
:10CBE800704782B04FF480330193019B0B4301934C
:10CBF800019BC361C161019BC361C3690193C3699F
:10CC0800019302B07047036919420CBF002001204C
:10CC18007047006980B27047436919420CBF002011
:10CC280001207047406980B2704701837047418393
:10CC380070470AB10183704741837047416170476B
:10CC480043694B404361704701F00703C908083145
:10CC580030B59B0050F821500F249C4025EA04046D
:10CC680040F8214050F8214012FA03F31C4340F8E1
:10CC7800214030BD08B5134B984207D14FF400103E
:10CC8800012100F069FB4FF4001014E00E4B9842AC
:10CC980007D14FF48000012100F05EFB4FF48000C3
:10CCA80009E00A4B98420BD14FF40000012100F033
:10CCB80053FB4FF400000021BDE8084000F04CBBD6
:10CCC80008BD00BF0054004000580040005C004010
:10CCD8007FB50446868868460D4600F06DFA0299CD
:10CCE8002C482B6826F03F063604B1FBF0F0360CD2
:10CCF80080B20643A680228822F001021204120C98
:10CD08002280254A93420AD85B00B1FBF3F3013035
:10CD18009BB280B22084032B98BF042321E0EE88C5
:10CD28004BF6FF72964205D103225343B1FBF3F34E
:10CD38009BB206E019225343B1FBF3F39BB243F4D1
:10CD480080431A054FF4967208BF43F0010350431D
:10CD58004FF47A7290FBF2F0013080B243F4004352
:10CD68002084A38323886989AA889BB243F001039E
:10CD78002380238823F4816323F002031B040A43DE
:10CD88001B0C13439BB223802A89AB8913439BB2A4
:10CD980023817FBD40420F00A086010041F2883305
:10CDA8000360002383804BF6FF72038143814FF4B5
:10CDB8008043C28083817047038819B19BB243F0D6
:10CDC800010303E023F001031B041B0C03807047DD
:10CDD800038819B19BB243F4807303E023F4807392
:10CDE8001B041B0C03807047038819B19BB243F4E2
:10CDF800007303E023F400731B041B0C03807047CB
:10CE080012B141F0010101E001F0FE010182704719
:10CE1800038819B19BB243F4806303E023F4806371
:10CE28001B041B0C0380704783899BB201F0FE0131
:10CE380023F0FE030B4383817047838919B19BB2AA
:10CE480043F0010303E023F001031B041B0C83815F
:10CE58007047038819B19BB243F0400303E023F005
:10CE680040031B041B0C03807047038829B16FEA39
:10CE780043436FEA53439BB201E05B045B0C0380BE
:10CE88007047038819B99BB243F0800303E023F08D
:10CE980080031B041B0C03807047B1F5804F838B04
:10CEA80004D023F480431B041B0C02E09BB243F420
:10CEB800804383837047B1F5006F038803D19BB229
:10CEC80043F4006303E023F400631B041B0C03809A
:10CED8007047B1F5005F038803D19BB243F4005358
:10CEE80003E023F400531B041B0C038070470388E2
:10CEF80019B19BB243F0100303E023F010031B04A5
:10CF08001B0C0380704701827047008AC0B27047CB
:10CF1800038819B19BB243F4805303E023F4805390
:10CF28001B041B0C03807047B1F5006F038803D105
:10CF38009BB243F4006303E023F400631B041B0C5F
:10CF480003807047038819B19BB243F0200303E0C4
:10CF580023F020031B041B0C03807047008BC0F3D5
:10CF680007207047838819B19BB243F4006303E03C
:10CF780023F400631B041B0C83807047838819B15A
:10CF88009BB243F4805303E023F480531B041B0C2F
:10CF98008380704782B0002301930190019BCB18D6
:10CFA8000193019B188880B202B0704783889BB2B6
:10CFB8000AB1194301E023EA010181807047838A9D
:10CFC800008B9BB243EA0040084020F07F40431AA0
:10CFD800584240EB03007047838A008B9BB243EAB8
:10CFE800004020F07F40704782B0002300930193F7
:10CFF8000B0F01900093009B21F07F4113B1019B1F
:10D00800143302E0019B090C18330193019B1B6840
:10D0180019420CBF0020012002B07047C94389B2F1
:10D02800818270478388808A80B208409BB206D08C
:10D0380001F0E06113EA11410CBF002001207047A4
:10D04800C94389B2818270470A4B1A6842F00102CB
:10D058001A6000229A60196821F0847121F48031E5
:10D06800196005495960196821F480211960DA604E
:10D07800704700BF0038024010300024024B0022E5
:10D088001A701870704700BF02380240034B1A68C4
:10D0980022F0F80242EAC0021A60704700380240E3
:10D0A800014B1860704700BF00004742064B002242
:10D0B80001281A701A7002D0042804D101E01870EF
:10D0C800704705221A70704770380240014B18608B
:10D0D800704700BF800E4742014341EA821200991F
:10D0E8005B08013B42EA016141EA0341014B596097
:10D0F800704700BF00380240014B1860704700BFFE
:10D10800600047428001034B40EA0171C3F8841074
:10D11800704700BF00380240014B1860704700BFDD
:10D1280068004742014B1860704700BF4C004742F7
:10D13800034B9A6822F0EC6202430A439A607047F4
:10D1480000380240034B9A6822F0784202430A43AF
:10D158009A60704700380240034B9A6822F0030235
:10D1680002439A60704700BF00380240024B98683B
:10D1780000F00C00704700BF00380240034B9A686B
:10D1880022F0F00202439A60704700BF0038024064
:10D19800034B9A6822F4E05202439A60704700BF3A
:10D1A80000380240034B9A6822F4604242EAC00207
:10D1B8009A607047003802401E4B9A6802F00C02D1
:10D1C800042A10B503D0082A03D01B4B18E01B4BC8
:10D1D80016E059685A6811F4800F596814BF174B44
:10D1E800154B02F03F02B3FBF2F3124A5268C2F346
:10D1F8000142C1F3881101324B435200B3FBF2F3F1
:10D208000C4903608B680E4A0468C3F30313D35CAC
:10D2180034FA03F343608C68C4F38224145D33FA50
:10D2280004F484608968C1F34231525CD340C3601E
:10D2380010BD00BF003802400024F40000127A003C
:10D24800D402002000F44073B3F5407F084B08D1A6
:10D25800996820F0704221F4F81122F440720A43D0
:10D268009A601A6F000542EA10501867704700BFAD
:10D2780000380240014B1860704700BF3C0E47421F
:10D28800014B1860704700BF400E4742014B1860C1
:10D29800704700BF5C014742044B1A6B09B1104349
:10D2A80001E022EA00001863704700BF003802401E
:10D2B800044B5A6B09B1104301E022EA000058639D
:10D2C800704700BF00380240044B9A6B09B1104305
:10D2D80001E022EA00009863704700BF003802406E
:10D2E800044B1A6C09B1104301E022EA00001864EB
:10D2F800704700BF00380240044B5A6C09B1104314
:10D3080001E022EA00005864704700BF003802407C
:10D31800044B1A6909B1104301E022EA00001861C0
:10D32800704700BF00380240044B5A6909B11043E6
:10D3380001E022EA00005861704700BF003802404F
:10D34800044B9A6909B1104301E022EA0000986190
:10D35800704700BF00380240044B1A6A09B11043F5
:10D3680001E022EA00001862704700BF003802405E
:10D37800044B5A6A09B1104301E022EA00005862DE
:10D38800704700BF00380240044B1A6D09B11043C2
:10D3980001E022EA00001865704700BF003802402B
:10D3A800044B5A6D09B1104301E022EA00005865A8
:10D3B800704700BF00380240044B9A6D09B1104312
:10D3C80001E022EA00009865704700BF003802407B
:10D3D800044B1A6E09B1104301E022EA00001866F6
:10D3E800704700BF00380240044B5A6E09B1104321
:10D3F80001E022EA00005866704700BF003802408A
:10D40800044B1A7809B1104301E022EA00001870B1
:10D41800704700BF0D3802404309012B074A01D16C
:10D42800136803E0022B0CBF136F536F00F01F004B
:10D4380033FA00F000F00100704700BF00380240E6
:10D4480007B5002301933120FFF7E6FF019B013365
:10D458000193019BB3F5A06F01D00028F3D03120D0
:10D46800FFF7DAFF003018BF01200EBD024B5A6FDC
:10D4780042F080725A67704700380240034BDB68FD
:10D4880018420CBF00200120704700BF003802403E
:10D49800014B1870704700BF0E38024008B5154B95
:10D4A80098420BD101214FF48050FFF761FF4FF4F0
:10D4B80080500021BDE80840FFF75ABF0E4B984244
:10D4C80007D14FF480400121FFF746FF4FF4804019
:10D4D80009E00A4B98420BD14FF400400121FFF7B5
:10D4E8003BFF4FF400400021BDE80840FFF734BF80
:10D4F80008BD00BF0030014000380040003C00403B
:10D508000B88028810B54C8823438C882343CC8829
:10D5180023430C8923434C8923438C892343CC8997
:10D5280002F44152234313439BB20380838B23F4B9
:10D5380000631B041B0C83830B8A038210BD838B3F
:10D5480023F47B6323F00F031B041B0C8383022348
:10D5580003848B68F0B5858B022BADB238D0294A8D
:10D568008E889468002E14BF02260126240203D553
:10D57800946824F400049460D2F88440D2F884704B
:10D588005268DFF884C002F03F02BCFBF2F2C4F339
:10D5980088145443C7F30272B4FBF2F4CA88B2F594
:10D5A800007F4FF00A0201D1240A02E07601B4FBA1
:10D5B800F6F46243B2FBF3F305330A229BB2B3FBE2
:10D5C800F2F303F001021202C3F34F0392B200E038
:10D5D80000229C1EA4B2FE2C28BF0022CC8828BFA3
:10D5E8000223134323439BB203840B884A882B43AB
:10D5F80043F4006313438A8813438A8913439BB215
:10D608008383F0BD0038024000127A0000230380B3
:10D6180043808380C380038143818381C38107233F
:10D628000382704700230222038043808380C380E3
:10D63800826083817047038819B19BB243F040032D
:10D6480003E023F040031B041B0C03807047838B0B
:10D6580019B19BB243F4806303E023F480631B0495
:10D668001B0C83837047038823F400631B041B0C83
:10D67800038003889BB20B4303807047B1F5804F4A
:10D68800038803D19BB243F4804303E023F480432F
:10D698001B041B0C038070474FF6FF6399420388F5
:10D6A80003D09BB243F4807303E023F480731B041C
:10D6B8001B0C03807047838819B19BB243F00403A5
:10D6C80003E023F004031B041B0C8380704783884A
:10D6D80019B19BB243F0100303E023F010031B04BD
:10D6E8001B0C83807047838B23F47B6323F00F0329
:10D6F8001B041B0C8383022303840B88828BB3F5E2
:10D70800007F10B592B205D0002B0CBF4FF4807388
:10D71800002301E04FF480734C8822438C88898968
:10D7280042F4006222430A4392B21343838310BD3A
:10D73800808980B2704781817047038819B19BB294
:10D7480043F4005303E023F400531B041B0C038031
:10D75800704703889BB243F48053038070470129C4
:10D7680002D0008B80B27047808A80B27047008AEE
:10D7780080B2704783889BB20AB1194301E023EA5B
:10D78800010181807047090901238B409BB21AB1BE
:10D79800828892B2134303E0828892B222EA03039A
:10D7A80083807047038919420CBF0020012070470D
:10D7B800C94389B20181704710B584880089012363
:10D7C80001F00F0280B213FA02F21040A4B205D0A1
:10D7D80009098B401C420CBF0020012010BD01F03C
:10D7E8000F0101238B40DB439BB20381704700BFCD
:10D7F80008B501214FF48040FFF7BAFD4FF480408F
:10D808000021BDE80840FFF7B3BD014B1860704721
:10D818000038014001F0030289080A4B023130B593
:10D82800920053F821500F24944025EA040443F849
:10D83800214053F8214010FA02F2144343F82140E2
:10D8480030BD00BF00380140014B1860704700BF71
:10D85800DC002742014B1860704700BF00042742D4
:10D86800024B186AC0F30020704700BF003801401F
:10D8780030B5048C24F001042404240C0484058BA2
:10D88800048CADB2A4B225F0F305154324F00A04C4
:10D8980045EA031544F00104ADB20C430583048442
:10D8A80030BD30B5048C24F010042404240C048406
:10D8B800048B058C24F44074ADB22405240D25F0A6
:10D8C800A00544EA022445F0100544EA033445EA79
:10D8D8000115A4B2ADB20483058430BD08B5474B29
:10D8E800984205D101200146FFF742FD01203DE0A5
:10D8F800B0F1804F05D101200146FFF72DFD012031
:10D9080076E03F4B984205D102200121FFF724FD24
:10D9180002206DE03B4B984205D104200121FFF71E
:10D928001BFD042064E0384B984205D108200121F2
:10D93800FFF712FD08205BE0344B984205D1102018
:10D948000121FFF709FD102052E0314B984205D123
:10D9580020200121FFF700FD202049E02D4B9842AF
:10D9680009D102200121FFF703FD02200021BDE8B3
:10D978000840FFF7FDBC284B984207D14FF4803090
:10D988000121FFF7F5FC4FF48030EFE7234B984275
:10D9980007D14FF400300121FFF7EAFC4FF40030C3
:10D9A800E4E71F4B984207D14FF480200121FFF78D
:10D9B800DFFC4FF48020D9E71A4B984205D140206C
:10D9C8000121FFF7C9FC402012E0174B984205D10E
:10D9D80080200121FFF7C0FC802009E0134B98420A
:10D9E8000BD14FF480700121FFF7B6FC4FF4807023
:10D9F8000021BDE80840FFF7AFBC08BD00000140AA
:10DA08000004004000080040000C004000100040E6
:10DA1800001400400004014000400140004401405F
:10DA28000048014000180040001C00400020004051
:10DA38001C4A038890429BB212D002F58062904241
:10DA48000ED0B0F1804F0BD0A2F58032904207D0B3
:10DA580002F58062904203D002F58062904203D1C1
:10DA68004A8823F0700313430F4A904208D002F506
:10DA78008062904204D023F440730A899BB2134316
:10DA880003804B68C3620B880385064B984203D01A
:10DA980003F58063984201D18B7A03860123838240
:10DAA800704700BF00000140001000404FF0FF33F6
:10DAB800436000230380038143808372704701859C
:10DAC80082827047038823F070031B041B0C0B43EE
:10DAD8000380704741627047C1627047406A70476F
:10DAE800008D80B27047038819B19BB243F00203DE
:10DAF80003E023F002031B041B0C03807047038818
:10DB080019B19BB243F0040303E023F004031B04A0
:10DB18001B0C03807047038819B19BB243F0800344
:10DB280003E023F080031B041B0C03807047038869
:10DB380023F008031B041B0C038003889BB20B43D0
:10DB480003807047038823F440731B041B0C038075
:10DB580003889BB20B4303807047038819B19BB2BB
:10DB680043F0010303E023F001031B041B0C0380B3
:10DB78007047038C23F001031B041B0C038470B54E
:10DB8800038C8488028B0D884E8822F0730212045D
:10DB9800120C2A438D8923F002031B0435431B0C06
:10DBA800ADB22B430E4DA842A4B203D005F5806553
:10DBB800A8420ED1CD894E8A23F008032B438D88C5
:10DBC80023F004032B430D8A354324F44074ADB28B
:10DBD8002C43848002838A684263038470BD00BF3B
:10DBE80000000140038C23F010031B041B0C03846A
:10DBF800038C828830B5048B0D8824F4E644240411
:10DC0800240C23F0200344EA05241B048D891B0CF3
:10DC180043EA05134D8843EA0513134DA84292B20F
:10DC2800A4B29BB203D005F58065A84215D1CD8971
:10DC380023F080039BB243EA05134FF6BF751D40DE
:10DC48008B8845EA03130D8A22F4406242EA850272
:10DC58004D8A42EA85029BB292B282808A68048326
:10DC68008263038430BD00BF00000140038C23F4AD
:10DC780080731B041B0C0384038C828830B5848B4F
:10DC88000D8824F073042404240C23F400731B046B
:10DC98002C438D891B0C43EA05234D8843EA052351
:10DCA800124DA84292B29BB203D005F58065A842F6
:10DCB80015D1CD8923F400639BB243EA05234FF6BF
:10DCC800FF351D408B8845EA03230D8A22F4405214
:10DCD80042EA05124D8A42EA05129BB292B282804C
:10DCE8008A688483C263038430BD00BF000001409A
:10DCF800038C23F480531B041B0C0384038C30B562
:10DD08008488828B0D8822F4E6421204120C23F4D4
:10DD1800005342EA05221B048D891B0C43EA053394
:10DD28004D8843EA05330B4DA842A4B292B29BB288
:10DD380003D005F58065A84205D10D8A24F48044F6
:10DD480044EA8514A4B2848082838A6802640384C6
:10DD580030BD00BF00000140002303804380838062
:10DD680083608381C38103824382704730B5058C09
:10DD78000124ADB28C4025EA040400F118030484A0
:10DD880009B1082907D149084FF68F70CC582040AF
:10DD9800C850C8580AE00439C1F34E0148F6FF706C
:10DDA800CC582040C8501202C85892B20243CA50F8
:10DDB80030BD4163704781637047C1637047016438
:10DDC8007047038B23F070031B041B0C0B43038366
:10DDD8007047038B23F4E0431B041B0C43EA012325
:10DDE8009BB203837047838B23F070031B041B0CC7
:10DDF8000B4383837047838B23F4E0431B041B0C82
:10DE080043EA01239BB283837047038B23F0080303
:10DE18001B041B0C0B4303837047038B23F4006321
:10DE28001B041B0C43EA01239BB203837047838BBB
:10DE380023F008031B041B0C0B4383837047838B5D
:10DE480023F400631B041B0C43EA01239BB2838366
:10DE58007047038B23F004031B041B0C0B43038341
:10DE68007047038B23F480631B041B0C43EA0123D4
:10DE78009BB203837047838B23F004031B041B0CA2
:10DE88000B4383837047838B23F480631B041B0C31
:10DE980043EA01239BB283837047038B23F08003FB
:10DEA8001B041B0C0B4303837047038B09025B04A1
:10DEB80041EA53439BB203837047838B23F080036B
:10DEC8001B041B0C0B4383837047838B09025B0481
:10DED80041EA53439BB283837047038C23F00203C8
:10DEE8001B041B0C0B4303847047038C23F00803AB
:10DEF8001B041B0C0B4303847047038C23F0200383
:10DF08001B041B0C43EA01139BB203847047038C68
:10DF180023F080031B041B0C43EA01139BB2038408
:10DF28007047038C23F400731B041B0C43EA012382
:10DF38009BB203847047038C23F400631B041B0CFF
:10DF480043EA01239BB203847047038C23F40053F4
:10DF58001B041B0C43EA01339BB20384704710B5C2
:10DF6800048C01238B40A4B224EA03030384038CAA
:10DF780012FA01F10B439BB2038410BD10B5048C57
:10DF880004238B40A4B224EA03030384038C12FA0B
:10DF980001F10B439BB2038410BD002301220380CF
:10DFA80043808280C38003817047406B7047806BD9
:10DFB8007047C06B7047006C7047038B23F00C03ED
:10DFC8001B041B0C0383038B9BB20B430383704717
:10DFD800038B23F440631B041B0C0383038B9BB24A
:10DFE80043EA01239BB203837047F8B50C4649887E
:10DFF800A288B4F800E02389054600290CBF02274F
:10E008000027012A14BF01260226BEF1000F10D1F5
:10E01800FFF72EFC2846E188FFF7CFFF2846394650
:10E0280032462389FFF73DFCE1882846BDE8F840E1
:10E03800CEE7FFF736FC2846E188FFF7C9FF2846F8
:10E04800394632462389FFF713FCE1882846BDE8A4
:10E05800F840B2E7838B23F00C031B041B0C83836B
:10E06800838B9BB20B4383837047838B23F440637A
:10E078001B041B0C8383838B9BB243EA01239BB253
:10E0880083837047F8B50D460B88AA8849880446EB
:10E098003BB92B89FFF7ECFBE9882046BDE8F8403F
:10E0A8008BE7042B07D12B89FFF7FBFBE988204678
:10E0B800BDE8F8408CE7082BB5F808C0078C1DD1DF
:10E0C80027F480773F043F0C0784868B038CB6B215
:10E0D8009BB226F0F30623F4206346EA0C1C43EABD
:10E0E80001211FFA8CFC89B24CEA020241F48071CA
:10E0F80082830184E988BDE8F840ABE727F48057BC
:10E108003F043F0C0784868B038C26F4407623F467
:10E11800005336055B04360D5B0C46EA022243EADF
:10E12800013342EA0C329BB2E98892B243F480533D
:10E1380082830384BDE8F84097E74A880B88134335
:10E148008A881343CA8813430A8913434A891343A5
:10E158008A8913439BB2A0F8443070470023038098
:10E1680043808380C3800381438183817047B0F8F3
:10E17800443029B16FEA43436FEA53439BB201E04D
:10E188005B045B0CA0F844307047838819B19BB2DC
:10E1980043F0040303E023F004031B041B0C8380F7
:10E1A8007047838819B19BB243F0010303E023F061
:10E1B80001031B041B0C8380704783899BB20AB13F
:10E1C800194301E023EA0101818170478182704788
:10E1D800038A19420CBF002001207047C94389B245
:10E1E80001827047038A828911EA030092B203D040
:10E1F80011420CBF002001207047C94389B2018237
:10E2080070470A43A0F84820704783899BB20AB137
:10E21800194301E023EA010181817047838819B11C
:10E228009BB243F0080303E023F008031B041B0C14
:10E2380083807047038923F007031B041B0C0381A9
:10E248007047038923F070031B041B0C0B430381E5
:10E2580003899BB243F007030381704738B50D4625
:10E2680011460122602D044602D1FFF71AFB01E096
:10E27800FFF7FEFA238923F070031B041B0C1D43D0
:10E28800258123899BB243F00703238138BD038985
:10E2980023F070031B041B0C0B4303817047838816
:10E2A80023F070031B041B0C838083889BB20B43F1
:10E2B80083807047038923F007031B041B0C038129
:10E2C80003899BB20B4303817047038923F08003C2
:10E2D8001B041B0C038103899BB20B43038170470A
:10E2E80010B50489E4B20C43144344EA0324A4B2ED
:10E2F800048110BD10B50446FFF7F2FF23899BB2D5
:10E3080043F48043238110BD10B50446FFF7E8FFAE
:10E31800238923F077031B041B0C43F07703238125
:10E3280010BD70B50489068B058C26F44076ADB215
:10E3380026F0030624F00704360425F022052404F9
:10E34800360C1543240C46F4807645EA0315214320
:10E3580046F00106ADB201810683058470BD83884D
:10E3680019B19BB243F0800303E023F080031B0440
:10E378001B0C83807047A0F85010704708B5234BDA
:10E38800984205D110200121FEF7F2FF102037E056
:10E398001F4B984207D14FF400300121FEF7DCFFF4
:10E3A8004FF4003009E01B4B98420BD14FF480200A
:10E3B8000121FEF7D1FF4FF480200021BDE808407D
:10E3C800FEF7CABF144B984207D14FF40020012131
:10E3D800FEF7C2FF4FF40020EFE7104B984207D139
:10E3E8004FF480100121FEF7B7FF4FF48010E4E7E7
:10E3F8000B4B984209D120200121FEF7B9FF2020BC
:10E408000021BDE80840FEF7B3BF08BD0010014079
:10E418000044004000480040004C004000500040CC
:10E4280000140140038ACA889BB223F4405330B5D4
:10E4380013430D46038283890989AA8823F4B053BC
:10E448000A43698923F00C031B040A431B0C92B28C
:10E4580013438381838AAA899BB223F440731343AD
:10E4680085B0838204466846FEF7A6FE1A4B9C4296
:10E4780003D003F580639C4201D1039B00E0029B1B
:10E48800A28912B2002A4FF019012A6801FB03F190
:10E4980001DA520000E092006423B1FBF2F1B1FB13
:10E4A800F3F21201100903FB1011A08900B2002831
:10E4B80006DAC9003231B1FBF3F303F0070305E0D4
:10E4C80009013231B1FBF3F303F00F031A4392B29F
:10E4D800228105B030BD00BF001001404FF4165333
:10E4E80003600C2200238380C380038142818381DF
:10E4F80070470B88028A10B54C8823438C88C988DA
:10E50800234392B20B4322F470629BB213430382FB
:10E5180010BD0023038043808380C38070478389B4
:10E5280019B19BB243F4005303E023F400531B04D6
:10E538001B0C83817047038B03F47F430383038B96
:10E548009BB20B4303837047838929B16FEA434326
:10E558006FEA53439BB201E05B045B0C8381704715
:10E56800838A19B19BB243F4006303E023F4006388
:10E578001B041B0C83827047C905C90D8180704735
:10E588008088C005C00D7047038A23F00F031B0461
:10E598001B0C0382038A9BB20B4303827047838957
:10E5A80019B19BB243F0020303E023F002031B04FA
:10E5B8001B0C83817047838923F400631B041B0CA5
:10E5C800838183899BB20B4383817047038A23F03D
:10E5D80020031B041B0C0382038A9BB20B43038298
:10E5E8007047038A19B19BB243F4804303E023F4D4
:10E5F80080431B041B0C0382704783899BB243F042
:10E60800010383817047838A19B19BB243F00803E1
:10E6180003E023F008031B041B0C83827047038B61
:10E62800DBB20383038B9BB243EA01230383704766
:10E63800838A19B19BB243F0200303E023F020033F
:10E648001B041B0C83827047838A19B19BB243F069
:10E65800100303E023F010031B041B0C8382704794
:10E66800838A23F004031B041B0C8382838A9BB2D6
:10E678000B4383827047838A19B19BB243F002032C
:10E6880003E023F002031B041B0C83827047838A78
:10E698009BB20AB1194301E023EA01018182704764
:10E6A800C1F3421310B501F01F01012414FA01F15E
:10E6B800A34201D10C3004E0022B01D1103000E05C
:10E6C800143003680AB1194301E023EA010101602B
:10E6D80010BD038819420CBF002001207047C943B0
:10E6E80089B201807047012210B501F01F03C1F300
:10E6F80042149A40012C01D1838903E0022C0CBFFB
:10E70800038A838A9BB21340028892B243B1090AF2
:10E71800012313FA01F111420CBF0020012010BDA2
:10E72800184610BD090A01238B40DB439BB20380C6
:10E73800704700BF81F0004102E000BF83F0004352
:10E7480030B54FEA41044FEA430594EA050F08BF84
:10E7580090EA020F1FBF54EA000C55EA020C7FEA48
:10E76800645C7FEA655C00F0E2804FEA5454D4EBC5
:10E778005555B8BF6D420CDD2C4480EA020281EA8F
:10E78800030382EA000083EA010180EA020281EAC7
:10E798000303362D88BF30BD11F0004F4FEA013119
:10E7A8004FF4801C4CEA113102D0404261EB410128
:10E7B80013F0004F4FEA03334CEA133302D05242AE
:10E7C80063EB430394EA050F00F0A780A4F101046A
:10E7D800D5F1200E0DDB02FA0EFC22FA05F28018A4
:10E7E80041F1000103FA0EF2801843FA05F359418A
:10E7F8000EE0A5F120050EF1200E012A03FA0EFC09
:10E8080028BF4CF0020C43FA05F3C01851EBE37132
:10E8180001F0004507D54FF0000EDCF1000C7EEB4F
:10E8280000006EEB0101B1F5801F1BD3B1F5001F8D
:10E838000CD349085FEA30004FEA3C0C04F10104AC
:10E848004FEA445212F5800F80F09A80BCF1004FD5
:10E8580008BF5FEA500C50F1000041EB045141EA57
:10E86800050130BD5FEA4C0C404141EB010111F458
:10E87800801FA4F10104E9D191F0000F04BF014603
:10E888000020B1FA81F308BF2033A3F10B03B3F1E1
:10E8980020020CDA0C3208DD02F1140CC2F10C0271
:10E8A80001FA0CF021FA02F10CE002F11402D8BFCF
:10E8B800C2F1200C01FA02F120FA0CFCDCBF41EA9B
:10E8C8000C019040E41AA2BF01EB0451294330BD6A
:10E8D8006FEA04041F3C1CDA0C340EDC04F1140447
:10E8E800C4F1200220FA04F001FA02F340EA03001E
:10E8F80021FA04F345EA030130BDC4F10C04C4F164
:10E90800200220FA02F001FA04F340EA0300294643
:10E9180030BD21FA04F0294630BD94F0000F83F48D
:10E92800801306BF81F480110134013D4EE77FEA70
:10E93800645C18BF7FEA655C29D094EA050F08BFBC
:10E9480090EA020F05D054EA000C04BF194610469D
:10E9580030BD91EA030F1EBF0021002030BD5FEAE1
:10E96800545C05D14000494128BF41F0004130BD09
:10E9780014F580043CBF01F5801130BD01F000455D
:10E9880045F0FE4141F470014FF0000030BD7FEAD0
:10E99800645C1ABF194610467FEA655C1CBF0B46CB
:10E9A800024650EA013406BF52EA033591EA030FE2
:10E9B80041F4002130BD00BF90F0000F04BF0021DA
:10E9C800704730B54FF4806404F132044FF000050D
:10E9D8004FF0000150E700BF90F0000F04BF002186
:10E9E800704730B54FF4806404F1320410F00045EC
:10E9F80048BF40424FF000013EE700BF42004FEAE7
:10EA0800E2014FEA31014FEA02701FBF12F07F4363
:10EA180093F07F4F81F06051704792F0000F14BF60
:10EA280093F07F4F704730B54FF4607401F00045A4
:10EA380021F0004120E700BF50EA010208BF7047FB
:10EA480030B54FF000050AE050EA010208BF7047F0
:10EA580030B511F0004502D5404261EB41014FF459
:10EA6800806404F132045FEA915C3FF4DCAE4FF05D
:10EA780003025FEADC0C18BF03325FEADC0C18BF44
:10EA8800033202EBDC02C2F1200300FA03FC20FA95
:10EA980002F001FA03FE40EA0E0021FA02F11444E2
:10EAA800C1E600BF70B54FF0FF0C4CF4E06C1CEAF7
:10EAB80011541DBF1CEA135594EA0C0F95EA0C0F6C
:10EAC80000F0DEF82C4481EA030621EA4C5123EADF
:10EAD8004C5350EA013518BF52EA033541F480110E
:10EAE80043F4801338D0A0FB02CE4FF00005E1FBC1
:10EAF80002E506F00042E0FB03E54FF00006E1FB0B
:10EB080003569CF0000F18BF4EF0010EA4F1FF044D
:10EB1800B6F5007F64F5407404D25FEA4E0E6D418D
:10EB280046EB060642EAC62141EA55514FEAC5209E
:10EB380040EA5E504FEACE2EB4F1FD0C88BFBCF51A
:10EB4800E06F1ED8BEF1004F08BF5FEA500E50F1CB
:10EB5800000041EB045170BD06F0004646EA010191
:10EB680040EA020081EA0301B4EB5C04C2BFD4EBC3
:10EB78000C0541EA045170BD41F480114FF0000EBC
:10EB8800013C00F3AB8014F1360FDEBF002001F02A
:10EB9800004170BDC4F10004203C35DA0C341BDCA4
:10EBA80004F11404C4F1200500FA05F320FA04F076
:10EBB80001FA05F240EA020001F0004221F00041AA
:10EBC80010EBD37021FA04F642EB06015EEA430E1D
:10EBD80008BF20EAD37070BDC4F10C04C4F120054D
:10EBE80000FA04F320FA05F001FA04F240EA020000
:10EBF80001F0004110EBD37041F100015EEA430ED1
:10EC080008BF20EAD37070BDC4F1200500FA05F2F0
:10EC18004EEA020E20FA04F301FA05F243EA02036F
:10EC280021FA04F001F0004121FA04F220EA02007E
:10EC380000EBD3705EEA430E08BF20EAD37070BDC4
:10EC480094F0000F0FD101F00046400041EB0101A4
:10EC580011F4801F08BF013CF7D041EA060195F086
:10EC6800000F18BF704703F00046520043EB030340
:10EC780013F4801F08BF013DF7D043EA060370472D
:10EC880094EA0C0F0CEA135518BF95EA0C0F0CD038
:10EC980050EA410618BF52EA4306D1D181EA03017E
:10ECA80001F000414FF0000070BD50EA410606BF78
:10ECB8001046194652EA430619D094EA0C0F02D1BD
:10ECC80050EA013613D195EA0C0F05D152EA033602
:10ECD8001CBF104619460AD181EA030101F0004120
:10ECE80041F0FE4141F470014FF0000070BD41F069
:10ECF800FE4141F4780170BD70B54FF0FF0C4CF443
:10ED0800E06C1CEA11541DBF1CEA135594EA0C0F61
:10ED180095EA0C0F00F0A7F8A4EB050481EA030EAE
:10ED280052EA03354FEA013100F088804FEA033395
:10ED38004FF0805545EA131343EA12634FEA022263
:10ED480045EA111545EA10654FEA00260EF0004124
:10ED58009D4208BF964244F1FD0404F5407402D276
:10ED68005B084FEA3202B61A65EB03055B084FEA07
:10ED780032024FF480104FF4002CB6EB020E75EB04
:10ED8800030E22BFB61A754640EA0C005B084FEA2C
:10ED98003202B6EB020E75EB030E22BFB61A7546A9
:10EDA80040EA5C005B084FEA3202B6EB020E75EBF4
:10EDB800030E22BFB61A754640EA9C005B084FEA6C
:10EDC8003202B6EB020E75EB030E22BFB61A754679
:10EDD80040EADC0055EA060E18D04FEA051545EA68
:10EDE80016754FEA06164FEAC30343EA52734FEA11
:10EDF800C2025FEA1C1CC0D111F4801F0BD141EA8A
:10EE080000014FF000004FF0004CB6E711F4801FEE
:10EE180004BF01430020B4F1FD0C88BFBCF5E06FCE
:10EE28003FF6AFAEB5EB030C04BFB6EB020C5FEADE
:10EE3800500C50F1000041EB045170BD0EF0004E33
:10EE48004EEA113114EB5C04C2BFD4EB0C0541EA65
:10EE5800045170BD41F480114FF0000E013C90E662
:10EE680045EA060E8DE60CEA135594EA0C0F08BF26
:10EE780095EA0C0F3FF43BAF94EA0C0F0AD150EA25
:10EE880001347FF434AF95EA0C0F7FF425AF1046B8
:10EE980019462CE795EA0C0F06D152EA03353FF4E0
:10EEA800FDAE1046194622E750EA410618BF52EA5D
:10EEB80043067FF4C5AE50EA41047FF40DAF52EA31
:10EEC80043057FF4EBAE12E74FF0FF3C06E000BFCE
:10EED8004FF0010C02E000BF4FF0010C4DF804CDDB
:10EEE8004FEA410C7FEA6C5C4FEA430C18BF7FEA9B
:10EEF8006C5C1BD001B050EA410C0CBF52EA430CC9
:10EF080091EA030F02BF90EA020F0020704710F148
:10EF1800000F91EA030F58BF994208BF90422CBFD7
:10EF2800D8176FEAE37040F0010070474FEA410CD0
:10EF38007FEA6C5C02D150EA013C07D14FEA430CEE
:10EF48007FEA6C5CD6D152EA033CD3D05DF8040B5F
:10EF5800704700BF8446104662468C461946634691
:10EF680000E000BF01B5FFF7B7FF002848BF10F168
:10EF7800000F01BD4DF808EDFFF7F4FF0CBF0120AD
:10EF880000205DF808FB00BF4DF808EDFFF7EAFF29
:10EF980034BF012000205DF808FB00BF4DF808EDE4
:10EFA800FFF7E0FF94BF012000205DF808FB00BFD9
:10EFB8004DF808EDFFF7CEFF94BF012000205DF863
:10EFC80008FB00BF4DF808EDFFF7C4FF34BF012070
:10EFD80000205DF808FB00BF4FEA410212F500125D
:10EFE80015D211D56FF47873B3EB625212D94FEA88
:10EFF800C12343F0004343EA505311F0004F23FA72
:10F0080002F018BF404270474FF00000704750EAC6
:10F01800013005D111F0004008BF6FF00040704783
:10F028004FF00000704700BF4A0011D212F50012DD
:10F0380011D20DD56FF47873B3EB62520ED44FEA48
:10F04800C12343F0004343EA505323FA02F07047C8
:10F058004FF00000704750EA013002D14FF0FF3006
:10F0680070474FF0000070474FEA4102B2F1E043A9
:10F0780024BFB3F5001CDCF1FE5C0DD901F0004C97
:10F088004FEAC0024CEA5070B2F1004F40EB8300E7
:10F0980008BF20F00100704711F0804F21D113F113
:10F0A8003872BCBF01F00040704741F480114FEA4C
:10F0B8005252C2F11802C2F1200C10FA0CF320FAD5
:10F0C80002F018BF40F001004FEAC1234FEAD323F2
:10F0D80003FA0CFC40EA0C0023FA02F34FEA43035C
:10F0E800CCE77FEA625307D150EA01331EBF4FF0E5
:10F0F800FE4040F44000704701F0004040F0FE4000
:10F1080040F40000704700BF4BB942B9002908BF5E
:10F11800002802D04FF0FF31084600F037B882B01F
:10F12800EC462DE9005000F01BF8DDF804E002B0D1
:10F138000CBC7047F8B5144606460F461D4600F04D
:10F1480027F804FB01F300FB0535A4FB0023EB18AB
:10F15800069CB21A67EB0303C4E90023F8BD00BF9D
:10F16800F8B5144606460F461D4600F075F900FB33
:10F1780005F5A0FB042304FB0155EB18069CB21A05
:10F1880067EB0303C4E90023F8BD00BF704700BF65
:10F1980000292DE9F0071D46C0F29E800024002DAD
:10F1A800C0F2958007460D4616469C46002B3ED178
:10F1B8008A4254D9B2FA82F343B1C3F1200620FA45
:10F1C80006F501FA03F19A4029439840160CB1FB61
:10F1D800F6F597B206FB15114FEA104C07FB05F33D
:10F1E8004CEA01418B4209D9891805F1FF3C80F0AE
:10F1F80015818B4240F21281023D8918C3EB010C44
:10F20800BCFBF6F306FB13C180B207FB03F740EA29
:10F218000140874207D9591E821880F0058197421C
:10F2280040F20281023B43EA0542002303E08B429D
:10F238000AD900231A461046194614B1404261EB18
:10F248004101BDE8F0077047B3FA83F3002B40F0A3
:10F2580087808C4501D38242ECD80122EBE712B9B2
:10F268000123B3FBF2F2B2FA82F6002E3AD1891AE0
:10F27800150C1FFA82FC0123B1FBF5F705FB1711EA
:10F288004FEA10480CFB07F648EA01418E4207D9BD
:10F29800891807F1FF3802D28E4200F2DA80474619
:10F2A800891BB1FBF5F605FB161180B20CFB06FCB9
:10F2B80040EA0140844507D9711E821880F0B08069
:10F2C800944540F2AD80023E46EA0742B3E7E44384
:10F2D800524263EB430365E7404261EB41014FF063
:10F2E800FF345CE7B240C6F1200521FA05F320FAA5
:10F2F80005F701FA06F9150CB3FBF5F847EA090911
:10F308001FFA82FC05FB18374FEA19410CFB08F37A
:10F3180041EA0747B040BB420AD9BF1808F1FF319C
:10F3280080F09580BB4240F29280A8F10208BF1895
:10F33800FE1AB6FBF5F305FB13611FFA89F90CFBFE
:10F3480003F649EA01418E4206D95F1E891878D230
:10F358008E4276D9023B8918891B43EA08438BE71A
:10F36800C3F1200726FA07F80CFA03F248EA020C60
:10F3780021FA07F105FA03FA4FEA1C4920FA07F5C2
:10F38800B1FBF9F845EA0A0509FB18172A0C1FFA18
:10F398008CFA0AFB08F142EA0747B94206FA03F673
:10F3A80009D917EB0C0708F1FF324ED2B9424CD9F4
:10F3B800A8F1020867447F1AB7FBF9F209FB12713A
:10F3C800ADB20AFB02FA45EA01418A4507D9551E42
:10F3D80011EB0C0137D28A4535D9023A614442EA29
:10F3E80008424FEA124C1FFA86F808FB0CF7360C55
:10F3F80095B208FB05F806FB057505EB184506FBF5
:10F408000CFCAF4288BF0CF5803CCAEB01010CEB49
:10F418001546B14212D309D000230CE76546EDE644
:10F428000E4646EA074206E70B46FCE61FFA88F84E
:10F4380000FA03F308EB0545AB42EDD2013A00238D
:10F44800F9E63B4688E72A46C9E79046B3E7884687
:10F458006EE7023F891823E72DE9F00F14460546A9
:10F468000E46002B3FD18A424AD9B2FA82F343B101
:10F47800C3F1200025FA00F201FA03F69C40164376
:10F488009D40210CB6FBF1F22F0CA0B201FB126CCF
:10F4980000FB02F347EA0C46B34208D9571E361957
:10F4A80080F0FF80B34240F2FC80023A3619F61A27
:10F4B800B6FBF1F301FB1361ADB200FB03F045EAC3
:10F4C8000141884207D95E1E091980F0EC80884204
:10F4D80040F2E980023B43EA024200231046194603
:10F4E800BDE8F00F70478B4243D8B3FA83F4002C81
:10F4F80042D18B42234601D382423BD80122EDE719
:10F5080012B90123B3FBF2F4B4FA84F2002A40F0F2
:10F518008A80091B260CA7B20123B1FBF6F006FB73
:10F5280010114FEA154C07FB00F24CEA01418A42E0
:10F5380007D9091900F1FF3C02D28A4200F2D380B0
:10F548006046C2EB010CBCFBF6F206FB12C1ADB281
:10F5580007FB02F745EA0145AF4207D9511E2C19AE
:10F5680080F0A380A74240F2A080023A42EA00421B
:10F57800B4E700231A46B1E7C4F1200722FA07F6D8
:10F5880003FA04F3334321FA07FA4FEA134C01FA5A
:10F5980004FB20FA07F141EA0B0BBAFBFCF70CFB62
:10F5A80017A61FFA83F84FEA1B4508FB07F945EA37
:10F5B8000645A94502FA04FA04D97A1EED18C0F0E6
:10F5C80088801746C9EB0505B5FBFCF60CFB1652FF
:10F5D8001FFA8BFB08FB06F84BEA0241884503D962
:10F5E800721EC91870D3164646EA0742170C1FFA4E
:10F5F8008AFC0CFB07F695B24FEA1A430CFB05FC94
:10F6080003FB056505EB1C4503FB07F3AE4288BF0A
:10F6180003F58033C8EB010103EB1543994250D33E
:10F6280047D000235AE79440C2F12008260C20FA5C
:10F6380008F721FA08F501FA02F9B5FBF6F847EAE6
:10F64800090906FB1855A7B24FEA194C4CEA054CB4
:10F6580007FB08F3634500FA02F509D91CEB040C13
:10F6680008F1FF323DD263453BD9A8F10208A44412
:10F67800C3EB0C02B2FBF6F306FB13201FFA89F961
:10F6880007FB03F249EA00418A4206D9581E0919C4
:10F6980025D28A4223D9023B0919891A43EA084329
:10F6A8003BE73A4603E7334615E70A4642EA004293
:10F6B80014E71FFA8CF100FA04F001EB0545A842A3
:10F6C800AFD2013A002309E788458CD9023EC91810
:10F6D8008AE7A9457FF675AF023FED1872E7034642
:10F6E800DBE79046C4E7023809192AE7002103E05E
:10F6F8000A4B5B584350043109480A4B42189A4256
:10F70800F6D3094A02E0002342F8043B074B9A4229
:10F71800F9D3FAF7E5F900F00DF8704744A20508A7
:10F7280000000020A40B0020A80B0020784F002028
:10F73800FEE70000984BF7B54FF4FA661E60974A4B
:10F74800974B984F1A60984A984B1A60984B42F218
:10F7580010721A60974B64241C6001233B70964B0F
:10F768004FF0FF321A60954B00251D70F8F7BEFB6D
:10F77800F6F730FDF6F73AFDF6F748FDF7F722FB06
:10F788002046F7F79FFFF7F743FB2046F7F79AFF66
:10F79800F8F792FBF8F7CCF9F7F7A2FF2046F7F74E
:10F7A80091FFFAF7BFFA2046F7F78CFF4FF4FA50AB
:10F7B800F7F7F4FE2046F7F785FFF7F75BFA2046E0
:10F7C800F7F780FF2846F8F75FF87D48F7F77AFFE4
:10F7D800F4F7BCFD2046F7F775FF7A4B03F11002EA
:10F7E80029468DE8240028465A681B68F4F7B4FFB8
:10F7F8003046F7F767FF2846F5F72EFA4FF6FF7001
:10F80800F5F740FA322003216F4A2B46F5F752FBF1
:10F8180096206E4A8C212B46F5F74CFB9620A021AA
:10F828006B4A2B46F5F746FB6A4A2B469620B421CD
:10F83800F5F740FBFAF7DAF85021DC20FAF7A9F8D7
:10F848003046F7F73FFF644A2B46DC212846F5F798
:10F8580031FB6248F7F736FF2046F7F733FFF6F734
:10F86800D1FF2046F7F72EFF9FED5D0AF8F724F841
:10F878002046F7F727FFF7F74DFFF5F7E3FD20469A
:10F88800F7F720FF14200146F6F72CFD2846F6F777
:10F898007FFD2046F7F716FFF6F7FEFE2046F7F73E
:10F8A80011FFF7F787FA2046F7F70CFFF6F7FAFF8C
:10F8B80000B13D70F7F702F808B1FAF741F8494B83
:10F8C80000241C70F2F792F9F5F772FD08B9464862
:10F8D80002E0464B46481C70F2F79FF9F6F7DCF950
:10F8E800F8F79FFFF8F7D2FFF8F71FFDF8F706FCC7
:10F8F800FAF749F8FAF7A8F9FAF798F83D4B3E4EA7
:10F908003E4D802814BF4FF480504FF4806018801B
:10F918003B4BC01018803746F6F7E6FF337833B113
:10F92800012B02D1F8F732F901E0F8F757F9002472
:10F938003C70F8F7A9FAF3F78BFFF9F747FF2A8825
:10F9480012B2012A0FD12F484FF40051FDF771F977
:10F95800F9F744F8F8F72EFA2A484FF400512246EE
:10F96800FDF767F92C80284B1B7843B1FAF73EF86E
:10F97800F0209621FAF70DF82448F7F799FC244C63
:10F988002046FBF7BAFC0028C6D02378112BC3D138
:10F99800F9F744FFC0E700BF2C3C0020E0673500C2
:10F9A800643C00202C0E002080C3C9018442002042
:10F9B800584200200C3C00205C3C0020E44300201E
:10F9C80000127A00A87A0108B09A0508CA9A0508B0
:10F9D800D59A0508E19A0508EA9A0508002D31012B
:10F9E8000000FA443C3C0020140F0020F43B0020A7
:10F9F80000110020583C00205C420020BC0C002074
:10FA08007042002000080240D80C002040420F003D
:10FA1800F53B002010B4314C0180B1F5807F446083
:10FA28008270C37052D00DD9B1F5806F39D017D913
:10FA3800B1F5006F2ED0B1F5805F24D0FF2040B221
:10FA480010BC704720293AD014D9402930D08029D9
:10FA5800F4D123494FF02012C26081600020EEE704
:10FA6800B1F5007FEAD11F4B4FF00811C1608360E8
:10FA78000020E4E71029E1D11B494FF00122C260C0
:10FA880081600020DBE7194B4FF00111C1608360F2
:10FA98000020D4E7164A4FF00213C36082600020AA
:10FAA800CDE714494FF00412C26081600020C6E718
:10FAB800114B4FF04011C16083600020BFE70F4A2F
:10FAC8004FF08013C36082600020B8E70C4A4FF003
:10FAD8001013C36082600020B1E700BFD09904080A
:10FAE8000E8A0508DE890508CE8B0508D089050829
:10FAF800D2890508D68905084E8A0508CE8A0508E0
:10FB0800EE8905082DE9F00FB2B02E9030932E9BA8
:10FB180000882E9C5B68309FA4682D90451E03EBDF
:10FB28004506BF08209328942C952F911F921E9666
:10FB3800319700F03A814FEA900A4FEACA0B00F079
:10FB480003002F99299003F1080504EB0B00CDF869
:10FB580084A0CDF8A8B019951A921B9718961791FA
:10FB68002B90179A189E13883380B2F802C0A6F813
:10FB780002C09488B480D788F78008361896219FE9
:10FB8800199E0832179256F8041C56F8082C4FF0A4
:10FB9800000A4FF0000B002F00F06982CDE904AB9A
:10FBA800CDE906ABCDE902ABCDE900AB289CBC465C
:10FBB800029BDDF80C902568C2FBC5394FF00008A0
:10FBC80048EA030ACB46CDE902AB049BDDF814B042
:10FBD800C1FBC53BCDF824B0CDF82080DDE908ABEA
:10FBE800C1EA02004AEA030ACDE904AB069BDDF844
:10FBF8001CB03268C0FBD53BCDF82CB0CDF82880BE
:10FC0800DDE90AABC2EA01074AEA030ACDE906AB15
:10FC18009DE80108C7FBD50BCDF834B0CDF830808E
:10FC2800DDE90CAB4AEA000A63680298CDE900AB4B
:10FC38000834DDF80CB0C1FBC30BCDF83CB0CDF8EF
:10FC48003880DDE90EAB4AEA000ACDE902AB7168FB
:10FC58000498DDF814B0C2FBC30BCDF844B0CDF85E
:10FC68004080DDE910AB4AEA000ACDE904AB06980A
:10FC7800DDF81CB0C7FBD30BCDF84CB0CDF84880ED
:10FC8800DDE912ABC1EA02054AEA000ACDE906AB92
:10FC98009DE80108C5FBD30BCDF854B0CDF85080D2
:10FCA800DDE914AB08364AEA000ABCF1010CCDE9DB
:10FCB80000AB7FF47DAF2A9D19982B9B2E18299FA6
:10FCC800002F35D01868039F029BC2FBC037002461
:10FCD8001D971C94DDE91C4544EA0304CDE902455F
:10FCE800049B059DC1FBC035002723952297DDE9BC
:10FCF800224544EA0304CDE90445C1EA0203079D0D
:10FD0800069AC3FBD02525952497DDE9244544EAC6
:10FD180002043368C3EA0101CDE9064553465D464E
:10FD2800C1FBD03527952697DDE926AB4AEA030AB9
:10FD3800069A029C0499039D079FD30B059AE60B2C
:10FD4800C90B46EA454043EA474441EA424604F3C0
:10FD58000F0500F30F0C199BCCEA054706F30F00BB
:10FD68001A9D1B9E2F604FEADA3A08334AEA4B4B3A
:10FD78000BF30F04C0EA04426A600835711E199338
:10FD88001A951B917FF4EDAE319A2F9E1E991F9BF9
:10FD9800DDF880B0D00037180D182F970BEB000A4C
:10FDA8001F181E951F97CDF880A0DDF8C0C01CF065
:10FDB800030BCDF820B000F086802D9BDDF8BC80C9
:10FDC800CDF808B05808DDF880A0DDF8A0B006909E
:10FDD800CDF81080049A1E9E32F8025B069826F829
:10FDE800025B0492BAF80270BBF80230BAF800203D
:10FDF800BBF800401E9617FB03F112FB04F6451EE4
:10FE08004FEAE17711EB06082B4605F0010047EBB6
:10FE1800E6790AF104020BF10401002D3BD0A8B1E8
:10FE2800B2F800C0BBF80470548848881CFB07F57A
:10FE380018EB050749EBE57614FB00F917EB090801
:10FE480046EBE97904320431013B24D00F88B2F83B
:10FE580000C0568848888C8895881CFB07FC18EBDE
:10FE68000C0816FB00F7D088CE8849EBEC7C15FB14
:10FE780004F518EB07084CEBE77918EB050710FBBE
:10FE880006FC49EBE57417EB0C0844EBEC790832F7
:10FE98000831023BDAD11F9A02994FEAD83545EA70
:10FEA800494404F30F0322F8023B4F1E0AF1020AE9
:10FEB8001F9202978ED1DDF880A0DDF820B00AEB02
:10FEC8004B0ACDF880A02C9E2E98B50840683FD0EC
:10FED800209F47EA000212F0030F00F1080307F120
:10FEE800080214BF002101219F4298BF904294BF8D
:10FEF80000260126314277D097E8420001600121AF
:10FF08006C1EA942466004EA010419D044B192E883
:10FF18001200196002215C6008320833A9420FD030
:10FF280092E850001C605E60966802F1080BD26887
:10FF38009E600231DA601033A9420BF10802EFD15A
:10FF4800DDF880C0ED000CEB050B4019CDF880B052
:10FF58002C9C14F0030343D05A085400002A00F0E4
:10FF68008E80209D40EA050717F0030F209F14BFDD
:10FF780000250125011D3E1D012B94BF002505F01C
:10FF880001058F4298BFB04294BF002101210D4264
:10FF980075D039689200BF18A342016020971044B9
:10FFA800C4EB03011CD0209B013933F8024B0A46ED
:10FFB80020F8024B01F0010192B129B133F8021B7C
:10FFC800013A20F8021B0BD01C46014634F802CB3C
:10FFD80021F802CB5D88A31C4580881C023AF3D126
:10FFE80032B0BDE8F00F7047B7F800C0A0F800C005
:08FFF8007C884480BE888680ED
:020000040801F1
:10000000691EFE880C46BA4601F00101C680002C2C
:100010009AD089B1B2F800B0A3F800B051885980E5
:10002000B2F804C0A3F804C0B2F806B00832A3F8CE
:1000300006B00833013C87D016881E80518859804D
:10004000B2F804B0A3F804B0B2F806C0A3F806C032
:1000500016891E8103F1080B5189ABF802109389B0
:10006000ABF80430D6891032023C0BF10803ABF830
:100070000660E1D168E7289BCDE904ABCDE906AB8A
:10008000CDE902AB1FE6194691E700BF2DE9F00F5D
:100090009CB006780F900F9C40880F9DA4686D68F7
:1000A0001990B3FBF6FA471E4FEA5A0804EB4709CA
:1000B000AAEB480340460A940D951A97CDF86C8038
:1000C0000C911492CDF82C901193002800F0B5817A
:1000D0001746199A199CCDF848809108CA001591C5
:1000E00004F00303A918179216931097189176003D
:1000F00075084FEA450C002D00F03B840B9FDDF89E
:10010000308047EA080010F0030F14BF00210121DE
:1001100008F10404381D012E94BF002101F00101F3
:10012000804598BFA74294BF4FF000094FF00109E6
:1001300011EA090F00F01D84BB46D8F80020012306
:100140006F1EAB42CBF8002007EA030721460246A8
:1001500014D237B1246802230431021DAB4204607B
:100160000CD20C46104654F8047B40F8047B4968D6
:1001700002335160211D021DAB42F2D3DDF8308005
:10018000DDF82CB04FEA4C05664508EB05020BEB99
:100190000503CCEB06001DD0013832F802CB014636
:1001A00023F802CB00F00100A1B128B132F8029B84
:1001B000013923F8029B0DD014461F4634F8029BE8
:1001C00027F8029BB2F802A0A21CA3F802A0BB1C55
:1001D0000239F1D10C9ADDF83CC00B989CF80080F4
:1001E000710053180A9E0C93159BCDF84C8045184E
:1001F00006EB48020B950E92002B00F0B183002411
:100200000025CDE90445CDE9024507930D99134634
:100210000A9AB3F804A0B2F806B0CDF804A0B3F877
:1002200006A00E881588CDF820B0CDF824A0DDE911
:1002300002AB15FB06F51AEB050A4BEBE57BCDE9A6
:1002400002AB1F884888B2F802C0B3F80290B2F837
:1002500004808C88CDF81880DDE904AB16FB07F626
:100260001AEB060A4BEBE67BDDE902671CFB00F5A7
:10027000761910FB09F047EBE5771AEB000A4BEB18
:10028000E07BCDE902ABDDF818B0DDF804C0B1F8D1
:100290000680099D1BFB04F016EB000A47EBE07B90
:1002A000DDE9026714FB0CF4361947EBE477089C90
:1002B00014FB08F00831083208331AEB000418FB6D
:1002C00005F84BEBE075079816EB080A47EBE87B5F
:1002D0000138CDE90245CDE904AB079099D1179ECD
:1002E0000E9C0A9B1899A7199A190E97169F002F12
:1002F00073D00E9B31F8020B32F8024B33F8026BCD
:10030000DDE90289DDE904AB14FB00F47D1E10FB7E
:1003100006F618EB040849EBE4791AEB060A4BEBF6
:10032000E67B2F4605F00100CDE90289CDE904AB5B
:10033000002D52D0002873D031F8024B32F8020B56
:1003400033F8025B10FB04F614FB05F0DDE902450F
:10035000DDE90489A41945EBE67518EB000849EBC3
:10036000E079013FCDE90245CDE9048935D0C246A7
:10037000CB46DDE902890D461446049721462846FE
:100380001A4630F8026B31F8027B32F802CB6D88E6
:1003900064885B8817FB06F718EB070816FB0CF65A
:1003A00049EBE7791AEB060714FB05FA4BEBE67B02
:1003B00015FB03FC8C1C931C0499851C18EB0A0884
:1003C00049EBEA7917EB0C0A4BEBEC7B8A1ECDE983
:1003D00002890492D2D1CDE904AB029D039904981D
:1003E000DDF828A0059BEA0B109D42EA41481299CE
:1003F00008F30F09A5F80090DDF84C90C70B0AEB45
:100400008908281D4A1E47EA4346CDF8288006F38E
:100410000F0410906C8012920AD00F9C267866E62A
:10042000DDE904AB0D4614460497DDE90289A5E732
:10043000149F1B9B07EB83061496119F002F00F05F
:10044000A681DDF864B0DDF86480DDF834C04FEAE1
:100450009B09CDF81C904FEAC90908F0030A0CEB80
:10046000090BCDF82090CDF810A0CDF824B0DDF820
:100470003CC09CF8006075084FEA450C002D00F068
:100480007E820C990B980B9F40EA010414F0030F35
:1004900014BF002201220C1D0430012E94BF002243
:1004A00002F00102814298BFA74294BF00230123BA
:1004B0001A4200F06482BA4601230F68691EAB42FB
:1004C000CAF80070024601EA0307214614D237B188
:1004D00027680223211D021DAB4207600CD20C4687
:1004E000104654F8047B40F8047B4968023351609D
:1004F000211D021DAB42F2D3DDF83090DDF82C80D7
:100500004FEA4C05664509EB050208EB0503CCEB09
:1005100006001DD0013832F802BB014623F802BBA9
:1005200000F00100A1B128B132F8025B013923F8D3
:10053000025B0DD014461F4634F802AB27F802AB1D
:10054000B2F802C0A21CA3F802C0BB1C0239F1D150
:10055000DDF82CA0DDF830B0079876000AEB060C29
:100560000BEB0608CDF82CC0CDF83080002800F049
:10057000F0810A9ADDF834805788B2F800A0DDF8DF
:1005800028909488B9F80690B8F8062084460D980B
:1005900041880588B8F8040017FB01F61AFB05F33B
:1005A000B3461BEB03014FEAE67714FB00F047EB81
:1005B000E3750F180A9B19FB02F145EBE0750CF18E
:1005C000FF3617EB010AB14606F0010008F10802F8
:1005D00003F1080345EBE17B002E00F0858048B372
:1005E000DDF834C01E88BCF80840588851889788C8
:1005F0009D88B2F80680B3F806C016FB04F41AEB27
:10060000040A10FB01F14BEBE4761AEB010415FB35
:1006100007FB46EBE17014EB0B011CFB08F640EB0B
:10062000EB740832083311EB060A44EBE67BB9F1B0
:10063000010959D0CDE902ABCB46B3F80080B3F83D
:1006400008901688CDF8389018FB06F6DDE9028987
:100650005D88548898889188B2F806C0DF88B2F81F
:1006600008A015FB04F418EB060810FB01F149EB98
:10067000E67918EB040817FB0CF749EBE47918EB63
:10068000010849EBE17918EB070849EBE779CDE977
:100690000289DDF838905D89548998899189B2F88A
:1006A0000EC0DE8919FB0AF7DDE9028915FB04F4A7
:1006B00018EB070810FB01F149EBE77918EB040888
:1006C00049EBE47916FB0CF618EB010449EBE175F4
:1006D00010321033A01945EBE671BBF1020BCDE9E6
:1006E0000201AAD182468B460DF1200898E8160037
:1006F0006318049D9DB332F802CB33F8026B16FBEE
:100700000CF4013D1AEB040A294605F001004BEBFD
:10071000E47B25B358B132F8028B33F8020B10FB9F
:1007200008F71AEB070A4BEBE77B691E17D0144654
:10073000184634F8025B30F8027B52885B8817FB5E
:1007400005F81AEB08064BEBE87713FB02FBA21C3B
:10075000831C16EB0B0A47EBEB7B0239E7D10F9DAD
:10076000DDF8508095F800C00A9A119E4FEADA33FE
:1007700043EA4B4404F30F0028F8020B02EB4C074A
:10078000711E0A97CDF8508011917FF470AE1A9EB9
:100790000F9CB508A06842D00A9F47EA000616F0F1
:1007A000030F07F1080200F1080314BF0021012123
:1007B0009F4298BF904294BF4FF0000A4FF0010A49
:1007C00011EA0A0F7FD097E84200016001216C1EF8
:1007D000A942466004EA010419D044B192E812002B
:1007E000196002215C6008320833A9420FD092E8F8
:1007F00050001C605E60966802F10804D2689E603A
:100800000231DA601033A94204F10802EFD1DDF8B9
:1008100028A0ED000AEB05094019CDF82890DDF875
:1008200068A01AF003034AD05A085400002A00F0C6
:10083000A480DDF828B040EA0B0515F0030F14BFC3
:10084000002501250BF10406011D012B94BF002595
:1008500005F001058B4598BFB04294BF4FF0000CE6
:100860004FF0010C15EA0C0F00F08780DBF8001048
:1008700092009344A3420160CDF828B01044C4EB29
:1008800003011CD00A9B013933F8024B0A4620F8B9
:10089000024B01F0010192B129B133F8021B013A78
:1008A00020F8021B0BD01C46014634F802CB21F87D
:1008B00002CB5D88A31C4580881C023AF3D11CB092
:1008C000BDE8F00F7047B7F80090A0F800907C8862
:1008D0004480BE888680691EFE880C46B84601F0BA
:1008E0000101C680002C92D091B111881980B2F814
:1008F00002C0A3F802C0B2F804A0A3F804A0B2F8A2
:1009000006900832A3F806900833013C3FF47FAF0D
:1009100011881980B2F802C0A3F802C0B2F804909E
:10092000A3F80490B2F806A0A3F806A016891E81C9
:1009300003F1080C5189ACF802109389ACF804302B
:10094000D6891032023C0CF10803ACF80660DFD106
:100950005DE70D9A0A9B4FF0000A4FF0000BC8E6C6
:1009600000260027CDE904670A9A0D99CDE90267B0
:10097000BCE430460B9B0C9A0EE4194682E73046E5
:100980000B9B0C9AC6E500BF00B553EC102B42F24E
:10099000FB1223F00043C3F6E972934285B026DDD3
:1009A0004FF6FF72C7F6EF7293420BDD51EC100B5E
:1009B00002460B46FDF7C6FE02460B4643EC102BE3
:1009C00005B000BD684600F0BFFB00F00300012841
:1009D0009DED000B9DED021B1AD0022810D0F8B936
:1009E00000F0D2FE53EC102B10461946E4E79FEDC1
:1009F000101B00F0C9FE53EC102B10461946DBE724
:100A000000F0C2FE53EC102B104603F10041D3E777
:100A100001F0F6FB53EC102B104603F10041CBE73D
:100A2000012001F0EDFB53EC102B10461946C3E7F3
:100A300000000000000000002DE9F04759EC108B89
:100A4000C9F30A56A6F57E74073C132C4D46CA46D8
:100A5000474626DC002C4FDB4FF6FF76C0F20F0630
:100A600046FA04F606EA090555EA080517D044A334
:100A7000D3E9002351EC100BFDF766FE00220023A2
:100A8000FEF7A4FA00284AD0B9F1000F6EDB2AEA7B
:100A9000060A4FF000085346424643EC102BBDE8CF
:100AA000F087332C0CDDB4F5806FF8D151EC100BCE
:100AB0003A460B46FDF748FE41EC100BBDE8F087C7
:100AC000A6F58265033D4FF0FF3323FA05F515EADD
:100AD000080FE4D02AA3D3E9002351EC100BFDF753
:100AE00033FE00220023FEF771FAC0B1B9F1000F06
:100AF0001CDB28EA050813E021A3D3E9002351EC0D
:100B0000100BFDF721FE00220023FEF75FFA38B13B
:100B1000B9F1000F1BDB4FF00008C24600E0CA46E7
:100B20005346424643EC102BBDE8F087142C09D005
:100B3000C6F5866303334FF0010808FA03F818EB93
:100B40000708D6D30AF1010A28EA0508E8E729F0E0
:100B5000004848EA07084FF0000AD045CBF6F07A83
:100B600008BFCA4618BF4FF00008D9E74FF48013FA
:100B700043FA04F409EB040A89E700BFAFF30080ED
:100B80009C7500883CE4377E00B553EC102B42F294
:100B9000FB1223F00043C3F6E972934285B027DDD0
:100BA0004FF6FF72C7F6EF7293420BDD51EC100B5C
:100BB00002460B46FDF7C6FD02460B4643EC102BE2
:100BC00005B000BD684600F0BFFA00F00300012840
:100BD0009DED000B9DED021B1DD0022812D008BB1D
:100BE000012001F00DFB53EC102B10461946E3E7F2
:100BF00000209FED111B01F003FB53EC102B10465E
:100C00001946D9E7012001F0FBFA53EC102B1046EE
:100C100003F10041D0E700F0B7FD53EC102B104674
:100C20001946C9E700F0B0FD53EC102B104603F154
:100C30000041C1E7AFF300800000000000000000A9
:100C400000F0E6B8D0B52DED048BB0EE408AF0EEA2
:100C5000608A3C4C8AB000F0DBF994F90030B0EEC9
:100C6000409AF0EE609A013335D0B0EE480AF0EECB
:100C7000680A01F04FFD00282DD051EC180B00221E
:100C80000023FEF78FF930B32F4B24780193002314
:100C900008938DED028B8DED048B002C23D0002763
:100CA0000026CFF6F07751EC180B00220023CDE997
:100CB0000667FEF763F9002825D002239C420093C3
:100CC00036D0684601F05EFD002831D0089B002B2D
:100CD00027D19DED069BB0EE490AF0EE690A0AB0F5
:100CE000BDEC048BD0BD4FF6FF774FF06046CCF2E1
:100CF000EF7751EC180B00220023CDE90667FEF7D1
:100D00003DF90028D9D10123022C009315D0684663
:100D100001F038FD88B10D4801F036FD8DED060B70
:100D2000D4E701F0EFFF089B9DED069B0360D2E73F
:100D300001F0E8FF22230360C8E701F0E3FF21236D
:100D40000360E8E7E4020020449D0508A89F050829
:100D500010B52DED048BB0EE408AF0EE608A294C80
:100D60008AB000F02DFC94F90030B0EE409AF0EE1D
:100D7000609A01332BD0B0EE480AF0EE680A01F019
:100D8000C9FC20B351EC180B00220023FEF700F938
:100D9000E8B11D4B247801930123009300230893AD
:100DA0008DED048B8DED028BCCB10020002102462D
:100DB0000B46FDF7A5FF022CCDE9060115D101F088
:100DC000A1FF21230360089BABB99DED069BB0EE0C
:100DD000490AF0EE690A0AB0BDEC048B10BD00228E
:100DE000002343EC172B8DED067B684601F0CAFC0F
:100DF0000028E8D1E3E701F085FF089B9DED069B05
:100E00000360E4E7E40200204C9D050800000000B8
:100E1000F8B5B0EE407AF0EE607A53EC112B544204
:100E200010461D46002125F00047044353EC102BCB
:100E300047EAD474C7F6F0718C4216463DD8544246
:100E4000344323F0004242EAD4748C4235D805F191
:100E5000404101F5801101434FD0AC1704F002046A
:100E6000164344EAD37435D0384341D00021C7F645
:100E7000F0718F424FD00021C7F6F0718A4237D00F
:100E8000D21B12153C2A42DC002D7DDB53EC112BCA
:100E900051EC170BFDF734FF41EC100B01F030FC67
:100EA00001F06AFA51EC100B012C68D0022C57D0DB
:100EB000002C48D141EC170B07E051EC170B53EC19
:100EC000112BFDF741FC41EC170BB0EE470AF0EE99
:100ED000670AF8BD032CC7D801A151F824F000BF60
:100EE000CB0E0108CB0E0108090F0108030F010802
:100EF000002B25DB9FED307BE7E7BDE8F84001F0F4
:100F00003BBA9FED2F7BE0E79FED2F7BDDE72AA12A
:100F1000D1E90001C8E7BA423CD0032CABD801A10B
:100F200051F824F03B0F0108350F0108090F0108A3
:100F3000030F01089FED267BC7E79FED277BC4E7E2
:100F40009FED277BC1E730A3D3E90023FDF7FAFB30
:100F50001DA3D3E90023FDF7F5FB41EC170BB4E724
:100F600029A3D3E90023FDF7EDFB02460B4616A1AA
:100F7000D1E90001FDF7E6FB41EC170BA5E701F114
:100F8000004141EC170BA0E73C32BFF67FAF0020D9
:100F9000002189E7032CABD8DFE804F00B08050239
:100FA0009FED117B91E79FED127B8EE79FED127B0A
:100FB0008BE79FED137B88E7182D4454FB21F93F05
:100FC000182D4454FB2109C0182D4454FB2109401D
:100FD0000000000000000080000000000000000091
:100FE000182D4454FB21F9BFD221337F7CD902C094
:100FF000D221337F7CD90240182D4454FB21E9BF14
:10100000182D4454FB21E93F075C143326A6A13C6C
:101010002DE9F84F55EC104BB5F5801F2F4622DA1D
:1010200025F00043234368D0002D2046294670DB7D
:1010300000230022C4F25033FDF738FD4FF6FF7352
:101040000F46C7F6EF739F4204460D466FF0350218
:1010500010DD2046294622462B46FDF775FB41EC64
:10106000100BBDE8F88F4FF6FF73C7F6EF73002241
:101070009F42EEDC3B15A3F57E73073B9A18D60F13
:10108000901927F07F47C6F57E76FDF7A9FC073655
:1010900027F4700747EA065545EC104B8046894611
:1010A00001F00AFC4046494621A3D3E9002355EC50
:1010B000104BFDF7FBFC20A3D3E9002382468B46AF
:1010C00040464946FDF7F2FC1DA3D3E9002306463E
:1010D0000F4620462946FDF7E9FC02460B463046FE
:1010E0003946FDF731FB02460B4650465946FDF79F
:1010F0002BFB41EC100BBDE8F88F00210020CCF257
:10110000503100220023FDF7FBFD41EC100BBDE840
:10111000F88F22462B46FDF715FB00220023FDF732
:10112000EFFD41EC100BBDE8F88F00BFAFF300807E
:1011300000609F501344D33F362BF111F3FE593D0D
:101140000EE526157BCBDB3F2DE9F04F53EC102B42
:1011500042F2FB1223F00044C3F6E97294428FB0CE
:101160001E46074640F3AA804DF67B13C4F20203E5
:101170009C422ADC002E51EC100BDDA3D3E90023A6
:1011800040F3CA81FDF7DEFA42F2FB13C3F6F973AE
:101190009C428046894600F0AA80D7A3D3E9002369
:1011A000FDF7D0FA0D4604462B462246C7E9004516
:1011B00040464946FDF7C6FACFA3D3E90023FDF721
:1011C000C1FA0125C7E9020181E042F2FB13C4F232
:1011D00039139C4240F3AA804FF6FF73C7F6EF73B2
:1011E0009C4278DC4FEA245AAAF5826AAAF1060AE0
:1011F00051EC100BA4EB0A5319461D460446FDF7AB
:10120000EFFEFDF7EDFB8046894642464B46204601
:101210002946CDE90889FDF795FA00230022C4F29A
:101220007013FDF743FC0D460446FDF7D9FEFDF7AC
:10123000D7FB804689462046294642464B46CDE9A3
:101240000A89FDF77FFA00230022C4F27013FDF72C
:101250002DFC002204460D460023CDE90C45FDF788
:101260008DFE002800F07B81404649460022002385
:10127000FDF784FE03240AAD013C40B175E902018B
:1012800000220023FDF77AFE013C0028F6D1234618
:10129000022400949E4C08A839465246019400F05E
:1012A000ABFB002E054612DA7A68FB6802F10042B9
:1012B00003F100437A60FB60454208E0002200230E
:1012C00043EC172B87ED000B80ED027B00252846B1
:1012D0000FB0BDE8F08F51EC100B02460B46FDF746
:1012E00031FA0025C7E90201C7E90001EFE77AA357
:1012F000D3E90023FDF726FA79A3D3E9002380463A
:101300008946FDF71FFA0D4604462B462246C7E9DB
:10131000004540464946FDF715FA71A3D3E900237D
:10132000FDF710FA0125C7E90201D0E701F0E8F95D
:1013300059EC108B6CA3D3E9002340464946FDF7D6
:10134000B5FB00230022C3F6E073FDF7FDF9FDF7BE
:1013500047FE0546FDF744FB65A3D3E90023CDE92D
:101360000201FDF7A3FB02460B4640464946FDF746
:10137000E9F961A3D3E9002382468B46DDE9020146
:10138000FDF794FB1F2DCDE90401504659462BDC97
:101390006A1E604B53F82230A34225D0DDE90423B6
:1013A000FDF7D0F902460B46C7E90023814688467F
:1013B0004A46434650465946FDF7C4F9DDE9042341
:1013C000FDF7C0F9002E02460B46C7E90223BFF61F
:1013D0007EAF08F1004301F10041C7F800907B6047
:1013E000B860F9606D4272E7DDE90423FDF7AAF900
:1013F00088462415C8F30A53E31A102B8146C7E91F
:101400000001D5DD34A3D3E90023DDE90201FDF7B6
:101410004DFB8046894642464B4650465946FDF7AD
:1014200091F9CDE90601DDE9062350465946FDF75D
:1014300089F942464B46FDF785F929A3D3E90023F4
:1014400080468946DDE90201FDF730FB42464B4606
:10145000FDF778F9CDE90401DDE90423DDE90601B2
:10146000FDF770F98846C8F30A53E41A312C814617
:10147000C7E9000140F3958021A3D3E90023DDE90A
:101480000201FDF713FB8046894642464B46DDE9E3
:101490000601FDF757F982468B4652465B46DDE969
:1014A0000601FDF74FF942464B46FDF74BF916A3EF
:1014B000D3E9002380468946DDE90201FDF7F6FA0B
:1014C00042464B46FDF73EF9CDE9040150465946E8
:1014D00064E700BFAFF300800000601A61B4D03D44
:1014E0007370032E8A19A33B83C8C96D305FE43F34
:1014F00000004054FB21F93F3163621A61B4D03DD2
:101500000000002E8A19A33BC14920259A837B390C
:10151000D49D0508549D0508FDF716F942F2FB130A
:10152000C3F6F9739C42804689461AD01EA3D3E9BC
:101530000023FDF709F90D4604462B462246C7E96C
:10154000004540464946FDF7FDF817A3D3E90023BF
:10155000FDF7FAF84FF0FF35C7E90201B7E60324BB
:1015600095E613A3D3E90023FDF7EEF812A3D3E920
:10157000002380468946FDF7E7F80D4604462B46D2
:101580002246C7E9004540464946FDF7DBF80AA375
:10159000D3E90023FDF7D8F84FF0FF35C7E9020182
:1015A00095E6DDE906AB03E73163621A61B4D03D2D
:1015B0000000601A61B4D03D7370032E8A19A33BFA
:1015C0002DE9F84353EC102B00242546C7F6F074A0
:1015D000C7F6F0751C40AC422DED028BB0EE408A90
:1015E000F0EE608A1946104600F0AB80002B7FDDDC
:1015F0001A1500F08980A2F57E7721F07F4323F44D
:101600007003073FD20743F4801366D5C20F4FF033
:10161000000C02EB43037F104200654616204FF496
:1016200000116C18D60F9C424FEA420202DC65188A
:101630001B1B8C444908013806EB4303F1D12026DB
:1016400080464FF0004107E043D0D40F49085200D4
:10165000013E04EB43031BD0AB4208EB0104F3DD76
:1016600004F00049B9F1004F04EB01082BD0A94662
:101670009442C5EB0303C4EB020288BF013B401850
:10168000D40F49085200013E4D4604EB4303E3D119
:101690001A4327D146084FEA6C0101F17E511CF034
:1016A000010F01F5C00118BF46F0004601EB0753DA
:1016B000324643EC182BB0EE480AF0EE680ABDEC57
:1016C000028BBDE8F883B8F1000FD0DB05F101090A
:1016D000CEE79442C4D91D46B7E7C20F02EB4303DD
:1016E000400093E7431C39D000F001031818D1E7FC
:1016F00023F000441443DED0002B36D11A46C10A31
:10170000153A40050029FAD011F4801329D1490077
:101710000133CC02FBD5C3F10105C3F1200420FA4B
:1017200004F4521921439840A2F57E7721F07F43BB
:1017300023F47003073FD20743F480133FF566AFED
:10174000CBE751EC100BFDF7B1F902460B4651EC1B
:10175000180BFCF7F9FF41EC180BACE70CF1010C8E
:1017600099E7202401250023D9E751EC100B0B4603
:10177000FCF7E8FF02460B46FDF7C2FA41EC180BF6
:1017800099E700BF000000002DE9F04F5BEC10ABC3
:101790002DED028BB0EE418AF0EE618A2BF0004411
:1017A000B4F1795F85B071DA50465946FDF718FCFF
:1017B000002800F0FD8052465B4650465946FDF732
:1017C00075F981A3D3E9002306460F46FDF76EF9AC
:1017D0007FA3D3E90023FCF7B7FF32463B46FDF772
:1017E00065F97DA3D3E90023FCF7ACFF32463B4605
:1017F000FDF75CF97AA3D3E90023FCF7A5FF324695
:101800003B46FDF753F978A3D3E90023FCF79AFF91
:1018100032463B46FDF74AF975A3D3E90023FCF7AE
:1018200093FF32463B46FDF741F980468946002347
:101830000022C3F6E07330463946FDF737F94246D9
:10184000CDE900014B4630463946FDF72FF953EC00
:10185000182B04460D4650465946FDF727F9024617
:101860000B4620462946FCF76DFF02460B46DDE994
:101870000001FCF767FF0B4600210246C3F6F0713A
:101880000020FCF75FFF41EC100B83E052465B4603
:1018900050465946FDF70AF94BA3D3E90023064603
:1018A0000F46FDF703F94AA3D3E90023FCF74CFFE9
:1018B00032463B46FDF7FAF847A3D3E90023FCF78D
:1018C00041FF32463B46FDF7F1F845A3D3E900233B
:1018D000FCF73AFF32463B46FDF7E8F842A3D3E96E
:1018E0000023FCF72FFF32463B46FDF7DFF840A30D
:1018F000D3E90023FCF728FF3B463246FDF7D6F834
:1019000043F23233C3F6D3739C42804689468EDD60
:101910000023C3F6E9739C4241DC0021A4F50013C7
:1019200000220020C3F6F07114461D46FCF70AFFA2
:10193000CDE9020100230022C3F6E07330463946A8
:10194000FDF7B4F822462B46FCF7FCFE4246CDE9F3
:1019500000014B4630463946FDF7A8F853EC182BEA
:1019600004460D4650465946FDF7A0F802460B4680
:1019700020462946FCF7E6FE02460B46DDE900015B
:10198000FCF7E0FE02460B46DDE90201FCF7DAFE59
:1019900041EC100B05B0BDEC028BBDE8F08F9FED64
:1019A000067B00258DED027B0024C3F6D275C1E7CE
:1019B0009FED030BEEE700BF000000000000E73FD3
:1019C000000000000000F03FD43888BEE9FAA8BD4E
:1019D000C4B1B4BD9EEE213EAD529C804F7E923E7E
:1019E0009015CB19A001FA3E7751C1166CC1563F34
:1019F0004C5555555555A53F2DE9F04F4AF6AB25A9
:101A0000ADF51B7DD41EC2F6AA2585FB0465E4173F
:101A1000A49F114E0690C4EBA50424EAE47456F882
:101A200027600A941F46E34303EB43037C1E02EB4B
:101A3000C30314EB0608099602940891079321D476
:101A40000A9EA599351B08F101080CAE4FEA8808DB
:101A5000002401EB85090BE0DC9E050859F8040021
:101A6000FCF7BEFF043401354445E6E9020109D024
:101A7000002DF3DA04340020002101354445E6E965
:101A80000201F5D1099C002C2CDB099C5EAE06EB13
:101A9000C4060DF5B87ABB460096029D002DC0F233
:101AA00054820EA9069D01EBCB064FF000084FF0C3
:101AB0000009002476E90223F5E80201FCF7F6FFAD
:101AC00002460B4640464946FCF73EFE0134BC4206
:101AD00080468946EED1EAE90289009DAA450BF1CC
:101AE000010BDAD1099E731E9B0086AC9AAD04EB04
:101AF0008604ED180B9300960C940D95009C009EA7
:101B0000E4009AAD2B19002E049453E93C892EDD94
:101B100004995EAC059485AE651800230022C3F6D7
:101B2000706340464946FCF7C1FFFDF759FAFCF7E0
:101B300057FF00230022C4F2701382468B46FCF745
:101B4000B5FF02460B4640464946FCF7FBFDFDF754
:101B500047FA044646F8044F75E9020152465B46CF
:101B6000FCF7F2FD059CA54280468946D5D149EC9B
:101B7000108B079800F010FE55EC104B00224FF030
:101B80007F5320462946FCF791FF41EC100BFEF7EE
:101B900053FF002351EC100B0022C4F22003FCF78A
:101BA00085FF02460B4620462946FCF7CBFD0D4635
:101BB0000446FDF715FA0646FCF712FF02460B46EF
:101BC00020462946FCF7BEFD079D002D804689462C
:101BD00040F3C180009C9AAD621E05EB8202079C17
:101BE00052F8503CC4F1180043FA00F101FA00F039
:101BF0001B1AC4F11700761842F8503C43FA00F55E
